:020000040000FA
:100000000EEF00F0FFFFFFFF83EF14F0FFFFFFFF95
:10001000FFFFFFFFFFFFFFFF82EF1EF01BEF12F05D
:10002000D86F0001D839E842070BD8B402D01F0EB0
:10003000D86F0A0EC06FD8518FEC1CF0D76F0A0E24
:10004000BC6FD851A2EC1DF0D66F01017205D8B477
:1000500003D07351D8A45FD00001D751D8B41FD0BA
:10006000420EC26FF10EC36F0A0EC46F030EC56F4E
:10007000D7510A0FC66F4D0EC76F010EC86F000E25
:10008000C96F000ECA6F000ECB6F000ECC6F000E52
:10009000CD6F6000D8F3CEF0C0EC06F01DD0420E5C
:1000A000C26FF10EC36F0A0EC46F030EC56F140E3C
:1000B000C66F4D0EC76F010EC86F000EC96F000EE0
:1000C000CA6F000ECB6F000ECC6F000ECD6F6000BC
:1000D000D8F3CEF0C0EC06F0420EC26FF10EC36F43
:1000E0000A0EC46F030EC56FD6510A0FC66F5A0EA3
:1000F000C76F010EC86F000EC96F000ECA6F000EE9
:10010000CB6F000ECC6F000ECD6F6000D8F3CEF039
:10011000C0EC06F03BD0420E0001C26FF10EC36F7F
:100120000A0EC46F030EC56F140EC66F4D0EC76F57
:10013000010EC86F000EC96F000ECA6F000ECB6FA4
:10014000000ECC6F000ECD6F6000D8F3CEF0C0EC87
:1001500006F0420EC26FF10EC36F0A0EC46F030E9B
:10016000C56F140EC66F5A0EC76F010EC86F000E12
:10017000C96F000ECA6F000ECB6F000ECC6F000E61
:10018000CD6F6000D8F3CEF0C0EC06F00A0EC26F5F
:10019000D40EC36F110EC46F050EC56F600060F3FF
:1001A000C6F0340EC76F010EC86F000EC96F000E87
:1001B000CA6F000ECB6F000ECC6F000ECD6F6000CB
:1001C000D8F3CEF0C0EC06F0120012EC1BF0E806FB
:1001D000D8A403D0010E0101E46F3E01F8B1120072
:1001E0000101E405D8A41200000EE46F304B312B5E
:1001F000B5D0FF0E0001C06F0F0EC16FDCEC1EF01A
:10020000C051BC17C151BD17BC5102017F2700016D
:10021000BD5102018023080E010130193111D8A40B
:100220001200000EAA6E010EA7EC1EF00101E56F90
:100230006000FCF9C0F0600000FAC1F00001D89045
:10024000C133C033D890C133C033D890C133C03329
:10025000600000F37DF2600004F37EF27DC27FF265
:100260007EC280F2000E0101316F010E306F010E6F
:10027000EA6F1200FF0E0001C06F0F0EC16FDCECC1
:100280001EF0C051BC17C151BD17BC5102017B27E4
:100290000001BD5102017C23040E0101301931110E
:1002A000D8A41200000EAA6E1B0EA7EC1EF00101CE
:1002B000E56F6000ECF9C0F06000F0F9C1F00001FA
:1002C000D890C133C033D890C133C033600000F33D
:1002D00079F2600004F37AF279C27BF27AC27CF29E
:1002E000000E0101316F010E306F010EE96F120037
:1002F000FF0E0001C06F0F0EC16FDCEC1EF0C0518D
:10030000BC17C151BD17BC51020177270001BD5177
:1003100002017823020E010130193111D8A4120014
:10032000000EAA6E200EA7EC1EF00101E56FD8901A
:10033000020178310001C06F02017731756F6000F2
:1003400000F376F275C277F276C278F2000E010100
:10035000316F010E306F010EE86F1200E551010A96
:10036000D8B488D71A0AD8B4C3D73B0AD8A4120085
:1003700040D7D76F480E0001D619D8A41ED00F0E53
:10038000C26FFD0EC36F0C0EC46F010EC56F020E5F
:10039000C66F5A0EC76F070EC86F000EC96F000EEA
:1003A000CA6F000ECB6F000ECC6F000ECD6F6000D9
:1003B000D8F3CEF0C0EC06F043D05A0ED619D8A42C
:1003C0001ED00F0EC26FFD0EC36F0C0EC46F010E58
:1003D000C56F010EC66F5A0EC76F070EC86F000EAD
:1003E000C96F000ECA6F000ECB6F000ECC6F000EEF
:1003F000CD6F6000D8F3CEF0C0EC06F021D0780EBF
:10040000D619D8A41DD00F0EC26FFD0EC36F0C0EEF
:10041000C46F010EC56F000EC66F5A0EC76F070E70
:10042000C86F000EC96F000ECA6F000ECB6F000EB2
:10043000CC6F000ECD6F6000D8F3CEF0C0EC06F0AC
:10044000480ED719D8A41ED00F0EC26FFD0EC36F71
:100450000C0EC46F010EC56F020EC66F3F0EC76F44
:10046000070EC86F000EC96F000ECA6F000ECB6F6B
:10047000000ECC6F000ECD6F6000D8F3CEF0C0EC54
:1004800006F01200540ED719D8A41ED00F0EC26F5A
:10049000FD0EC36F0C0EC46F010EC56F030EC66F49
:1004A0003F0EC76F070EC86F000EC96F000ECA6FF0
:1004B000000ECB6F000ECC6F000ECD6F6000D8F336
:1004C000CEF0C0EC06F01200780ED719D8A41200B6
:1004D0000F0EC26FFD0EC36F0C0EC46F010EC56F01
:1004E000000EC66F5A0EC76F070EC86F000EC96F99
:1004F000000ECA6F000ECB6F000ECC6F000ECD6FDA
:100500006000D8F3CEF0C0EC06F012000001BC6F22
:10051000A7D0000E01019C6F000E9B6F000E9A6F1A
:10052000000E996F000E986F000E976F000E966F79
:10053000000E956F000E8C6F000E8B6F000E8A6F91
:10054000000E896F000E886F000E876F000E866F99
:10055000000E856F000E946F000E936F000E926F69
:10056000010E916F000E846F000E836F000E826F7C
:10057000010E816F000E096F08693F68030E346E2B
:100580003368030E0B6F0A6976D0010E01019C6F70
:10059000010E9B6F000E9A6F010E996F000E986FFF
:1005A000000E976F000E966F000E956F010E8C6F08
:1005B000010E8B6F000E8A6F010E896F000E886F1F
:1005C000000E876F000E866F000E856F000E946F11
:1005D000010E936F000E926F000E916F000E846FEC
:1005E000010E836F000E826F000E816F000E096F87
:1005F000E60E086F630E3F6E000E346E630E2AD057
:10060000010E01019C6F000E9B6F010E9A6F010E8F
:10061000996F000E986F000E976F000E966F000E88
:10062000956F010E8C6F000E8B6F000E8A6F010E9E
:10063000896F000E886F000E876F000E866F000EA8
:10064000856F000E096F000E086F4D0E3F6E000E95
:10065000346E3D0E336E000E0B6F3D0E0A6F0BD0E5
:100660000001BC51010AD8B454D7030AD8B48DD7BD
:10067000010AD8B4C5D700017A51335C7B51345894
:10068000D8B009D0AE05D8B403D0AF05D8A403D0F4
:10069000010E0101506F0001BC5112000101E20581
:1006A000D8A41FD035AD02D0010E01D0000E02013A
:1006B0008B6FA7EC1AF0D86FD85101016119D8B42B
:1006C00005D0600060F361F1010E766F6005D8A47B
:1006D00006D0230E48ECF2F0000E0101606F000E10
:1006E000E26F5550D8A464D05450D8A461D0535070
:1006F000D8A45ED0010E0001C96F230EC3ECE9F04F
:100700000201C56F010E566E000E0001D96F0ED0AA
:10071000D951600FD96EDA6AC60ED925E16EE26A48
:10072000020EE2226F007FFFE7FFD92B0201C551C5
:100730000001D95DD8A0ECD7040E5518D8A402D07A
:10074000010E556E040E5418D8A402D0010E546E3A
:10075000040E5318D8A402D0010E536E000E566E2C
:10076000000EDA6F11D0C50E0001DA25D96EDA6AF3
:10077000020EDA22B00EDA25E16EE26A020EE22201
:100780006F007FFFE7FFDA2BDA510201C55DD8B0B9
:10079000EAD75504D8A402D0020E556E5404D8A44A
:1007A00002D0020E546E5304D8A402D0020E536E2F
:1007B0000201665104E1C80E655DD8A00BD0000EA1
:1007C0000001AE6F000E0101BD6F000E0201666FE9
:1007D000000E656F0001AE51D8A41200000E7B6FB1
:1007E000000E7A6F000E0201936F000E366E000E3F
:1007F000356E010E0101AA6F000E616F010E766F5A
:100800001200C46F0001C451D8A4BFAF22D0600051
:10081000F0F2C0F06000F4F2C1F06000F8F2C2F053
:100820006000FCF2C3F0C01FC11FC21FC31FC02B5A
:10083000000EC123C223C323600000F3C6F0600092
:1008400004F3C7F0600008F3C8F060000CF3C9F0CF
:100850000CD06000F0F2C6F06000F4F2C7F0600067
:10086000F8F2C8F06000FCF2C9F0BC51BD11BE1135
:10087000BF11D8A409D0000EBC6F000EBD6F000ED2
:10088000BE6F000EBF6F1200960EC56F06D0C52B4F
:10089000D890C933C833C733C633000EC615C06FEE
:1008A000000EC715C16F000EC815C26FFE0EC91528
:1008B000C36FC051C111C211C311D8B40DD0E7D755
:1008C000C52B010EC627000EC723C823C923D89005
:1008D000C933C833C733C633000EC615C06F000E08
:1008E000C715C16F000EC815C26FFF0EC915C36FC3
:1008F000C051C111C211C311D8B407D0E1D7C50787
:10090000D890C637C737C837C937C8BF03D0020E1B
:10091000C561F5D7C5A1C89FD890C533600014F351
:10092000C0F0C16BC26BC36B600000F3C3F0C26B5D
:10093000C16BC06BC051C613C151C713C251C8139C
:10094000C351C913C451D8A4BFAF01D0C98F60002F
:1009500018F3BCF060001CF3BDF0600020F3BEF0A3
:10096000600024F3BFF01200010E0001B46F010E0D
:100970000101D56F000E0201746F000E736F000E3F
:100980000101CF6F3D0178B103D03901A2AF12D080
:100990006F00A8F502F03901A29F3D0177A70AD0A8
:1009A000522AE60E5224D96EDA6A030EDA22600069
:1009B0000BF0DFFF3D0177A966D079A50FD07995BF
:1009C0003901A3933D0178856C69000E766F000EA6
:1009D000526E010E0101CF6F000EE66F3D0176A948
:1009E00006D076993901A3953D01788545D0390126
:1009F000A3A142D0A3913D017851522A0101D4050F
:100A0000D8A40BD0DA0E5224D96EDA6A030EDA2299
:100A1000DF503D016B6F010E0DD05604D8A40CD0F1
:100A2000CE0E5224D96EDA6A030EDA22DF503D016F
:100A30006B6F020E0101E66F5204D8A41DD0600056
:100A400054F101F0030E0116D8B403D0010ED36F98
:100A500013D0600050F101F0030E0116D8B403D09A
:100A6000010ED26F09D060004CF101F0030E0116A7
:100A7000D8B402D0010ED16F3D0179A723D0799768
:100A80003901A3931FD079A706D079973901A39391
:100A9000000E526E17D079A515D0000E796F39016E
:100AA000A3933D0178856C69000E766F010E0101FC
:100AB000D06F600048F1E6F3000E526E010ECF6F6A
:100AC000000EE66F3D017399120060006CF102F3B5
:100AD0000301036B600068F104F3056BB0C006F31B
:100AE000076B92C008F3096B600020F10AF30B6BEF
:100AF000B2C00CF30D6B600008F10EF30F6B000138
:100B0000B751BC6FBD6B060ED890BC37BD37E82E11
:100B1000FBD7B851BE6FBF6B050ED890BE37BF373D
:100B2000E82EFBD740501F0BC06FC16BBE51C027D2
:100B3000BF51C123BC51C0250301106F0001BD513D
:100B4000C1210301116F00018851BC6FBD6B070EFD
:100B5000D890BC37BD37E82EFBD78B51BE6FBF6B2B
:100B6000060ED890BE37BF37E82EFBD78751C06F2F
:100B7000C16B050ED890C037C137E82EFBD70101F5
:100B800046510001C26FC36BC23BC33BF00EC3179B
:100B9000C2510F0BC313F00EC2178551C46FC56B42
:100BA000D890C437C537D890C437C537D890C43724
:100BB000C5378E51070BC66FC76BC451C627C551C9
:100BC000C723C251C627C351C723C051C627C1512D
:100BD000C723BE51C627BF51C723BC51C625030139
:100BE000126F0001BD51C7210301136F78C016F3C6
:100BF00079C017F374C018F375C019F36000DCF006
:100C00001AF36000E0F01BF300019A05D8A405D0A8
:100C100072C01CF373C01DF305D0000E03011D6FDD
:100C2000000E1C6F000E506E1200600008F3C9F039
:100C300060000CF3C8F0C15104E1020EC05DD8A001
:100C400042D0C0B140D05A0EC419D8A43CD06000E4
:100C500000F3BCF0600004F3BDF0FBEC1EF00001FB
:100C6000C919D8B418D0600000F3BCF0600004F3D8
:100C7000BDF0600024F3BEF097EC1BF0FF0E000106
:100C8000C025BC6FFF0EC121BD6F600010F3BEF028
:100C900097EC1BF01200FF0EC025BC6FFF0EC121A8
:100CA000BD6FFBEC1EF00001C419D8B41200FF0E9A
:100CB000C025BC6FFF0EC121BD6F600010F3BEF0F8
:100CC00097EC1BF01200C15104E1210EC05DD8A0C9
:100CD00012005B0EC419D8A41200010EC025BC6F0F
:100CE000000EC121BD6FFBEC1EF00001C56F080EA8
:100CF000C527600000F3BCF0600004F3BDF0FBEC1E
:100D00001EF00001C66FC76BC52B03D0D890C63745
:100D1000C737C52FFBD70001C251C61904E1C35123
:100D2000C719D8B424D0600000F3BCF0600004F30D
:100D3000BDF0600020F3BEF097EC1BF0010E000147
:100D4000C025BC6F000EC121BD6F600024F3BEF052
:100D500097EC1BF0FF0E0001C025BC6FFF0EC121F8
:100D6000BD6F600010F3BEF097EC1BF01200FF0E99
:100D7000C025BC6FFF0EC121BD6FFBEC1EF093D7E9
:100D8000000ED46FCE05D8A402D01E0EC727010EC8
:100D9000D56F9AD0BB98BB9AD551C825AF0F26EC1A
:100DA0001FF0BB8A0001CE05D8A40FD0BB98BB9A18
:100DB000C7510F0B26EC1FF0BB8ABB9A0001C73945
:100DC0000F0B100F26EC1FF00ED0BB98BB9AC73943
:100DD0000F0B100F26EC1FF0BB8ABB9A0001C75106
:100DE0000F0B26EC1FF0BB8ABB88000E0001D36FEF
:100DF00066D0C651C503D551CF6FD06BF350CF2706
:100E0000F450D023FF0ECF25BC6FFF0ED021BD6F55
:100E1000600010F3BEF0BF6B49EC1DF0D351C2254A
:100E2000D16F000EC321D26FBC51D127BD51D22347
:100E3000600047F3F6FF60004BF3F7FF000EF86E1B
:100E400008006F00D4FFD4F0600030F3CFF0030E41
:100E5000CF17600050F3D0F0CF2B02D0D890D03312
:100E6000CF2FFCD70001D051D46F600034F3CFF006
:100E7000030ECF17600050F3D0F0CF2B02D0D890E4
:100E8000D037CF2FFCD70001D051D46FC905D8A4DB
:100E900004D0C551D519D8B4D48FCA05D8A403D06D
:100EA000D505D8B4D481CB05D8A402D0FF0ED41B6D
:100EB000BB9AD45126EC1FF0BB8A0001D32BC4513E
:100EC000D35DD8A096D7D52BD551C55DD8B062D704
:100ED000BB881200D66F96D04D0EC26FFA0EC36F4C
:100EE0000B0EC46F010EC56F020EC66F3F0EC76FAB
:100EF000000EC86F010EC96F000ECA6F000ECB6FD7
:100F0000000ECC6F000ECD6F6000D8F3CEF0C0ECB9
:100F100006F012004D0EC26FFA0EC36F0B0EC46FB7
:100F2000010EC56F030EC66F3F0EC76F000EC86F70
:100F3000010EC96F000ECA6F000ECB6F000ECC6F92
:100F4000000ECD6F6000D8F3CEF0C0EC06F01200BA
:100F50004D0EC26FFA0EC36F0B0EC46F010EC56F3C
:100F6000040EC66F3F0EC76F000EC86F010EC96F2B
:100F7000000ECA6F000ECB6F000ECC6F000ECD6F4F
:100F80006000D8F3CEF0C0EC06F012004D0EC26F38
:100F9000FA0EC36F0B0EC46F010EC56F050EC66F40
:100FA0003F0EC76F000EC86F010EC96F000ECA6FEB
:100FB000000ECB6F000ECC6F000ECD6F6000D8F32B
:100FC000CEF0C0EC06F012004D0EC26FFA0EC36FE9
:100FD0000B0EC46F010EC56F000EC66F3F0EC76FBC
:100FE000000EC86F010EC96F000ECA6F000ECB6FE6
:100FF000000ECC6F000ECD6F6000D8F3CEF0C0ECC9
:1010000006F012000001D651000AD8B4BFD7210A59
:10101000D8B49ED7630AD8B47DD7260AD8B45CD793
:10102000D3D7D76F020E0101EB6F60005CF3ECF1D8
:1010300067D0600030F3EDF1030E34D0CC51CD25F4
:10104000D56FD5290101ED6F600038F3EEF1040E84
:101050000001D86FCD05D8A405D0600040F3EFF1B2
:10106000050ED86F020ECD19D8A408D060003CF34D
:10107000EFF1600040F3F0F1060ED86F030ECD19CA
:10108000D8A452D060003CF3EFF1600040F3F0F1DF
:10109000600044F3F1F1070E05D0000E0101ED6F81
:1010A000030E2CD0D86F40D0010E0101ED6F60000F
:1010B00040F3EEF1040E0001D86FD105D8A034D072
:1010C0000101ED2B600044F3EFF1050E17D0010E86
:1010D000E5D7020E0101ED6F600048F3EEF160000C
:1010E0004CF3EFF1050E0001D86FD405D8A01CD049
:1010F0000101ED2B600050F3F0F1060E0001D2D794
:101100000001D751000AD8B494D7010AD8B496D7B1
:10111000040AD8B4C2D70D0AD8B4C6D7010AD8B4C5
:10112000D8D7180AD8B4D3D7600028F3C1F060002C
:101130002CF3C2F06000B4F7C3F0600060F3C4F0B9
:1011400052EC10F0D66F600058F3BCF00101EB5187
:10115000CDEC1DF01200000ED06F600024F3C2F041
:10116000600028F3C3F0030EC56FE80EC46FB0EC47
:1011700019F0C251D26F600048F3BCF0BD6BFC0E99
:10118000BF6F180EBE6F49EC1DF0C951BC25C26F70
:10119000CA51BD21C36F000EC56F640EC46FB0ECA1
:1011A00019F0C251D16F600048F3BCF0BD6BFC0E6A
:1011B000BF6F180EBE6F49EC1DF06000F0F2CCF06E
:1011C0006000F4F2CDF0600044F3BCF0BD6BFF0EA4
:1011D000BF6F9C0EBE6F49EC1DF0BC51CC27BD51BA
:1011E000CD23C951CC25C26FCA51CD21C36F000E8A
:1011F000C56F0A0EC46FB0EC19F0C251CF6FD25157
:10120000180D6F00CCFFCCF0D1519C0D6F00CCFFBE
:10121000CDF0CF51F60DF350CD25CC25C925CE6F9D
:10122000540ECB19D8B404D0740ECB19D8A404D062
:10123000600048F3D0F022D0480ECB19D8B404D0C7
:10124000680ECB19D8A404D0600044F3D0F016D0B7
:101250005A0ECB19D8B404D07A0ECB19D8A404D026
:1012600060003CF3D0F00AD0450ECB19D8B403D0BF
:10127000650ECB19D8B4600038F3D0F0D05112000D
:101280001C6E020E0101EB6F600070F0ECF15BD0A0
:10129000600044F0EDF1030E54D0115012241A6E88
:1012A0001A28ED6F60004CF0EEF1040E1D6E120472
:1012B000D8A405D0600054F0EFF1050E1D6E020EAB
:1012C0001218D8A408D0600050F0EFF1600054F07C
:1012D000F0F1060E1D6E030E1218D8A447D0600060
:1012E00050F0EFF1600054F0F0F1600058F0F1F1CF
:1012F000070E27D0000EED6FCED7010EED6F600008
:1013000054F0EEF1040E1D6E1604D8A02FD0ED2B74
:10131000600058F0EFF1050E14D0010EECD7020E6C
:10132000ED6F60005CF0EEF1600060F0EFF1050E33
:101330001D6E1904D8A01AD0ED2B600064F0F0F1F6
:10134000060E1D6E13D01C50000AD8B4A1D7010A96
:10135000D8B4A3D7040AD8B4CDD70D0AD8B4CDD702
:10136000010AD8B4DCD7180AD8B4D7D760003CF04B
:1013700006F0600040F007F06000B4F708F060008D
:1013800074F009F0A3EC10F01B6E60006CF001F03B
:101390000101EB5134EC1EF01200216E79D04E04A5
:1013A000D8A412005604D8A414D0000E0201AC6FC9
:1013B000000EAD6F3E0EAE6F000EAF6F000EB06F41
:1013C000AC0E1E6E020E1F6E050E206ED8EC1BF0CA
:1013D00013D0000E0201C16F000EC26F3E0EC36F2C
:1013E000000EC46F000EC56FC10E1E6E020E1F6E82
:1013F000050E206ED8EC1BF0050E0201886F100E52
:10140000876F12004E04D8A4120018C237F119C217
:1014100036F16000D8F45AF06000DCF45BF0010EA5
:101420000101B46F010E4F6E5604D8A417D06000AE
:101430006CF1ACF2600068F1ADF23F0E0201AE6FEC
:10144000600068F1AFF2000EB06FAC0E1E6E020EBF
:101450001F6E050E206ED8EC1BF016D060006CF1EC
:10146000C1F2600068F1C2F23F0E0201C36F60007A
:1014700068F1C4F2000EC56FC10E1E6E020E1F6E23
:10148000050E206ED8EC1BF0050E0201886F1200CD
:101490002150220AD8B41200010AD8B412000D0A51
:1014A000D8B47DD7010AD8A41200ACD70101E90550
:1014B000D8A454D06000E4F9EDF06000E8F9EEF053
:1014C000CBEC17F06000B4F30CF16000B8F30DF151
:1014D000010E01015D6F5C51D8A40ED0000EBF6FEC
:1014E000000EBE6F600030F4BCF0600034F4BDF05C
:1014F000DBEC19F0010113D0010EBF6F270EBE65A2
:1015000023D0000EBE6F0DD0000E09D0640E07D0A0
:10151000500E05D03C0E03D0280E01D0140E5E6F85
:1015200013D05F51000AD8B4F9D7140AD8B4F4D74D
:101530003C0AD8B4EFD7140AD8B4EAD76C0AD8B4A6
:10154000E5D7340AD8B4E0D75F515E19D8B404D0D7
:101550005EC15FF1010E766F000EE96F0001B40508
:10156000D8B403D0AD05D8A406D0010E01015C6F3C
:10157000000E5B6F1200800E01010C5D0C0E0D5908
:10158000D8B014D05C51D8A412005150D8A4120085
:101590000201465104E1650E455DD8A004D0010E5C
:1015A00001015B6F1200454B462B1200000E5C6F71
:1015B000000E5B6F12000101EA05D8A41200600062
:1015C000F4F9EDF06000F8F9EEF094EC17F060003B
:1015D000B4F31AF16000B8F31BF1010E01017D6F45
:1015E000600068F4EFF060006CF4F0F01AC151F2A2
:1015F0001BC152F2A10E0001EF5D0F0EF059D8A0F1
:1016000002D0000E4FD0B90EEF5D0B0EF059D8B0DE
:10161000F8D7D10EEF5D070EF059D8A002D0640EB6
:1016200041D0E90EEF5D030EF059D8A002D05A0E5A
:1016300039D0590EEF5D020EF059D8A002D0500EED
:1016400031D0C30EEF5D010EF059D8A002D04B0E81
:1016500029D02D0EEF5D010EF059D8A002D0400E1A
:1016600021D0F05104E1A10EEF5DD8A002D0320EDE
:1016700019D0F05104E16F0EEF5DD8A002D0300E0A
:1016800011D0F05104E15B0EEF5DD8A002D0200E26
:1016900009D0F05104E1470EEF5DD8A002D0190E39
:1016A00001D0100E4B6E0101A705D8A405D02F0E56
:1016B0004B6402D0000E4B6E000EEA6F1200000E5B
:1016C0000001C06F000EC16F010EC26FC251020D4A
:1016D0002A0EF324D96E020EF420DA6EBC51DE1805
:1016E00007E1BD51DE18D8A403D0010EC06F12D09F
:1016F000C251020D2A0EF324D96E020EF420DA6EC6
:10170000DE50DE10D8B4600008F3C1F0C22B050E25
:10171000C265DCD7C051D8A41200C151D8B43FD0A3
:10172000C151020D2A0EF324D96E020EF420DA6E96
:101730006000F3F2DEFF6000F7F2DDFF600004F30B
:1017400053F112006000F0F22EF26000F4F22FF27A
:10175000020E536F12006000F0F230F26000F4F2FB
:1017600031F2030E536F12006000F0F232F26000AB
:10177000F4F233F2040E536F12006000F0F234F210
:101780006000F4F235F2050E536F12006000F0F2C3
:101790002CF26000F4F22DF2010E536F12000101E1
:1017A0005351010AD8B4CED7030AD8B4D4D7010A0A
:1017B000D8B4DAD7070AD8B4E0D7010AD8A41200FF
:1017C000E5D7000EE76F000EE86F63D0600EC26FC2
:1017D000E50EC36F070EC46F020EC56FE851D62524
:1017E000E06F000ED721E16F600083F3F6FF600029
:1017F00087F3F7FF000EF86E0800F550E00FC66F94
:10180000E751FC0D6F00CCFFE2F0E851080DF350FA
:10181000E225D925C76F600068F3C8F060006CF35B
:10182000C9F0600070F3CAF0600074F3CBF06000A0
:1018300078F3CCF060007CF3CDF06000D8F3CEF00C
:10184000C0EC06F0E851D625E06F000ED721E16F1D
:10185000600083F3F6FF600087F3F7FF000EF86E79
:101860000800F550490AD8B412D0E851D625E06FE7
:10187000000ED721E16F600083F3F6FF600087F36D
:10188000F7FF000EF86E0800F550690AD8B4E72B90
:10189000E82BFF0EE06FFF0EE16FD851E26FE36BB4
:1018A000E051E227E151E323E851E46FE56BE251B7
:1018B000E45DE551800AE66FE351800AE659D8B04D
:1018C000120084D7216E050E0201176506D00C0E9A
:1018D0001C6103D01CC200F202D0000E006F005148
:1018E000D8B462D0010E226E10D01C0E2224D96E04
:1018F000DA6A020EDA22000E2224E16EE26A020E99
:10190000E2226F007FFFE7FF222A2250005DD8B05D
:10191000ECD7010E0101606F47D04D50D8A44D06A1
:101920005604D8A415D060006CF1ACF2600068F1E8
:10193000ADF2310E0201AE6F34C1AFF2AC0E1E6ECD
:10194000020E1F6EB051050F206ED8EC1BF014D0A4
:1019500060006CF1C1F2600068F1C2F2310E020168
:10196000C36F34C1C4F2C10E1E6E020E1F6EC5518C
:10197000050F206ED8EC1BF05550D8B411D00F0EC7
:101980000201CA17CAC2B5F23F0EC6171C0EC7170E
:101990001C0EC8173F0EB1171C0EB2171C0EB31742
:1019A0000B0E0201886F12002150210AD8B4B5D75E
:1019B000030AD8B41200010A1200BC6F05D0000E51
:1019C00001D0010EBD6F66D00001BC51000AD8B431
:1019D000F6D70A0AD8B4F3D7010AD8B4F0D7070A61
:1019E000D8B4EDD7010AD8B4EAD7030AD8B4E7D7F8
:1019F000010AD8B4E4D71F0AD8B4E1D7010AD8B491
:101A0000DED70F0AD8B4DBD7010AD8B4D8D73F0A3B
:101A1000D8B4D5D7010AD8B4D2D7030AD8B4CFD70F
:101A2000010AD8B4CCD70B0AD8B4C9D7010AD8B4A4
:101A3000C6D7030AD8B4C3D7010AD8B4C0D7070A97
:101A4000D8B4BDD7010AD8B4BAD7030AD8B4B7D727
:101A5000010AD8B4B4D71C0AD8B4B1D7070AD8B48D
:101A6000AED7010AD8B4ABD70C0AD8B4A8D7780A35
:101A7000D8B4A5D7030AD8B4A2D7010AD8B49FD73F
:101A8000080AD8B49CD7070AD8B499D7010AD8B4A1
:101A900096D797D7BD511200C76F0001C005D8A4D3
:101AA00002D01E0EBE27010ECA6F5CD0BB98BB9A37
:101AB000CA51BF25AF0F26EC1FF0BB8A0001C0053D
:101AC000D8A40FD0BB98BB9ABE510F0B26EC1FF0C9
:101AD000BB8ABB9A0001BE390F0B100F26EC1FF01A
:101AE0000ED0BB98BB9ABE390F0B100F26EC1FF01F
:101AF000BB8ABB9A0001BE510F0B26EC1FF0BB8ABC
:101B0000BB88000E0001C96F28D0000EC86FCA053F
:101B1000D8B4C881BD51CA19D8B4C88FC951D8B476
:101B200014D0C951C16FC26BFF0EC36FFF0EC46FDB
:101B3000C751C56FC66BC351C527C451C623C15118
:101B4000C51904E1C251C619D8B4C869BB9AC851B5
:101B500026EC1FF0BB8A0001C92BC751C95DD8A074
:101B6000D4D7CA2BCA51BD5DD8B0A0D7BB8812004C
:101B70004305D8A418D07E0E0001D66FFF0ED76F94
:101B80000A0ED86F000ED96F070EDA6F000EDB6FEA
:101B9000000EDC6F000EDD6F000EDE6F010EDF6FDA
:101BA000ABECEBF012003E04D8A418D0B30E000149
:101BB000D66FFF0ED76F070ED86F000ED96F070EC6
:101BC000DA6F000EDB6F000EDC6F000EDD6F000EB3
:101BD000DE6F010EDF6FABECEBF012004105D8A415
:101BE00018D0740E0001D66FFF0ED76F0A0ED86F93
:101BF000000ED96F070EDA6F000EDB6F000EDC6F80
:101C0000000EDD6F000EDE6F010EDF6FABECEBF050
:101C10001200F50E0001D66FFE0ED76F0D0ED86FB5
:101C2000000ED96F070EDA6F000EDB6F000EDC6F4F
:101C3000000EDD6F000EDE6F000EDF6FABECEBF021
:101C40001200E535E635EC6FEC51D8A409D0000E52
:101C5000E36F000EE46F000EE56F000EE66F1200FA
:101C600060008CF3E7F0600090F3E8F0600094F31C
:101C7000E9F0600098F3EAF0200E05D0D890EA333E
:101C8000E933E833E733E82EF9D7E751EB6FE58F17
:101C9000FF0EE317FF0EE417FF0EE517000EE61721
:101CA000960EEC5FECAF0DD0EC51800A970FD8A0E8
:101CB000CED7D890E633E533E433E333EC3FF9D7BE
:101CC0000DD01F0EEC6507D0C2D7D890E337E437AC
:101CD000E537E637EC07EC51D8A4F7D7EB51D8B489
:101CE00008D0E61FE51FE41FE36D000EE423E523A3
:101CF000E62360008CF3E3F0600090F3E4F0600012
:101D000094F3E5F0600098F3E6F012000001BC6F78
:101D10000101E605D8B42DD0000ED46F000E0001ED
:101D2000BD6F0ED0BD51600FD96EDA6ADB0EBD25D6
:101D3000E16EE26A030EE2226F007FFFE7FFBD2B38
:101D4000BC51BD5DD8A0EED7040E5518D8A402D062
:101D5000010E556E040E5418D8A402D0010E546E14
:101D6000040E5318D8A402D0010E536E010E0101C7
:101D7000D46F020EE619D8B41200000E566E000E93
:101D80000001BE6F10D0DA0EBE25D96EDA6A030EDE
:101D9000DA22CE0EBE25E16EE26A030EE2226F0069
:101DA0007FFFE7FFBE2BBE51BC5DD8B0ECD755041A
:101DB000D8A402D0020E556E5404D8A402D0020E4C
:101DC000546E5304D8A402D0020E536E010E566E08
:101DD0001200256E600058F824F0000E266E4DD0DB
:101DE0002550D8B40ED02350D8B40BD025500201C2
:101DF0001819D8A408D023501919D8A404D0010E5A
:101E000001D0000E266E02011A51BF0B0101356F81
:101E1000335102011B19D8B407D01BC233F133C1AF
:101E2000A3F1010E01019F6F2604D8A414D0010E66
:101E30000101E26F010EBD6F000E0201666F000E20
:101E4000656F010E0001AE6F010E4F6E010135513D
:101E500062EC0CF004D001013551CDEC09F0130E09
:101E60000101DD25D96EDA6A020EDA22DF50346F05
:101E700011D0010E0001906F0DD02450400AD8B44B
:101E800009D0110AD8B406D0D00AD8B4A9D7040A08
:101E9000D8B4EFD726501200040EBE6E000EBD6EF1
:101EA000010EBA6E500EBB6E980EBC6E030EC66E5F
:101EB000FE0EC26E030EC36E270EC46EFC0EC56E00
:101EC0000C0E3A01706F000E606F040E506F010E21
:101ED000806F020E406FF00E716F040E816F000E66
:101EE000516FFC0E416F070E616F040E826F000E82
:101EF000426F000E526F180E626F030E726F4369CD
:101F0000536963697369070E836F180EE36F210EBF
:101F1000136F220E146F090EE56F130EE16F190E89
:101F2000E46F0B0EDE6F140EE26F040ED96F1F0EFE
:101F30000A6F1E0E0B6F230E186F240E196F050EFD
:101F4000DA6F130E166F160EDF6F12004F04D8A44F
:101F500013D05550D8A410D05450D8A40DD05350FD
:101F6000D8A40AD0020EC96F230EC3ECE9F0030116
:101F7000DA6FDA5186EC0EF00101D005D8A405D055
:101F800068ECFFF0000E0101D06F4E04D8A415D00C
:101F90006651D8A412D0CF05D8A40FD0410E0001AD
:101FA000B519D8B40AD0010EBF6F410EEDEC16F092
:101FB000030E426E000E0001B26F0101AE05D8A4FF
:101FC0001200470E0001B56FB551B5253D016F6F89
:101FD000FE0E706F010E0101B26F000E0201986FCC
:101FE000000E0001AF6F010E0101AD6F000EAE6F6C
:101FF000000E4E6E000E666F1200BD6F000E0001E7
:10200000BF6FBB98BB9ABF51B00F26EC1FF0BB8AC5
:102010000001BD05D8A40AD0BB9A0E0E26EC1FF015
:10202000BB8ABB9A110E26EC1FF009D0BB9A000E9A
:1020300026EC1FF0BB8ABB9A100E26EC1FF0BB8A61
:10204000BB88000E0001BE6FBB9A000E26EC1FF08D
:10205000BB8A0001BE2B650EBE65F6D7BF2B070EEF
:10206000BF65CFD7BB98BB9AB00E26EC1FF0BB8ADA
:102070000001BD05D8A40AD0BB9A0E0E26EC1FF0B5
:10208000BB8ABB9A110E26EC1FF009D0BB9A000E3A
:1020900026EC1FF0BB8ABB9A100E26EC1FF0BB8A01
:1020A000BB881200000EC96F2CD0C951C125C56F65
:1020B000000EC221C66F600017F3F6FF60001BF32D
:1020C000F7FF000EF86EEB0EC76F010EC86FC95117
:1020D000C727000EC823C451C725D96E000EC821DA
:1020E000DA6E1F0EF76403D00800F55007D06F00BA
:1020F000DBFFE1FF6F00DFFFE2FFE750DF6E000173
:10210000C92BC351C95DD8A0D0D7EB0EBC6F010E4F
:10211000BD6FC951C425BE6F0CEC1EF0C56FEB0E30
:10212000C66F010EC76FC951C627000EC723C45121
:10213000C625D96E000EC721DA6E600017F3DFFFE7
:10214000C951C4251200000E0E6E2BD00E5006246D
:102150000A6E000E07200B6E60002BF0F6FF600089
:102160002FF0F7FF000EF86EEB0E0C6E010E0D6EE9
:102170000E500C26000E0D2209500C24D96E000EB4
:102180000D20DA6E1F0EF76403D00800F55007D05B
:102190006F00DBFFE1FF6F00DFFFE2FFE750DF6E64
:1021A0000E2A08500E5CD8A0D1D7EB0E016E010E9E
:1021B000026E0E500924036E48EC1EF00A6EEB0E00
:1021C0000B6E010E0C6E0E500B26000E0C220950E9
:1021D0000B24D96E000E0C20DA6E60002BF0DFFFAE
:1021E0000E5009241200BE6F600020F1BDF0180EE1
:1021F0000001BD17D8B41DD048380F0B010B4A1A87
:102200004A04D8A40CD04950FF0ABD6FBE51BD5D31
:10221000D8A02BD04950BE2729D01F0E05D0495039
:10222000BE5DD8B003D0000EBE6F24D04950BE5F53
:1022300021D048A41FD04A04D8A40FD0BC51D8B490
:10224000E2D7BE51D8A403D0000E0101586F495007
:102250000001BE5DD8A0E7D7E9D7BC51D8A4D3D739
:10226000BE51D8A4F4D7010EF0D7BE691F0EBE65CB
:1022700001D0D3D7000E496EBE511200D96F0A0E9D
:102280000001D76502D00A0ED76FF10EC26FF80EAB
:10229000C36F570EC46F020EC56F010EC66F60008C
:1022A00064F3C7F0600058F3C8F0000EC96F000E69
:1022B000CA6F000ECB6F000ECC6F000ECD6F6000AA
:1022C000D8F3CEF0C0EC06F0CA0EC26FFD0EC36F9D
:1022D000050EC46F020EC56F000EC66FD751080DF4
:1022E000F350D925D86FD829C76F600058F3C8F0CC
:1022F000000EC96F000ECA6F000ECB6F000ECC6FC0
:10230000000ECD6F6000D8F3CEF0C0EC06F0D751D0
:1023100012004A04D8A421D04950BE6FBF6BBE1D25
:10232000C06FBF1DC16FBC51C05DBD51C159D8B098
:1023300003D0BC69BD6904D04950BC27000EBD2341
:10234000BC51335CBD513458D8B024D06000CCF0BF
:10235000BCF06000D0F0BDF01DD0FF0EBE6FFF0ED0
:10236000BF6F6000F0F2C0F06000F4F2C1F0BE5147
:10237000C027BF51C1234950C05D000EC159D8B01C
:1023800005D0000EBD6F010EBC6F04D04950BC5F7C
:10239000000EBD5B000E496E6000F0F2BCF0600004
:1023A000F4F2BDF01200BE6F4A04D8A436D04950F2
:1023B000FF0A0001BD6FBE51BD5DD8B002D0BE693D
:1023C00012D04950BE270FD0050EBE6530D0050E85
:1023D0002AD0030EBE652BD0030E25D0020EBE659B
:1023E00026D0020E20D0BC51640AD8B4EDD70A0A18
:1023F000D8B4EFD7010AD8B4ECD7150AD8B4E9D7C6
:10240000060AD8B4EBD7FE0AD8B4E8D7010AD8B484
:10241000E0D7070AD8B4DDD7D7D70001BE51495C51
:10242000D8A003D0010EBE6F02D04950BE5F000E8F
:10243000496EBE511200140EF66E3E0EF76E000E7F
:10244000F86E00EED8F210EE1CF009006F00D7FF16
:10245000EEFFE550E150F9E1540EF66E3F0EF76ED7
:10246000000EF86E09006F00D4FFF6F000EE00F3E6
:10247000F20EEE6AE806FDE100EE00F2D80EEE6A1A
:10248000E806FDE100EE00F110EE00F1EE6AE55025
:10249000E150FCE1E250FAE100EE60F0590EEE6A24
:1024A000E806FDE100EE2FF02D0EEE6AE806FDE1F4
:1024B000080ED56E000ED66E000ED76E00018BEFA3
:1024C000AAF093970E0E0001BC6F2B0EBD6F000E8D
:1024D000BE6F6EEC1FF0390193995A0E0001BC6F6C
:1024E000390EBD6F000EBE6F64EC1FF0000E3D0193
:1024F000EC6F000EED6F000EEE6F000EEF6F000E32
:10250000F06F000EF16FB00EF26F800EF36F000EE1
:10251000F46F8A0EF56F000EF66F000EF76F000E67
:10252000F86F000EF96F000EFA6F000E586E000E75
:102530000101DA6F150E0201FE6F000E596E000EDA
:102540000101D96F000EDC6F39019387120002017F
:10255000745104E13D0E735DD8A00DD0000E000152
:10256000B46F000E0101666F000ED56F000E020100
:10257000746F000E736F3C0E0101BB651ED0000E20
:10258000BC6F000EBB6F000E0001AF6F010E0101AA
:10259000AD6F000E666F000E416E420E0001B56F0A
:1025A000B551B5253D016F6FFE0E706F010E010133
:1025B000B26F000E4F6E010EAA6F02015B515719E8
:1025C00004E15C515819D8B412005BC257F25CC2E6
:1025D00058F2010E0101A16F1200C96F600024F3CF
:1025E000CAF06000F4F2CBF06000F8F2CCF06000CA
:1025F000FCF2CDF0600000F3CEF0600004F3CFF009
:10260000600008F3D0F060000CF3D1F0600010F32C
:10261000D2F0600014F3D3F0600018F3D4F060003F
:102620001CF3D5F0600020F3D6F0BA90E40E00D091
:1026300000D0E82EFCD700D000D0BA80BB98000EA6
:102640000001D76FBB9AD751CA0FD96EDA6ADF5033
:1026500026EC1FF0BB8A0001D72B0C0ED765F2D7F2
:10266000BB881200EC51FD0DF350360FEE6F600089
:10267000B0F3EDF0FF0EED27EDB1EE2B690EC26F5A
:10268000FC0EC36F660EC46F010EC56F000EC66FE1
:10269000000EC76F010EC86F000EC96F000ECA6F23
:1026A000010ECB6F000ECC6F000ECD6F6000D8F323
:1026B000CEF0C0EC06F06000A8F3D6F06000ACF3FA
:1026C000D7F06000B0F3D8F06000B8F3D9F0010E95
:1026D000DA6F000EDB6F000EDC6F010EDD6F000E97
:1026E000DE6F000EDF6FABECEBF012000001D66F77
:1026F000890E0001C26FF70EC36F0F0EC46F020E7A
:10270000C56FD651020DF350060FC66F4A0EC76F44
:10271000040EC86F000EC96F000ECA6F000ECB6F9B
:10272000000ECC6F000ECD6F6000D8F3CEF0C0EC81
:1027300006F0890EC26FF70EC36F0F0EC46F020E44
:10274000C56FD651020DF350070FC66F590EC76FF4
:10275000040EC86F000EC96F000ECA6F000ECB6F5B
:10276000000ECC6F000ECD6F6000D8F3CEF0C0EC41
:1027700006F01200C06F000E0001C16FC005D8A4A2
:102780002FD0010E0101C36F0001BC51BE6FBF6BA2
:10279000BE510101245D0001BF5101012559D8A09E
:1027A00006D000019705D8A402D0000E12D0000177
:1027B000BD51BE6FBF6BBE510101245D0001BF5111
:1027C00001012559D8A016D000019751D8A412D0E4
:1027D000010E976F000E0101256F000E246F07D0C8
:1027E000000E0101256F000E246F000EC36F010E55
:1027F0000001C16F0001C1511200D66F040E00012B
:10280000D66502D0040ED66F890EC26FF70EC36F65
:102810000F0EC46F020EC56FD629C66F3A0EC76F72
:10282000060EC86F000EC96F000ECA6F000ECB6F88
:10283000000ECC6F000ECD6F6000D8F3CEF0C0EC70
:1028400006F0D70EC26FFC0EC36F050EC46F010EEB
:10285000C56F600058F3C6F04D0EC76F070EC86F06
:10286000000EC96F000ECA6F000ECB6F000ECC6F4A
:10287000000ECD6F6000D8F3CEF0C0EC06F0120071
:10288000D66F040E0001D66502D0040ED66F560E28
:10289000C26FEB0EC36F220EC46F040EC56FD62934
:1028A000C66F220EC76F030EC86F000EC96F000EF1
:1028B000CA6F000ECB6F000ECC6F000ECD6F6000A4
:1028C000D8F3CEF0C0EC06F0420EC26FF10EC36F2B
:1028D0000A0EC46F030EC56FD6510A0FC66F480E9D
:1028E000C76F040EC86F000EC96F000ECA6F000ECE
:1028F000CB6F000ECC6F000ECD6F6000D8F3CEF022
:10290000C0EC06F012006F00D8FF2BF06F00DCFF68
:102910002CF06F00E0FF2DF06F00D4FF2EF0390196
:1029200093B1A3A103D0B4EC04F023D093A302D0BD
:10293000A3B3F9D793B7A3A703D087EC15F019D0A9
:1029400093B9A3A903D0ADEC1CF013D09AB3AAA3FA
:1029500003D0C4EC15F00DD093A502D0A3B5E3D7F6
:1029600092AF02D0A2BFDFD79AB3AAA302D0A8EC3D
:102970001FF06000BBF0F5FF6000B7F0F8FF6000EB
:10298000B3F0F7FF6000AFF0F6FF11004CEC1FF062
:10299000CBEC1EF04CEC0FF040EC1FF09DEC1FF068
:1029A0002AEC19F060EC1DF0ECEC1EF018EC1FF0B6
:1029B00032EC1DF076EC1DF01AEC1DF0B8EC1BF0BB
:1029C00034EC1BF061EC12F034EC1FF0E2EC1DF083
:1029D00002EC18F0A00E0001BD6FC80EBE6FA40E71
:1029E000BF6FA60EC06FA20EC16F2F0EC26F270E53
:1029F000C36F810EC46F100EC56FFA0EC66F900EB6
:102A0000C76FAF0EC86F400EEDEC12F01200C66F2C
:102A1000240E0001C66102D0240E04D0F00EC6655B
:102A200002D0F00EC66F600018F3C4F0C43B0F0E66
:102A3000C417C451C65D01017C6F600018F3C4F077
:102A40000001C43B0F0EC417600018F3C5F0D89006
:102A5000C533C451C55D01017B6FD8907B317A6F5E
:102A60000001C6390F0B0101796F140E0001C06F10
:102A7000C6518FEC1CF00101786F160E0001C06F7B
:102A8000C6518FEC1CF00101776F0001C651120096
:102A90004A04D8A424D04950BE6FBF6BBE1DC06F7E
:102AA000BF1DC16FBC51C05DBD51C159D8B003D06D
:102AB000BC69BD6904D04950BC27000EBD23BC5180
:102AC0000101085D0001BD5101010959D8B016D0BE
:102AD000600020F4BCF0600024F4BDF00FD0495039
:102AE000BC5D000EBD59D8B005D0000EBD6F000E04
:102AF000BC6F04D04950BC5F000EBD5B000E496E38
:102B00006000F0F2BCF06000F4F2BDF01200000EC4
:102B1000926E010E0101D86F150E5924D96EDA6A32
:102B2000020EDA226F00A3F7DFFF592A140E596450
:102B300002D0000E596E030E5918D8B417C2DFF137
:102B40005950276E286ADF51296E2A6A040E2926F9
:102B5000000E2A222750291814E128502A18D8A438
:102B600010D0000ED86F600064F1DDF1000E596ED8
:102B7000600068F123F05B50E9EC0EF00101DE6FBC
:102B80001200000ED76F1200AA933C016AAB02D06C
:102B9000010E01D0000E4A18D8B405D0000E6ABB51
:102BA000010E4A6E2AD056AB27D09E50D8B424D0FE
:102BB000010177519E5CD8B002D04F0E17D07851EA
:102BC0009E5CD8B002D0270E11D079519E5CD8B04F
:102BD00002D0130E0BD07A519E5CD8B002D0090EF1
:102BE00005D07B519E5CD8B003D0040E492604D09A
:102BF0007C519E5CD8A0492A492A010E0101A86F88
:102C00001200C16F05D0000E01D0010EC06F21D09F
:102C10000001C1510A0AD8B4F6D7010AD8B4F3D7D3
:102C2000070AD8B4F0D7010AD8B4EDD7030AD8B44C
:102C3000EAD7240AD8B4E7D7190AD8B4E4D7070AE0
:102C4000D8B4E1D7010AD8B4DED70C0AD8B4DBD7A0
:102C5000DCD70A0EBC6FC151A2EC1DF0080AD8B433
:102C600008D00A0EBC6FC151A2EC1DF0090AD8A40D
:102C700002D0000EC06FC051120001011C511D1185
:102C8000D8B402D0010EA86F0001A351D8B403D06C
:102C9000010E0101A86F0101A805D8A406D0000EFD
:102CA000216F000E206F000EA86F0001AD51D8A457
:102CB00006D0B451D8A403D0AE51D8B402D0000E7F
:102CC00001D0010E0101BA6FBA05D8A41200E00EBE
:102CD000205D2E0E2159D8A01200060E0001A21967
:102CE000D8B41200A2C0A1F0060EA26F010E9F6F11
:102CF000120001012A510001CA5DC26F01012B516E
:102D00000001CB59C36F000EC56F640EC46FB0ECE9
:102D100019F0C251936F01016F5100019319D8B49A
:102D20000DD001012A510001CA5D01012B510001A2
:102D3000CB59D8A003D0010E01016E6F0001CA511A
:102D400001012A5D0001CB5101012B59D8A01200CD
:102D500065EC05F003D08FECFEF0506E5050D8B407
:102D6000FAD7A1EC1FF0120001013805D8A420D039
:102D7000000E386F000E3B6F000E3A6F000E000120
:102D8000CC6F6000E4F0CDF06000E8F0CEF0020E11
:102D9000D06F020ECF6F040ED26F040ED16F090EEA
:102DA000DAECE0F0600030F339F0600034F33AF030
:102DB00001013905D8A402D0000E396F6000ECF48F
:102DC000DCF03B50ABECF8F001013A6F3B513A19A3
:102DD000D8B412003AC13BF11200C06F600000F39A
:102DE000B5F00001B551B5253D016F6FFE0E706F56
:102DF000010E0101B26F010E666F000E0201986FA5
:102E0000000E0001AF6F010E0101AD6F000E646F87
:102E10004104D8A40FD0000E0001606FBF51D8B498
:102E200002D00C0E01D0000E616F000E626F000E1A
:102E3000636F08D0000E0001606FBF51D8B4F3D7A4
:102E40001C0EF2D7040E86EC0EF01200AE0E00013E
:102E5000CE6F470ECF6FA10ED06F3F0ED16F6000C7
:102E6000B4F3BCF06000B8F3BDF0BE6BBF6B000EF6
:102E700001EC04F06000F0F2CAF06000F4F2CBF074
:102E80006000F8F2CCF06000FCF2CDF070ECEDF0F8
:102E9000600028F3E3F060002CF3E4F0600030F30E
:102EA000E5F0600034F3E6F021EC0EF060008CF306
:102EB000EDF0600090F3EEF01200AE0E0001CE6F68
:102EC000470ECF6FA10ED06F3F0ED16F6000B4F3ED
:102ED000BCF06000B8F3BDF0BE6BBF6B000E01EC40
:102EE00004F06000F0F2CAF06000F4F2CBF0600091
:102EF000F8F2CCF06000FCF2CDF070ECEDF0600088
:102F000028F3E3F060002CF3E4F0600030F3E5F028
:102F1000600034F3E6F021EC0EF060008CF3EDF08D
:102F2000600090F3EEF01200000E0001CE6F000E74
:102F3000CF6F800ED06F3F0ED16F6000B4F3BCF046
:102F40006000B8F3BDF0BE6BBF6B000E01EC04F087
:102F50006000F0F2CAF06000F4F2CBF06000F8F22A
:102F6000CCF06000FCF2CDF070ECEDF0600028F3E6
:102F7000E3F060002CF3E4F0600030F3E5F0600073
:102F800034F3E6F021EC0EF060008CF3EDF060001D
:102F900090F3EEF01200140E0001CE6FAE0ECF6F64
:102FA000C70ED06F3F0ED16F6000B4F3BCF060006D
:102FB000B8F3BDF0BE6BBF6B000E01EC04F0600017
:102FC000F0F2CAF06000F4F2CBF06000F8F2CCF05E
:102FD0006000FCF2CDF070ECEDF0600028F3E3F05F
:102FE00060002CF3E4F0600030F3E5F0600034F3AF
:102FF000E6F021EC0EF060008CF3EDF0600090F351
:10300000EEF01200420E0001B56FB551B5253D013D
:103010006F6FFE0E706F000E716F000E726F000EFC
:10302000746F100E756F000E7B6F6C69900E736F6E
:103030003901A29FA3933D0179953901A391A395ED
:103040003D01769979973901928F93833D017A8575
:103050003901938193853D0176817A87210E3A016A
:10306000136F000E3D01796F000E766F7399120099
:10307000C15104E1020EC05DD8A012D0C15110E1CF
:103080001F0EC05DD8A0C0B10BD0FF0EC025BC6F15
:10309000FF0EC121BD6FFBEC1EF05A0AD8B412D04E
:1030A0000001C15104E1210EC05DD8A01200FF0E45
:1030B000C025BC6FFF0EC121BD6FFBEC1EF05B0A8B
:1030C000D8A41200FF0E0001C025BC6FFF0EC12165
:1030D000BD6FFF0EBE6F97EC1BF0120001011C517B
:1030E0001D11D8B402D0010EA86F0001A351D8B4AD
:1030F00003D0010E0101A86F5150D8A403D0010ED6
:103100000101B96F0101A805D8A408D0000E020181
:10311000646F000E636F000E0101A76FA00E020125
:10312000635D0F0E6459D8A012000001AD51D8A400
:103130001200B451D8A41200010E0101A76F1200B1
:10314000BD6F010E0001BC6FBD05D8A402D0010EF9
:1031500023D0020EBD19D8A402D0020E1DD0040E39
:10316000BD19D8A402D0030E17D0080EBD19D8A4DB
:1031700002D0040E11D0100EBD19D8A402D0050E35
:103180000BD0200EBD19D8A402D0060E05D0400EDB
:10319000BD19D8A402D0070EBC6FBC511200CB6F72
:1031A0000001C851D8B40DD0C851070BC46F180E18
:1031B00035EC1CF0020E0001C46F150E35EC1CF04E
:1031C00005D0010EC46F150E35EC1CF00001CB517B
:1031D000D8B40DD0CB51070BC46F190E35EC1CF0D1
:1031E000020E0001C46F160E35EC1CF01200010E29
:1031F000C46F160E35EC1CF012000101E805D8A4CE
:1032000012006000D4F9EDF06000D8F9EEF026EC81
:1032100017F06000B4F359F26000B8F35AF2A10E4F
:103220000201595D0F0E5A59D8A006D00001B451C1
:10323000D8A402D0010E01D0000E0101AB6F000135
:10324000AD510101AB19D8B41200ABC1ADF0010E04
:10325000766F1200000EDE6F000EDF6F000EE06F63
:10326000000EE16F000EE46F000EE56F000EEA6FD6
:10327000000EEC6F000EF16F000EF36F000EF46F96
:10328000000EF56F000EF66F000EF76F000EF96F6F
:10329000000EFA6F000EFB6F000EFC6F030EFD6F49
:1032A000160EFE6F1F0EFF6F940EF86F12000001D6
:1032B000C76F000E0001C56F000EC66F640EC06FB1
:1032C000C7518FEC1CF0300FC46F0A0EC06F640E34
:1032D000BC6FC751A2EC1DF08FEC1CF0300FC56F16
:1032E0000A0EBC6FC751A2EC1DF0300FC66F600014
:1032F00010F3EFF22E0E0201F06F600014F3F1F202
:10330000600018F3F2F21200C16F6000F8F2C2F030
:103310006000FCF2C3F0E2EC1DF00001C151C125D8
:103320003D01586F6FEC1EF0600003F356FD3D0148
:103330005D8B5CEC1EF00CD060000BF3D9FF6000DD
:103340000FF3DAFFDF5001EC1DF00001C24BC32B7D
:103350000001C007C029D8A4EFD795EC1EF01200D9
:10336000000EC86F000EC76FC451C511D8B41CD071
:10337000010EC66F04D0D890C437C537C62BC5AF71
:10338000FAD7D890C737C837C451C25DC551C359A1
:10339000D8A005D0C451C25FC551C35BC781D890C6
:1033A000C533C433C62FEDD760001CF3C2F06000F4
:1033B00020F3C3F01200050E0001BC5D100EBD59D4
:1033C000D8A002D0640E12001F0EBC5D0F0EBD59B6
:1033D000D8A002D0500E1200610EBC5D0E0EBD5979
:1033E000D8A002D03C0E1200C10EBC5D0D0EBD591E
:1033F000D8A002D0280E1200E50EBC5D0C0EBD59FF
:10340000D8A002D0140E1200000E1200D86F600077
:1034100060F3D9F01FD0690EC26FFC0EC36F660E49
:10342000C46F010EC56F000EC66F000EC76F60003F
:1034300064F3C8F0000EC96F000ECA6F000ECB6FA8
:10344000000ECC6F000ECD6F60005CF3CEF0C0ECD0
:1034500006F0D92B0001D951D65DD8A01200DBD7D8
:103460000001BD6F4A04D8A411D04950FF0A0001E1
:10347000BC6FBD51BC5DD8B002D0BD6902D049500F
:10348000BD27120EBD6511D0120E0ED00001BD5128
:10349000495CD8A003D0010EBD6F02D04950BD5F7A
:1034A000080EBD6102D0080EBD6F000E496EBD5101
:1034B00012000001BD6F0001BD05D8A40FD0BB985C
:1034C000BB9AA00E26EC1FF0BB8A350EE82EFED765
:1034D00000F0BB9AC80E26EC1FF00ED0BB98BB9A2A
:1034E000A10E26EC1FF0BB8A350EE82EFED700F0A9
:1034F000BB9AC00E26EC1FF0BB8ABB880001BD51F1
:103500001200BD6F4A04D8A414D04950FF0A00012C
:10351000BC6FBD51BC5DD8B002D0BD6902D049506E
:10352000BD27BD513F5CD8B00ED06000FCF0BDF0AF
:103530000AD049500001BD5DD8B003D0000EBD6F68
:1035400002D04950BD5F000E496EBD51120001010D
:10355000D851D8A41BD06000D0F4BCF0A50E000157
:10356000BC6502D0640E0BD09B0EBC6502D0420E2F
:1035700006D0960EBC6502D0210E01D0000EBC6FA5
:1035800034C163F1010E0101626F03D0600084F564
:10359000BCF00001BC511200BD6F4A04D8A411D088
:1035A0004950FF0A0001BC6FBD51BC5DD8B002D0CC
:1035B000BD6902D04950BD27040EBD650CD0040E74
:1035C00006D049500001BD5DD8B003D0000EBD6FDC
:1035D00002D04950BD5F000E496EBD511200BE5170
:1035E000BF11D8B418D0010EC06F04D0D890BE3728
:1035F000BF37C02BBFAFFAD7BE51BC5DBF51BD595D
:10360000D8A004D0BE51BC5FBF51BD5BD890BF33C2
:10361000BE33C02FF1D76000F0F2BCF06000F4F2CE
:10362000BDF012003C0174AB04D00001BC6BBC2B9C
:1036300002D00001BC6B3C0174AB02D0010E01D082
:10364000000E0101B619D8B402D0010E01D0000E4F
:103650000001BC15BD6F3C01000E74BB010E0101E1
:10366000B66F0001BD511200000EB36E000EB46EB5
:10367000050EB56EEC0EB16E780EB06EB0506F00E8
:10368000C4FEBCF00001BD6B6000F0F2BDF0BC6B8D
:10369000BC110201FC6F0001BD510201FD6F390137
:1036A000A4919481010EB26E1200C95101011C1542
:1036B0000001C26FCA5101011D150001C36F6000F6
:1036C00024F3C4F0600028F3C5F0B0EC19F0C25147
:1036D000CB6FCB51D8B407D00A0EA219D8A403D00F
:1036E000010E01017E6F0001CB511200C951020190
:1036F00053150001C26FCA51020154150001C36F76
:10370000600024F3C4F0600028F3C5F0B0EC19F0B9
:10371000C251CB6FCB51D8B407D00A0EA219D8A48E
:1037200003D0010E01017E6F0001CB511200000E8B
:10373000D2BE010EBF6FBD51030B3901E16F6000B6
:10374000F3F2E0F96000FBF2E3F93F0EE517E585DF
:10375000D29E550EE66FAA0EE66FE583E5B3FED75F
:10376000E5950001BFB102D0D29E01D0D28E1200E9
:10377000000E9B6E000E9C6E020E9D6EE20E996E08
:10378000000E986E98506F0064FEBCF00001BD6B97
:103790006000F0F2BDF0BC6BBC110201FA6F0001D9
:1037A000BD510201FB6F3901A89D010E9A6E1200F6
:1037B0000D0E20601200600078F00FF060007CF0C9
:1037C00010F0600080F011F0000E126E000E136E0B
:1037D000000E146E000E166E000E156E000E176EA3
:1037E000000E196E000E186E000E40EC09F012006B
:1037F000000E0001BE6FCABE02D0010E01D0000E45
:10380000BE6FBE51A519BD6FBD51BE15A36FBE5190
:10381000D8A403D0BC6BBC2B02D00001BC6BBD5143
:10382000BE19BC15A46F6000F8F2A5F01200C56FB8
:10383000D60E0001C66F020EC76F600014F3D6F2F9
:10384000600010F3D7F2080EC4611200C451D8B45E
:103850001200600018F3BEF060001CF3BFF0020E0F
:10386000C06F580E84EC19F01200C56FD60E00011F
:10387000C66F020EC76F600014F3D6F2600010F33B
:10388000D7F2080EC4611200C451D8B4120060000F
:1038900018F3BEF060001CF3BFF0020EC06F580EAC
:1038A00084EC19F012004D0EC26FFA0EC36F0B0EAE
:1038B000C46F010EC56F060EC66F3F0EC76F000EB8
:1038C000C86F010EC96F000ECA6F000ECB6F000EDD
:1038D000CC6F000ECD6F6000D8F3CEF0C0EC06F0D8
:1038E00012004D0EC26FFA0EC36F0B0EC46F010EA5
:1038F000C56F010EC66F3F0EC76F000EC86F010E79
:10390000C96F000ECA6F000ECB6F000ECC6F000E99
:10391000CD6F6000D8F3CEF0C0EC06F01200C16F9E
:10392000000E0001C36FC051D8B415D0010EC26F94
:1039300003D0D890C037C22BC0AFFBD7D890C337C5
:10394000C051C15DD8A003D0C051C15FC381D89020
:10395000C033C22FF3D7C35112000201FE51D8B4B5
:1039600010D0EB0E5824D96EDA6A010EDA22DF503D
:103970003D01EA6F582A150E58640AD0150E586E8C
:1039800007D039019399000E0101D66F000E596ED0
:103990000201FE071200010E0001CA6FFF0ECB6F7D
:1039A000000ECC6F000ECD6F000ECE6F000ECF6FED
:1039B000000ED16F000ED06F000ED26F000ED46FCC
:1039C000000ED36F050E11EC08F012000001BD6F60
:1039D0001F0E0001BD6502D01F0EBD6FBB98BB9AC4
:1039E000270E26EC1FF0BB8ABB9A810E26EC1FF037
:1039F000BB8ABB9A0001BD5126EC1FF0BB8ABB8875
:103A000012000001BC6F0001BD695750D8A412001C
:103A10000BD03D0162AB04D06000F3F255FD120003
:103A2000050EE82EFED700F00001BD2FF2D7010EE3
:103A3000576E1200050E576F000E586F070E596F24
:103A4000010E5A6F070E5B6F110E5C6F000E5D6FFB
:103A5000220E5E6F000E5F6F9B0E566F3901AA93A8
:103A60009A831200010E966E000E956E000E976EF0
:103A70009368000E926EA9919981000E0001BC6FAF
:103A8000000EBD6F000EBE6F78EC1FF0D00E946E6E
:103A90001200BC51BE036F00CCFFC0F06F00D0FF1E
:103AA000C1F0BC51BF03F350C127BD51BE03F35059
:103AB000C127600000F3BCF0600004F3BDF0120009
:103AC0000F0E3C016B6F000E6C6F010E6D6F270EB9
:103AD0006E6F070E6F6F260E706F190E716F290EC5
:103AE000726F160E736F830E6A6F12000A0E3C011E
:103AF000756F0E0E766F050E776F050E786F050EDB
:103B0000796F020E7A6F000E7B6F000E7C6F000ED5
:103B10007D6F860E746F1200C951020155150001A8
:103B2000C26FCA51020156150001C36F600024F331
:103B3000C4F0600028F3C5F0B0EC19F0C251CB6FAF
:103B4000CB511200BD6F080E0001BE6F000EBF6F9B
:103B5000D890BD35BF35BF6FD890BD37BC51BF5D64
:103B6000D8A002D0BC51BF5FBE2FF2D7BF51120008
:103B7000BC6F0001BC05D8A40BD0010EBD6F120EA6
:103B8000406408D0120E8F6F010E01015A6F02D0EF
:103B9000000EBD6F0001BD5112000001BD6F010E8E
:103BA0000101D66F6000F0F2DBF16000F0F2FEF28E
:103BB000390193B905D06000F7F2EAFD010E586EA5
:103BC000938912003D015DAF03D05750D8B4120065
:103BD000000E576E800E5E6F200E5F6F030E656FD6
:103BE000840E5D6F000E636F000E606F1200B2C036
:103BF000B5F00001B251B2253D016F6FFE0E706F3E
:103C0000010E0101B26F010E4F6E010E0001AF6F88
:103C1000010E0101AD6F1200000EBF6F000EC06FEC
:103C200009D0C051BC25D96E000EBD21DA6EDF501F
:103C3000BF1BC02BBE51C05DD8A0F3D7BF5112002F
:103C4000070E0001926503D0120E926504D00D0E8E
:103C5000926F92C06AF1B051D8B403D0030EB06530
:103C60001200020EB06F1200026E010E0101D66F3B
:103C7000600004F0DBF1600004F0FEF2390193B95A
:103C800005D060000BF0EAFD010E586E938912001A
:103C9000000E046E000E056E09D005500124D96E89
:103CA000000E0220DA6EDF50041A052A0350055C6C
:103CB000D8A0F3D7045012000001BC695750D8A413
:103CC000120007D03D015DAB1200050EE82EFED7B5
:103CD00000F00001BC2FF6D7010E576E1200000154
:103CE000BC695750D8A4120007D03D0161BF120033
:103CF000050EE82EFED700F00001BC2FF6D7010E0E
:103D0000576E12006F0060FFBBF0390194B1A4A19F
:103D100003D058EC1FF005D099B1A9A102D08CECCA
:103D20001FF06000EFF2D8FF1100BC695750D8A413
:103D3000120007D03D0163B51200050EE82EFED734
:103D400000F00001BC2FF6D7010E576E12000001E3
:103D5000BC6F0101E5510001BC19D8B407D03E0188
:103D6000F89F6000F3F2F1FEF88FF89D0001BC515E
:103D70001200B2A409D0B2906000EBF2B1FF600073
:103D8000E7F2B0FFB28012006000EBF2B1FF60001A
:103D9000E7F2B0FF1200000EC06F000EC16F000E00
:103DA000C26F000EC36F000EC46F000EC56F000E11
:103DB000C66F000EC76F12003E01F0510001BF6FC9
:103DC000BE6B3E01EF510001BE25BC6F3E01000EEF
:103DD0000001BF21BD6F1200040EA26E130EA16E72
:103DE000140EA36EF00E9F6E000E9E6E3901A79109
:103DF000E00EA06E1200BD51030B3901E16F6000AF
:103E0000F3F2E0F93F0EE517E58100F000F039012B
:103E1000E3511200AE47A13FAE47A13F6666663F41
:103E200014AEC73F0000803F5E0105202020200027
:103E3000060EAE6E000EAD6E000EAF6E610EAB6E76
:103E4000000EAA6EA495C00EAC6E12000001BC6FED
:103E5000010E3D01126F6000F3F211FD3901A2A9BC
:103E6000FDD73D0110511200200E3D01156F030ECC
:103E7000166F070E196F010E1C6F830E146F120060
:103E8000600E3901D96F000EDB6F000EDD6F080E7A
:103E9000DF6F000EDE6F1200D28A390183818383C7
:103EA000838783898385828F8A8384918991120095
:103EB000A4916000F0FBB9F06000F4FBBAF0B9EC3B
:103EC0001EF0CAECFCF012006000F0F2F4F26000A8
:103ED000F4F2F5F26000F8F2F6F212006000F0F28F
:103EE000F7F26000F4F2F8F26000F8F2F9F2120072
:103EF0006000F0F2F2F36000F4F2F3F36000F8F225
:103F0000F4F3120000019051D8B403D04EEC03F04A
:103F10001200A6EC0FF01200A991010E0101E36F4F
:103F2000000E596E1200BC6F6000F0F29DF012009E
:103F30000001BC6F0001BC511200820E3E01C16F36
:103F40001200BE92C6921200AC8E1200B280120015
:103F5000AA93120001FFFFFFFFFFFFFFFFFFFFFF1C
:103F6000FFFFFFFFFFFFFFFFFFFFFFFFFFFFFFFF61
:103F7000FFFFFFFFFFFFFFFFFFFFFFFFFFFFFFFF51
:103F8000FFFFFFFFFFFFFFFFFFFFFFFFFFFFFFFF41
:103F9000FFFFFFFFFFFFFFFFFFFFFFFFFFFFFFFF31
:10AE7000FFFFFFFFFFFFFFFFFFFF000000000000DC
:10AE8000000000000000000000FEFE0000000000C6
:10AE90007F7F606060606080C0C0C0C0C0803F7F56
:10AEA0006060607F3FFEFE0080C0C0407F7F1F3B30
:10AEB0007160400000606000000000000C0C0000A9
:10AEC00000F0FC1E061EFCF07F7F0303037F7FC0A3
:10AED000E0F070E0FEFE1F3F7870387F7FF0F0807A
:10AEE000C0E070707F7F03010000000000000000E0
:10AEF0000000005A7765697465204C6F6B00496EDD
:10AF0000746572666163650050726F6772616D008F
:10AF1000537461747573005365747570009F0000FD
:10AF20000000000000000000000000000000000021
:10AF30000000000000000000000000000000000011
:10AF40000000000000000000000000000000000001
:10AF500000000000000000000000000000000000F1
:10AF600000000000000000000000000000000000E1
:10AF700000000000000000000000000000000000D1
:10AF800000000000000000000000000000000000C1
:10AF900000000000000000000000000000000000B1
:10AFA00000000000000000000000000000000000A1
:10AFB0000000000000000000000000000000000091
:10AFC0000000000000000000000000000000000081
:10AFD0000000000000000000000000000000000071
:10AFE0000000000000000000000000000000000061
:10AFF0000000000000000000000000000000000051
:10B000000000000000000000000000000000000040
:10B010000000000000000000000000000000000030
:10B020000000000000000000000000000000000020
:10B030000000000000000000000000000000000010
:10B040000000000000000000000000000000000000
:10B0500000000000000000000000000000000000F0
:10B0600000000000000000000000000000000000E0
:10B07000000000FE020202020202020202020202BA
:10B0800002020202020202020202020202020202A0
:10B090000202020202020202020202020202020290
:10B0A0000202020202020202020202020202020280
:10B0B00002020202FE0000FF00000000000000008B
:10B0C0000000000000000000000000000000000080
:10B0D0000000000000000000000000000000000070
:10B0E0000000000000000000000000000000000060
:10B0F0000000000000000000FF0000FF0000000052
:10B10000000000000000000000000000000000003F
:10B11000000000000000000000000000000000002F
:10B12000000000000000000000000000000000001F
:10B13000000000000000000000000000FF0000FF11
:10B1400000000000000000000000000000000000FF
:10B1500000000000000000000000000000000000EF
:10B1600000000000000000000000000000000000DF
:10B1700000000000000000000000000000000000CF
:10B18000FF00007F40404040404040404040404041
:10B1900040404040404040404040404040404040AF
:10B1A000404040404040404040404040404040409F
:10B1B000404040404040404040404040404040408F
:10B1C000404040407F0000FE0202020202020202F2
:10B1D000020202020202FA32C202FA02824242422F
:10B1E000820242FA420202FA8242428202824242CF
:10B1F00082C202FA020242FA42020202020202027F
:10B200000202020202020202FE0000FF0000000031
:10B21000808000800080000000800780E09317009D
:10B22000F304848403000083840400F70080800713
:10B230000003848402078003848400030404000064
:10B240000000A0008000808000000000FF0000FFE0
:10B25000000000070808050F00070808040F000099
:10B260000F0000000F0100000F00070A0A0B000F7B
:10B270000908080700070A0A0B000F0100000F0069
:10B280000000000000000F000F0100000F00000090
:10B29000FF0000FF000000000000000000000000B0
:10B2A0000000000000000000000000FF010101019B
:10B2B00001FF000000FF0101010101FF000000008B
:10B2C000000000000000000000000000000000007E
:10B2D00000000000FF00007F4040404040404040F0
:10B2E000404040404040404040404040404040FF9F
:10B2F0008080808080FF404040FF8080808080FF91
:10B30000404040404040404040404040404040403D
:10B3100040404040404040407F0000FE02020202A8
:10B32000FA02020202E29AE20202FA82422202FADD
:10B3300082422202C2020202C2028242424202420D
:10B34000FA42020282424282C202C2824242820225
:10B3500082424282FA020202FA020202FE0000FF68
:10B3600000008080058000F0078080000700878152
:10B3700082040087818204F00384840207008485AC
:10B38000058200F0030484F0830404028780070030
:10B390008000878003040404A700800085800000EB
:10B3A000FF0000FF00070808050F000F0908080745
:10B3B00000090A0A040007080808000F0100000F2E
:10B3C00000070808050F000708080007080800071D
:10B3D0000A0A0B000F0100000F0000000F000F0110
:10B3E00000000F00FF0000FF000000000000000050
:10B3F0000000000000000000000000FF010101014A
:10B4000001FF0000FF0101010101FF000000FF0139
:10B4100001010101FF000000000000000000000029
:10B420000000000000000000FF00007F404040409E
:10B43000404040404040404040404040404040FF4D
:10B440008080808080FF4040FF8080808080FF403F
:10B450004040FF8080808080FF404040404040402E
:10B460004040404040404040404040407F0000FE5F
:10B4700002020202020282424282C202FA82424274
:10B48000820282424242028242424202FA824243A3
:10B49000820282424282C202FA020242FA4202025C
:10B4A0008242428202C282424282020202020202BC
:10B4B000FE0000FF0000000000000304040207007B
:10B4C0000704040403000405050200030404040047
:10B4D000A70080008780030404020700030404001F
:10B4E0000304040003050505000700000007000031
:10B4F00000000000FF0000FF00000000000000004E
:10B50000000000000000000000000000000000003B
:10B51000000000000F000F0100000F0000000000FD
:10B52000000000000000000000000000000000001B
:10B530000000000000000000FF0000FF000000000D
:10B5400000000000000000000000000000000000FB
:10B55000000000FF0101010101FF000000FF0101E7
:10B56000010101FF000000000000000000000000D9
:10B57000000000000000000000000000FF00007F4D
:10B5800040404040404040404040404040404040BB
:10B5900040404040404040FF8080808080FF4040ED
:10B5A00040FF8080808080FF4040404040404040DD
:10B5B000404040404040404040404040404040408B
:10B5C0007F0000FE020202020202020202020202E6
:10B5D0000202F2628202F20202828282020282F29B
:10B5E000820202F20282820202028282028202F25B
:10B5F000020282F28202020202020202020202023B
:10B6000002020202FE0000FF000000000000000035
:10B610000000000000000F0001060F0007080808E6
:10B62000070000070808000F0100000F00070808C6
:10B63000050F0007080800070808000000000000C8
:10B640000000000000000000FF0000FF00000000FC
:10B6500000000000000070888850F800788080406A
:10B66000F80008FE090100FF100808F00070A8A803
:10B67000B000FF908888700070A8A8B000F810088B
:10B6800008F000000000000000000000FF0000FFC4
:10B690000080008080000090000080808000F0002A
:10B6A0008080000080F080010000000080800000A9
:10B6B0008000008000F0000000008080008000809A
:10B6C0000000008000F0008080000080F08000001A
:10B6D000FF00007F404F4140404F404F40474848A7
:10B6E00048404F4140404F40404748484040404715
:10B6F0004A4A4B404F4241404047484840474848EB
:10B70000454F40474848444F404F494848474040CC
:10B71000474848407F0000FE0202C232C2020202D5
:10B72000828202F202820202820202828202020209
:10B730008282820202828282029202028282020259
:10B740008202028202820202028202820282820259
:10B750000202828202820202FE0000FF000E01014C
:10B76000010E00070808090F000F02010000070A78
:10B770000A0B00090A0A0400090A0A04000F00075C
:10B780000A0A0B000F02010000070808040F000F4F
:10B790000100000F00072828251F0000FF0000FF00
:10B7A0000000000000000000000000000000000099
:10B7B0000000000000F8100808F000F90070888808
:10B7C0008800FF100808F000087F88800000000053
:10B7D0000000000000000000000000000000000069
:10B7E000FF0000FF0000000000000000000000005B
:10B7F000000000E02020C02020C000C0242024C081
:10B8000000C0202040E000FC000000E400C0202038
:10B810002000FC402020C0000000000000000000CC
:10B8200000000000FF00007F40404040404040409A
:10B8300040404040404040434040434040434041FE
:10B840004242424140414A4A4947404142424043C4
:10B8500040414242424043404040434040404040DB
:10B8600040404040404040407F0000FE0202C24253
:10B8700042428202020202020202020202020202A8
:10B880000202020202024202020202020202020258
:10B89000020202824242020202020202C2020202C8
:10B8A0000202020202020202C2020202FE0000FFC3
:10B8B00000003F060A1221001C2222143E003E0412
:10B8C00002023C001CA2A2947E003E001C2A2A2CEC
:10B8D000003E0804020002FF02001C2222143E0067
:10B8E0003F0402023C003E08040200021F22200026
:10B8F000FF0000FF0000000000000000000000004A
:10B900000000000000000000000000000000000037
:10B910000000000000000000000000000000000027
:10B920000000000000000000000000000000000017
:10B9300000000000FF0000FF000000000000000009
:10B94000000000000000000000000000E01010A057
:10B95000F000FE40A0100010FE100000F20030C009
:10B9600000C03000000000000000000000000000E7
:10B970000000000000000000FF00007F4040404049
:10B9800040404040404040404040404040404040B7
:10B9900040414140414041404041404040414140A0
:10B9A0004140404041404040404040404040404095
:10B9B0004040404040404040404040407F0000FE0A
:10B9C00002020202020202020202020202020282D7
:10B9D00082828202020202020202020202020202C7
:10B9E0000202020202020202020202020202020237
:10B9F0000202020202020202020202020202020227
:10BA0000FE0000FF00000000000000000000000039
:10BA10000000007F4444443B007C1008040038547C
:10BA20005458007C040478040478004854542400DA
:10BA300038545458000000000000000000000000CE
:10BA400000000000FF0000FF0000000000000000F8
:10BA500000000000000000000000000000000000E6
:10BA600000000000000000000000000000000000D6
:10BA700000000000000000000000000000000000C6
:10BA80000000000000000000FF0000FF00000000B8
:10BA900000000000000000000000000000000000A6
:10BAA000E01010A0F000FE40A0100010FE100000FA
:10BAB000F20030C000C030000000000000000000B4
:10BAC000000000000000000000000000FF00007FF8
:10BAD0004040404040404040404040404040404066
:10BAE0004040404040414140414041404041404051
:10BAF0004041414041404040414040404040404042
:10BB00004040404040404040404040404040404035
:10BB10007F0000FE0202020202020202C232C202E0
:10BB20000282020202820282F28202020282828285
:10BB300002028282820282820202028282028202E5
:10BB400082F28202029202F20202820202020202E5
:10BB500002020202FE0000FF000000000000000ED2
:10BB60000101010E00070808040F000007C8282083
:10BB7000070808080700EF00000F00000F00070883
:10BB80000805EF0000070808000F000F0205080075
:10BB90000101010101000000FF0000FF00000000A2
:10BBA0000000000000000000000000000000000095
:10BBB000017F01000E11110A1F001F0201011E006A
:10BBC0001F04020100010F1110000000000000001E
:10BBD000000000000000000000000000FF0000FF67
:10BBE0000000000000000000000000000000000055
:10BBF00000000000E01010A0F000FE40A0100010B7
:10BC0000FE100000F20030C000C030000000000054
:10BC10000000000000000000000000000000000024
:10BC2000FF00007F40404040404040404040404096
:10BC30004040404040404040404141404140414000
:10BC400040414040404141404140404041404040EF
:10BC500040404040404040404040404040404040E4
:10BC6000404040407F0000FE020202021AE202E26F
:10BC70001A0202C2A2A2C20202E28242220202FA14
:10BC8000422222C20202EA0202E2422222C202024C
:10BC9000C2222242FA0202C2A2A2C20202E242224C
:10BCA00022C2020202020202FE0000FFF8F8F8F8C7
:10BCB000F8F8FBF8F8F8F8F9FAFAFAF8F8FBF8F8F7
:10BCC000F8F8F8FBFAFAFAF9F8F8FBF8F8FBF8F8E4
:10BCD000F8FBF8F8F9FA1A1A1B1818191A1A1A1890
:10BCE000181B1818181B181818181818FF0000FF30
:10BCF0000303FBFBFBFBFBFBFB0303FFFFFFFFFF60
:10BD0000FFFFFFFFFFFFFFFFFFFFFFFFFFFFFFFF43
:10BD1000FFFFFFFFFFFFFFFFFFFF0080C04040C0AD
:10BD20008000C0C04040C0800040404040C0C000D3
:10BD3000FF0000FFFE00E2F0FAF8FAF0E200FEFF7A
:10BD4000FFFFFFFFFFFFFFFFFFFFFFFFFFFFFFFF03
:10BD5000FFFFFFFFFFFFFFFFFFFFFFFFFFFF000FE2
:10BD60001F10101D0D001F1F10101F0F00181C1694
:10BD700013111000FF00007F414054414B434B41E1
:10BD80005440417F7F7F7F7F7F7F7F7F7F7F7F7F6B
:10BD90007F7F7F7F7F7F7F7F7F7F7F7F7F7F7F7FB3
:10BDA0007F7F404040404040404040404040404015
:10BDB00040404040404040407F0000FE02020202FE
:10BDC00002020202020202020202020202E29AE2FB
:10BDD000020202FA028242020242FA42020202CA4B
:10BDE000020282424242820202C282424282020233
:10BDF000020202020202020202020202FE0000FF2E
:10BE00000000000000000000000000000000000032
:10BE100007000000070000070102040000000304FF
:10BE200004000007000003040404030000070000EE
:10BE300000070000000000000000000000000000FB
:10BE4000FF0000FF000000000000000000000000F4
:10BE500000000000000000F8100808F00000F900E1
:10BE600000708888880000FF100808F00000087F34
:10BE700088800000000000000000000000000000BA
:10BE800000000000FF0000FF00804040800000C074
:10BE9000008040000040F0480000804040408000AA
:10BEA00000F80000000080404080C00000C000801A
:10BEB000400000804040800000C8000080404040BA
:10BEC0000000F88040408000FF00007F404345456F
:10BED000454040474140404040405F40404043442F
:10BEE00044444340404344444040435454524F40F0
:10BEF0004047414040404043454545404047404021
:10BF00004344444440404740404047407F0000FE97
:10BF10000202020202020202020202020202020201
:10BF200002826282020202E2020202020202E202D1
:10BF300002020222020202020202020202020202C1
:10BF400002020202020202020202020202020202D1
:10BF5000FE0000FF000000000000000000000000E4
:10BF6000000000001C0302031C00001F040A110053
:10BF700000010F111000001F00000E1111110E0022
:10BF8000001F0201011E0000000000000000000070
:10BF900000000000FF0000FF0000000000000000A3
:10BFA000000000000000C0200000000000000000B1
:10BFB00000E00000000000000000000000000000A1
:10BFC0000000000000000000002000000000000051
:10BFD0000000E00000000000FF0000FF000E15154B
:10BFE0001600001F0402010000017F0100000E1175
:10BFF00011110E00000F101000000E51514A3F00A9
:10C00000001F04020100000E15151600001F00009D
:10C010000E11111100001F0201011E00FF00007F20
:10C020004040404040404040404040404040404010
:10C030004040404040404040404040404040404000
:10C0400040404040404040404040404040404040F0
:10C0500040404040404040404040404040404040E0
:10C060007F0000FE0202020202020202020202E25B
:10C070009AE20202C2020202C20242FA42020282B0
:10C080004242428302028282820202F20A0A0AF2D7
:10C090000242F24A0A0242F24A0A02020202020280
:10C0A00002020202FE0000FF00000000000000008B
:10C0B000000007000000070003040402070000035B
:10C0C00004040003A4048403808000000000000333
:10C0D0000404040300001F000000001F0000000013
:10C0E0000000000000000000FF0000FF0000000052
:10C0F0000000000000000000000000000000000040
:10C1000000000000000000000F000F0100000F0001
:10C11000000000000000000000000000000000001F
:10C12000000000000000000000000000FF0000FF11
:10C1300000000000000000000000000000000000FF
:10C1400000000000000000FF0101010101FF0000EC
:10C1500000FF0101010101FF0000000000000000DC
:10C1600000000000000000000000000000000000CF
:10C17000FF00007F40404040404040404040404041
:10C180004040404040404040404040FF80808080F0
:10C1900080FF404040FF8080808080FF40404040E2
:10C1A000404040404040404040404040404040408F
:10C1B000404040407F0000FE020202020202FA02FA
:10C1C000020202824242428202FA824222028242F7
:10C1D0004282C20282424282FA02C2824242028207
:10C1E00042428202824242420282424242028242EF
:10C1F0004282020202020202FE0000FF0000000072
:10C2000000000704048400030404048300078182FF
:10C2100004000384848207F0038484040700878079
:10C2200080000083850505F00405058200848505EE
:10C23000020003850505000000000000FF0000FF6C
:10C2400000000000000000000001060C070C0601C1
:10C2500000070A0A0B0007080808000F0100000F7A
:10C2600000090A0A0400070A0A0B00070808000F61
:10C270000100000F000000040000000000000000AA
:10C28000FF0000FF00000000000000000000FF01B0
:10C2900001010101FF0000FF0101010101FF000098
:10C2A000FF0101010101FF0000FF0101010101FF88
:10C2B000000000000000000000000000000000007E
:10C2C00000000000FF00007F4040404040404040F0
:10C2D0004040FF8080808080FF4040FF80808080E1
:10C2E00080FF4040FF8080808080FF4040FF808052
:10C2F000808080FF404040404040404040404040BF
:10C3000040404040404040407F00000000000000AE
:10C31000000000000000000000000000000000001D
:10C32000000000000000000000000000000000000D
:10C3300000000000000000000000000000000000FD
:10C3400000000000000000000000000000000000ED
:10C3500000000000000000000000000000000000DD
:10C3600000000000000000000000000000000000CD
:10C3700000000000000000000000000000000000BD
:10C3800000000000000000000000000000000000AD
:10C39000000000FCFA060606060606060606064625
:10C3A000A6262626460606068686860606068606ED
:10C3B000868606060606868606E6060606868686BD
:10C3C000060606860686860606060606060606068D
:10C3D000060606FAFC00003F5F6060606060606017
:10C3E000606060646869696A646060676A6A6A63F9
:10C3F00060606F6160606F6060676868656F6060F3
:10C40000676A6A6A6360606F6160606F60606060E5
:10C41000606060606060605F3F0000FCFA0606E6F6
:10C42000C686060606060646A626262646060606EC
:10C43000868686060606860686860606060686869C
:10C4400006E60606068686860606068606868606AC
:10C4500006060606060686C6E60606FAFCFE003F47
:10C460005FE0E0EFE7E3E1E0E0E0E0E4E8E9E9EA0B
:10C47000E4E0E0E7EAEAEAE3E0E0EFE1E0E0EFE071
:10C48000E0E7E8E8E5EFE0E0E7EAEAEAE3E0E0EF4A
:10C49000E1E0E0EFE0E0E0E0E0E1E3E7EFE0E0DF73
:10C4A000BF7FFF0305F9F9F9F9F9F9F9F9F9F9B9D4
:10C4B00059D9D9D9B9F9F9F9797979F9F9F979F92C
:10C4C0007979F9F9F9F97979F919F9F9F97979793C
:10C4D000F9F9F979F97979F9F9F9F9F9F9F9F9F94C
:10C4E000F9F9F90503FFFFC0A09F9F9F9F9F9F9FA2
:10C4F0009F9F9F9B979696959B9F9F989595959CA0
:10C500009F9F909E9F9F909F9F9897979A909F9F85
:10C51000989595959C9F9F909E9F9F909F9F9F9F72
:10C520009F9F9F9F9F9F9FA0C0FF00FCFA0606064B
:10C53000060606060606060606060606060606069B
:10C5400006060606E6F63636F6E6060606F6F6C6EB
:10C55000E6763606060606060606060606060606FB
:10C560000606060606060606060606FAFC00003F54
:10C570005F606060606060606060606060606060BC
:10C580006060606060606060676F6C6C6F67606067
:10C59000606F6F63676E6C60606060606060606059
:10C5A0006060606060606060606060606060605F8C
:10C5B0003F0000FCFA0606E6C686060606060606E4
:10C5C000060606060606060606060606E6F63636DB
:10C5D000F6E6060606F6F6C6E6763606060606060B
:10C5E000060606060606060606060606060686C6AB
:10C5F000E60606FAFCFE003F5FE0E0EFE7E3E1E07D
:10C60000E0E0E0E0E0E0E0E0E0E0E0E0E0E0E0E02A
:10C61000E7EFECECEFE7E0E0E0EFEFE3E7EEECE094
:10C62000E0E0E0E0E0E0E0E0E0E0E0E0E0E0E0E00A
:10C63000E0E1E3E7EFE0E0DFBF7FFF0305F9F9F9B1
:10C64000F9F9F9F9F9F9F9F9F9F9F9F9F9F9F9F95A
:10C65000F9F9F9F91909C9C90919F9F9F9090939EA
:10C660001989C9F9F9F9F9F9F9F9F9F9F9F9F9F9BA
:10C67000F9F9F9F9F9F9F9F9F9F9F90503FFFFC041
:10C68000A09F9F9F9F9F9F9F9F9F9F9F9F9F9F9FB9
:10C690009F9F9F9F9F9F9F9F9890939390989F9FEE
:10C6A0009F90909C9891939F9F9F9F9F9F9F9F9FDC
:10C6B0009F9F9F9F9F9F9F9F9F9F9F9F9F9F9FA089
:10C6C000C0FF00FCFA06060606060606C626162663
:10C6D000C60606F6864646860606F686464686065A
:10C6E00006C6068646460606C6060606C60606862A
:10C6F000464646860606F68646468606060606062A
:10C70000060606FAFC00003F5F60606060606060E3
:10C710006F6161616F60606F6468686760606F64BB
:10C7200068686760606F61606060606067686864C7
:10C730006F6060676868686460606F6060606F60A9
:10C74000606060606060605F3F0000FCFA0606E6C3
:10C75000C6860606C6261626C60606F686464686F9
:10C760000606F6864646860606C606864646060639
:10C77000C6060606C6060686464646860606F686A9
:10C7800046468606060686C6E60606FAFCFE003F14
:10C790005FE0E0EFE7E3E1E0EFE1E1E1EFE0E0EFD0
:10C7A000E4E8E8E7E0E0EFE4E8E8E7E0E0EFE1E034
:10C7B000E0E0E0E0E7E8E8E4EFE0E0E7E8E8E8E42C
:10C7C000E0E0EFE0E0E0EFE0E0E1E3E7EFE0E0DF32
:10C7D000BF7FFF0305F9F9F9F9F9F9F939D9E9D971
:10C7E00039F9F90979B9B979F9F90979B9B979F959
:10C7F000F939F979B9B9F9F939F9F9F939F9F97969
:10C80000B9B9B979F9F90979B9B979F9F9F9F9F948
:10C81000F9F9F90503FFFFC0A09F9F9F9F9F9F9F6E
:10C82000909E9E9E909F9F909B9797989F9F909B76
:10C830009797989F9F909E9F9F9F9F9F9897979B4A
:10C84000909F9F989797979B9F9F909F9F9F909F48
:10C850009F9F9F9F9F9F9FA0C0FF00FE0202D2024A
:10C8600002C2824242820202C2020202C202028268
:10C87000424242820202C202824242020282424298
:10C8800042820202020202020202020206FE0602C4
:10C89000826212120A0A121262820206FE00007FEF
:10C8A00040404F40404F4040404F404040434C4349
:10C8B000404040474949494940404F41404040403D
:10C8C0004044494B4A444040404040404040404042
:10C8D000607F60404146484850504848464140606B
:10C8E0007F0000FE0202D20202C2824242820202A3
:10C8F000C2020202C2020282424242820202C20218
:10C900008242420202824242428202020202020247
:10C910000202020206FE0602826212120A0A1212C3
:10C9200062820206FEFE003F40C0CFC0C0CFC0C042
:10C93000C0CFC0C0C0C3CCC3C0C0C0C7C9C9C9C9AB
:10C94000C0C0CFC1C0C0C0C0C0C4C9CBCAC4C0C0B1
:10C95000C0C0C0C0C0C0C0C0E0FFE0C0C1C6C8C841
:10C96000D0D0C8C8C6C1C0C0BF7F00FE06FA2AFA30
:10C97000FA3A7ABABA7AFAFA3AFAFAFA3AFAFA7A57
:10C98000BABABA7AFAFA3AFA7ABABAFAFA7ABABA07
:10C99000BA7AFAFAFAFAFAFAFAFAFAFA06FE060293
:10C9A00082E2F2F2FAFAF2F2E2820206FE00007F7E
:10C9B000605F505F5F505F5F5F505F5F5F5C535CC5
:10C9C0005F5F5F58565656565F5F505E5F5F5F5FB2
:10C9D0005F5B5654555B5F5F5F5F5F5F5F5F5F5F8D
:10C9E000607F604041474F4F5F5F4F4F474140601E
:10C9F0007F0000FE06FA2AFAFA3A7ABABA7AFAFA06
:10CA00003AFAFAFA3AFAFA7ABABABA7AFAFA3AFA86
:10CA10007ABABAFAFA7ABABABA7AFAFAFAFAFAFA36
:10CA2000FAFAFAFA06FE060282E2F2F2FAFAF2F2F2
:10CA3000E2820206FEFE003F60DFD0DFDFD0DFDFF4
:10CA4000DFD0DFDFDFDCD3DCDFDFDFD8D6D6D6D642
:10CA5000DFDFD0DEDFDFDFDFDFDBD6D4D5DBDFDF1C
:10CA6000DFDFDFDFDFDFDFDFE0FFE0C0C1C7CFCF29
:10CA7000DFDFCFCFC7C1C0C0BF7F00FE0202F2829E
:10CA80008282F20202F29292926202023242824266
:10CA90003202020202020202020202020202020246
:10CAA00002020202020202020202020206FE060262
:10CAB000826212120A0A121262820206FE00007FCD
:10CAC00040404F4040404F40404F4142444840402A
:10CAD0004C4241424C404040404040404040404039
:10CAE0004040404040404040404040404040404046
:10CAF000607F604041464848505048484641406049
:10CB00007F0000FE0202F2828282F20202F2929220
:10CB100092620202324282423202020202020202A5
:10CB200002020202020202020202020202020202E5
:10CB30000202020206FE0602826212120A0A1212A1
:10CB400062820206FEFE003F40C0CFC0C0C0CFC020
:10CB5000C0CFC1C2C4C8C0C0CCC2C1C2CCC0C0C09A
:10CB6000C0C0C0C0C0C0C0C0C0C0C0C0C0C0C0C0C5
:10CB7000C0C0C0C0C0C0C0C0E0FFE0C0C1C6C8C81F
:10CB8000D0D0C8C8C6C1C0C0BF7F00FE06FA0A7AAE
:10CB90007A7A0AFAFA0A6A6A6A9AFAFACABA7ABA15
:10CBA000CAFAFAFAFAFAFAFAFAFAFAFAFAFAFAFA15
:10CBB000FAFAFAFAFAFAFAFAFAFAFAFA06FE0602B1
:10CBC00082E2F2F2FAFAF2F2E2820206FE00007F5C
:10CBD000605F505F5F5F505F5F505E5D5B575F5FA0
:10CBE000535D5E5D535F5F5F5F5F5F5F5F5F5F5F72
:10CBF0005F5F5F5F5F5F5F5F5F5F5F5F5F5F5F5F45
:10CC0000607F604041474F4F5F5F4F4F47414060FB
:10CC10007F0000FE06FA0A7A7A7A0AFAFA0A6A6A43
:10CC20006A9AFAFACABA7ABACAFAFAFAFAFAFAFAB4
:10CC3000FAFAFAFAFAFAFAFAFAFAFAFAFAFAFAFA54
:10CC4000FAFAFAFA06FE060282E2F2F2FAFAF2F2D0
:10CC5000E2820206FEFE003F60DFD0DFDFDFD0DFD2
:10CC6000DFD0DEDDDBD7DFDFD3DDDEDDD3DFDFDF0F
:10CC7000DFDFDFDFDFDFDFDFDFDFDFDFDFDFDFDFC4
:10CC8000DFDFDFDFDFDFDFDFE0FFE0C0C1C7CFCF07
:10CC9000DFDFCFCFC7C1C0C0BF7F00FE0202F2827C
:10CCA0008282F20202F29292926202020202020274
:10CCB000028202028202028282020282F282020264
:10CCC00082020282020282828202020206FE0602C0
:10CCD000826212120A0A121262820206FE00007FAB
:10CCE00040404F4040404F40404F41424448404107
:10CCF00041414141404F42414040474A4A4B4040F8
:10CD0000474848404F4241404047484848474040D4
:10CD1000607F604041464848505048484641406026
:10CD20007F0000FE0202F2828282F20202F29292FE
:10CD30009262020202020202028202028202028263
:10CD400082020282F2820202820202820202828253
:10CD50008202020206FE0602826212120A0A1212FF
:10CD600062820206FEFE003F40C0CFC0C0C0CFC0FE
:10CD7000C0CFC1C2C4C8C0C1C1C1C1C1C0CFC2C17E
:10CD8000C0C0C7CACACBC0C0C7C8C8C0CFC2C1C054
:10CD9000C0C7C8C8C8C7C0C0E0FFE0C0C1C6C8C8D7
:10CDA000D0D0C8C8C6C1C0C0BF7F00FE06FA0A7A8C
:10CDB0007A7A0AFAFA0A6A6A6A9AFAFAFAFAFAFAC3
:10CDC000FA7AFAFA7AFAFA7A7AFAFA7A0A7AFAFAB3
:10CDD0007AFAFA7AFAFA7A7A7AFAFAFA06FE06020F
:10CDE00082E2F2F2FAFAF2F2E2820206FE00007F3A
:10CDF000605F505F5F5F505F5F505E5D5B575F5E7F
:10CE00005E5E5E5E5F505D5E5F5F585555545F5F6E
:10CE10005857575F505D5E5F5F58575757585F5F71
:10CE2000607F604041474F4F5F5F4F4F47414060D9
:10CE30007F0000FE06FA0A7A7A7A0AFAFA0A6A6A21
:10CE40006A9AFAFAFAFAFAFAFA7AFAFA7AFAFA7AB2
:10CE50007AFAFA7A0A7AFAFA7AFAFA7AFAFA7A7AA2
:10CE60007AFAFAFA06FE060282E2F2F2FAFAF2F22E
:10CE7000E2820206FEFE003F60DFD0DFDFDFD0DFB0
:10CE8000DFD0DEDDDBD7DFDEDEDEDEDEDFD0DDDEE7
:10CE9000DFDFD8D5D5D4DFDFD8D7D7DFD0DDDEDFF1
:10CEA000DFD8D7D7D7D8DFDFE0FFE0C0C1C7CFCF0B
:10CEB000DFDFCFCFC7C1C0C0BF7F00FE0202F2825A
:10CEC0008282F20202F29292926202020202020252
:10CED00002020212121292720202221212926202D2
:10CEE00002820202028202020202020206FE06021E
:10CEF000826212120A0A121262820206FE00007F89
:10CF000040404F4040404F40404F414244484040E5
:10CF100041414141414040404E41404040404C4AE7
:10CF200049484840404845424548404040404040CC
:10CF3000607F604041464848505048484641406004
:10CF40007F0000FE0202F2828282F20202F29292DC
:10CF50009262020202020202020202121212927291
:10CF60000202221212926202028202020282020271
:10CF70000202020206FE0602826212120A0A12125D
:10CF800062820206FEFE003F40C0CFC0C0C0CFC0DC
:10CF9000C0CFC1C2C4C8C0C0C1C1C1C1C1C0C0C06E
:10CFA000CEC1C0C0C0C0CCCAC9C8C8C0C0C8C5C234
:10CFB000C5C8C0C0C0C0C0C0E0FFE0C0C1C6C8C8CE
:10CFC000D0D0C8C8C6C1C0C0BF7F00FE06FA0A7A6A
:10CFD0007A7A0AFAFA0A6A6A6A9AFAFAFAFAFAFAA1
:10CFE000FAFAFAEAEAEA6A8AFAFADAEAEA6A9AFA01
:10CFF000FA7AFAFAFA7AFAFAFAFAFAFA06FE06026D
:10D0000082E2F2F2FAFAF2F2E2820206FE00007F17
:10D01000605F505F5F5F505F5F505E5D5B575F5F5B
:10D020005E5E5E5E5E5F5F5F515E5F5F5F5F53553A
:10D030005657575F5F575A5D5A575F5F5F5F5F5F35
:10D04000607F604041474F4F5F5F4F4F47414060B7
:10D050007F0000FE06FA0A7A7A7A0AFAFA0A6A6AFF
:10D060006A9AFAFAFAFAFAFAFAFAFAEAEAEA6A8A40
:10D07000FAFADAEAEA6A9AFAFA7AFAFAFA7AFAFA40
:10D08000FAFAFAFA06FE060282E2F2F2FAFAF2F28C
:10D09000E2820206FEFE003F60DFD0DFDFDFD0DF8E
:10D0A000DFD0DEDDDBD7DFDFDEDEDEDEDEDFDFDFB3
:10D0B000D1DEDFDFDFDFD3D5D6D7D7DFDFD7DADDCD
:10D0C000DAD7DFDFDFDFDFDFE0FFE0C0C1C7CFCFD0
:10D0D000DFDFCFCFC7C1C0C0BF7F00FCFA060606A6
:10D0E000060606060606060606060606060686E680
:10D0F000763676E686060606F6F6060606F6F606A0
:10D1000006E6F6B6B6B6B6360606060606060606FF
:10D110000606060606060606060606FAFC00003F98
:10D120005F60606060606060606060606060606000
:10D13000606E6F63636363636F6E6060676F6C6C78
:10D140006C6F6F60606C6D6D6D6D6F67606060605F
:10D150006060606060606060606060606060605FD0
:10D160003F0000FCFA0606E6C68606060606060628
:10D1700006060606060686E6763676E6860606067F
:10D18000F6F6060606F6F60606E6F6B6B6B6B636BF
:10D19000060606060606060606060606060686C6EF
:10D1A000E60606FAFCFE003F5FE0E0EFE7E3E1E0C1
:10D1B000E0E0E0E0E0E0E0E0E0EEEFE3E3E3E3E343
:10D1C000EFEEE0E0E7EFECECECEFEFE0E0ECEDEDC4
:10D1D000EDEDEFE7E0E0E0E0E0E0E0E0E0E0E0E01F
:10D1E000E0E1E3E7EFE0E0DFBF7FFF0305F9F9F9F6
:10D1F000F9F9F9F9F9F9F9F9F9F9F9F9F9F97919FF
:10D2000089E9891979F9F9F90909F9F9F90909F99E
:10D21000F91909494949C9F9F9F9F9F9F9F9F9F98E
:10D22000F9F9F9F9F9F9F9F9F9F9F90503FFFFC085
:10D23000A09F9F9F9F9F9F9F9F9F9F9F9F9F9F9FFD
:10D240009F91909C9C9C9C9C90919F9F9890939365
:10D250009390909F9F9392929290989F9F9F9F9F51
:10D260009F9F9F9F9F9F9F9F9F9F9F9F9F9F9FA0CD
:10D27000C0FF00FCFA0606060606060606060606B7
:10D28000060606066696961626060686F68606069E
:10D290000686464686C60606C606864646060686AE
:10D2A000F6860606060606060606060606060606AE
:10D2B000060606FAFC00003F5F6060606060606028
:10D2C000606060606060606064686969666060603A
:10D2D0006768686060676868646F60606F616060FD
:10D2E0006060606067686860606060606060606027
:10D2F000606060606060605F3F0000FCFA0606E608
:10D30000C6860606060606060606060666969616ED
:10D3100026060686F68606060686464686C606065D
:10D32000C606864646060686F686060606060606ED
:10D3300006060606060686C6E60606FAFCFE003F58
:10D340005FE0E0EFE7E3E1E0E0E0E0E0E0E0E0E044
:10D35000E4E8E9E9E6E0E0E0E7E8E8E0E0E7E8E87B
:10D36000E4EFE0E0EFE1E0E0E0E0E0E0E7E8E8E083
:10D37000E0E0E0E0E0E0E0E0E0E1E3E7EFE0E0DF94
:10D38000BF7FFF0305F9F9F9F9F9F9F9F9F9F9F9A5
:10D39000F9F9F9F9996969E9D9F9F9790979F9F99D
:10D3A000F979B9B97939F9F939F979B9B9F9F9796D
:10D3B0000979F9F9F9F9F9F9F9F9F9F9F9F9F9F94D
:10D3C000F9F9F90503FFFFC0A09F9F9F9F9F9F9FB3
:10D3D0009F9F9F9F9F9F9F9F9B979696999F9F9F81
:10D3E0009897979F9F9897979B909F9F909E9F9F9E
:10D3F0009F9F9F9F9897979F9F9F9F9F9F9F9F9F54
:10D400009F9F9F9F9F9F9FA0C0FF2A3E003E00F8C6
:10D41000080808080808080808C8380000000000C4
:10D42000FF0000000000000000F8070000000000FE
:10D4300000FF000000000000C03F000000000000EE
:10D440000000FF0000000000F80700000000001CC2
:10D45000221C000F080808080F0000000000002A26
:10D460003E003E00F8080808080808080808C83800
:10D470000000000000FF0000000000000000F807AE
:10D48000000000000000FF000000000000C03F009E
:10D4900000000000000000FF0000000000F807008E
:10D4A000000000001C221C000F0C0C0C0C0F0000D4
:10D4B000000000002A3E003E00F80808080808089E
:10D4C000080808C8380000000000FF000000000045
:10D4D000000000F807000000000000FF000000004E
:10D4E0000000C03F0000000000000000FF0000003E
:10D4F0000000F80700000000001C221C000F0E0EA8
:10D500000E0E0F0000000000002A3E003E00F8084A
:10D510000808080808080808C8380000000000FFCC
:10D520000000000000000000F807000000000000FC
:10D53000FF000000000000C03F00000000000000ED
:10D5400000FF0000000000F80700000000001C229F
:10D550001C000F0F0F0F0F0F0000000000002A3EED
:10D56000003E00F8080808080808080808C838003D
:10D5700000000000FF0000000000000000F80700AD
:10D580000000000000FF000000000000C03F00009D
:10D59000000000000000FF8080808080F80700000D
:10D5A0000000001C221C000F0F0F0F0F0F000000C7
:10D5B0000000002A3E003E00F80808080808080895
:10D5C0000808C8380000000000FF0000000000004C
:10D5D0000000F807000000000000FF00000000004D
:10D5E00000C03F0000000000000000FFC0C0C0C03D
:10D5F000C0F80700000000001C221C000F0F0F0FD6
:10D600000F0F0000000000002A3E003E00F808084E
:10D6100008080808080808C8380000000000FF00D3
:10D6200000000000000000F807000000000000FFFC
:10D63000000000000000C03F0000000000000000EB
:10D64000FFE0E0E0E0E0F80700000000001C221C22
:10D65000000F0F0F0F0F0F0000000000002A3E0008
:10D660003E00F8080808080808080808C83800003C
:10D67000000000FF0000000000000000F8070000AC
:10D6800000000000FF000000000000C03F0000009C
:10D690000000000000FFF0F0F0F0F0F807000000DC
:10D6A00000001C221C000F0F0F0F0F0F00000000C6
:10D6B00000002A3E003E00F808080808080808088C
:10D6C00008C8380000000000FF0000000000000053
:10D6D00000F807000000000000FF0000000000004C
:10D6E000C03F0000000000000000FFF8F8F8F8F864
:10D6F000F80700000000001C221C000F0F0F0F0F86
:10D700000F0000000000002A3E003E00F808080854
:10D71000080808080808C8380000000000FF0000DA
:10D72000000000000000F807000000000000FF00FB
:10D730000000000000C03F0000000000000000FFEB
:10D74000FCFCFCFCFCFC0700000000001C221C0090
:10D750000F0F0F0F0F0F0000000000002A3E003EC9
:10D7600000F8080808080808080808C83800000079
:10D770000000FF0000000000000000F807000000AB
:10D78000000000FF000000000000C03F000000009B
:10D7900000000000FFFEFEFEFEFEFE07000000008F
:10D7A000001C221C000F0F0F0F0F0F0000000000C5
:10D7B000002A3E003E00F808080808080808080883
:10D7C000C8380000000000FF00000000000000005A
:10D7D000F807000000000000FF000000000000C08B
:10D7E0003F0000000000000000FFFFFFFFFFFFFF01
:10D7F0000700000000001C221C000F0F0F0F0F0F6E
:10D800000000000000002A3E003E00F8080808085A
:10D810000808080808C8380000000000FF000000E1
:10D820000000000000F807000000000000FF8080FA
:10D8300080808080C03F0000000000000000FFFFEB
:10D84000FFFFFFFFFF0700000000001C221C000F6D
:10D850000F0F0F0F0F0000000000002A3E003E00D7
:10D86000F8080808080808080808C8380000000078
:10D8700000FF0000000000000000F80700000000AA
:10D880000000FFC0C0C0C0C0C0C03F00000000001A
:10D89000000000FFFFFFFFFFFFFF07000000000088
:10D8A0001C221C000F0F0F0F0F0F000000000000C4
:10D8B0002A3E003E00F8080808080808080808C8BA
:10D8C000380000000000FF0000000000000000F829
:10D8D00007000000000000FFE0E0E0E0E0E0E03FE3
:10D8E0000000000000000000FFFFFFFFFFFFFF0738
:10D8F00000000000001C221C000F0F0F0F0F0F0074
:10D9000000000000002A3E003E00F8080808080851
:10D9100008080808C8380000000000FF00000000E8
:10D9200000000000F807000000000000FFF0F0F029
:10D93000F0F0F0F03F0000000000000000FFFFFFEB
:10D94000FFFFFFFF0700000000001C221C000F0F5C
:10D950000F0F0F0F0000000000002A3E003E00F8ED
:10D96000080808080808080808C83800000000006F
:10D97000FF0000000000000000F8070000000000A9
:10D9800000FFF8F8F8F8F8F8F83F00000000000091
:10D990000000FFFFFFFFFFFFFF0700000000001C6B
:10D9A000221C000F0F0F0F0F0F0000000000002AB5
:10D9B0003E003E00F8080808080808080808C838AB
:10D9C0000000000000FF0000000000000000F80759
:10D9D000000000000000FFFCFCFCFCFCFCFC3F0025
:10D9E00000000000000000FFFFFFFFFFFFFF070037
:10D9F000000000001C221C000F0F0F0F0F0F000073
:10DA0000000000002A3E003E00F808080808080848
:10DA1000080808C8380000000000FF0000000000EF
:10DA2000000000F807000000000000FFFEFEFEFE00
:10DA3000FEFEFE3F0000000000000000FFFFFFFFB1
:10DA4000FFFFFF0700000000001C221C000F0F0F4B
:10DA50000F0F0F0000000000002A3E003E00F808F3
:10DA60000808080808080808C8380000000000FF77
:10DA70000000000000000000F807000000000000A7
:10DA8000FFFFFFFFFFFFFFFF3F000000000000005F
:10DA900000FFFFFFFFFFFFFF0700000000001C2248
:10DAA0001C000F0F0F0F0F0F0000000000002A3E98
:10DAB000003E00F8080808080808080808C83800E8
:10DAC00000000000FF8080808080808080F8070058
:10DAD0000000000000FFFFFFFFFFFFFFFF3F00000F
:10DAE000000000000000FFFFFFFFFFFFFF07000036
:10DAF0000000001C221C000F0F0F0F0F0F00000072
:10DB00000000002A3E003E00F8080808080808083F
:10DB10000808C8380000000000FFC0C0C0C0C0C076
:10DB2000C0C0F807000000000000FFFFFFFFFFFF7C
:10DB3000FFFF3F0000000000000000FFFFFFFFFFAD
:10DB4000FFFF0700000000001C221C000F0F0F0F3A
:10DB50000F0F0000000000002A3E003E00F80808F9
:10DB600008080808080808C8380000000000FFE09E
:10DB7000E0E0E0E0E0E0E0F807000000000000FF87
:10DB8000FFFFFFFFFFFFFF3F00000000000000005D
:10DB9000FFFFFFFFFFFFFF0700000000001C221C2B
:10DBA000000F0F0F0F0F0F0000000000002A3E00B3
:10DBB0003E00F8080808080808080808C8380000E7
:10DBC000000000FFF0F0F0F0F0F0F0F0F8070000D7
:10DBD00000000000FFFFFFFFFFFFFFFF3F0000000E
:10DBE0000000000000FFFFFFFFFFFFFF0700000035
:10DBF00000001C221C000F0F0F0F0F0F0000000071
:10DC000000002A3E003E00F8080808080808080836
:10DC100008C8380000000000FFF8F8F8F8F8F8F835
:10DC2000F8F807000000000000FFFFFFFFFFFFFF04
:10DC3000FF3F0000000000000000FFFFFFFFFFFFAC
:10DC4000FF0700000000001C221C000F0F0F0F0F29
:10DC50000F0000000000002A3E003E00F8080808FF
:10DC6000080808080808C8380000000000FFFCFC8D
:10DC7000FCFCFCFCFCFCFC07000000000000FFFFBB
:10DC8000FFFFFFFFFFFF3F0000000000000000FF5C
:10DC9000FFFFFFFFFFFF0700000000001C221C0029
:10DCA0000F0F0F0F0F0F0000000000002A3E003E74
:10DCB00000F8080808080808080808C83800000024
:10DCC0000000FFFEFEFEFEFEFEFEFEFE0700000060
:10DCD000000000FFFFFFFFFFFFFFFF3F000000000D
:10DCE00000000000FFFFFFFFFFFFFF070000000034
:10DCF000001C221C000F0F0F0F0F0F000000000070
:10DD0000002A3E003E00F80808080808080808082D
:10DD1000C8380000000000FFFFFFFFFFFFFFFFFF0C
:10DD2000FF07000000000000FFFFFFFFFFFFFFFFF5
:10DD30003F0000000000000000FFFFFFFFFFFFFFAB
:10DD40000700000000001C221C000F0F0F0F0F0F18
:10DD50000000000000002A3E003E00F88888888805
:10DD60008888888888C8380000000000FFFFFFFF0F
:10DD7000FFFFFFFFFFFF07000000000000FFFFFFA5
:10DD8000FFFFFFFFFF3F0000000000000000FFFF5B
:10DD9000FFFFFFFFFF0700000000001C221C000F18
:10DDA0000F0F0F0F0F0000000000002A3E003E0082
:10DDB000F8C8C8C8C8C8C8C8C8C8C8380000000063
:10DDC00000FFFFFFFFFFFFFFFFFFFF070000000056
:10DDD0000000FFFFFFFFFFFFFFFF3F00000000000C
:10DDE000000000FFFFFFFFFFFFFF07000000000033
:10DDF0001C221C000F0F0F0F0F0F0000000000006F
:10DE00002A3E003E00F8E8E8E8E8E8E8E8E8E8E864
:10DE1000380000000000FFFFFFFFFFFFFFFFFFFFD4
:10DE200007000000000000FFFFFFFFFFFFFFFF3FB4
:10DE30000000000000000000FFFFFFFFFFFFFF07E2
:10DE400000000000001C221C000F0F0F0F0F0F001E
:10DE500000000000002A3E003E00F8F8F8F8F8F84C
:10DE6000F8F8F8F8F8380000000000FFFFFFFFFFA7
:10DE7000FFFFFFFFFF07000000000000FFFFFFFFA4
:10DE8000FFFFFFFF3F0000000000000000FFFFFF5A
:10DE9000FFFFFFFF0700000000001C221C000F0F07
:10DEA0000F0F0F0F00000000000000000000000036
:10DEB0000000000000000000000000000000000062
:10DEC0000000000000000000000000000000000052
:10DED0000000000000000000000000000000000042
:10DEE0000000000000000000000000000000000032
:10DEF0000000000000000000000000000000000022
:10DF00000000000000000000000000000000000011
:10DF10000000000000000000000000000000000001
:10DF200000000000000000000000000000000000F1
:10DF300000000000000000000000000000000000E1
:10DF400000000000000000000000000000000000D1
:10DF500000000000000000000000000000000000C1
:10DF600000000000000000000000000000000000B1
:10DF700000000000000000000000000000000000A1
:10DF80000000000000000000000000000000000091
:10DF90000000000000000000000000000000000081
:10DFA0000000000000000000000000000000000071
:10DFB0000000000000000000000000000000000061
:10DFC0000000000000000000000000000000000051
:10DFD0000000000000000000000000000000000041
:10DFE0000000000000000000000000000000000031
:10DFF0000000000000000000000000000000000021
:10E000000000000000000000000000000000000010
:10E010000000000000000000000000000000000000
:10E0200000000000000000000000000000000000F0
:10E0300000000000000000000000000000000000E0
:10E0400000000000000000000000000000000000D0
:10E0500000000000000000000000000000000000C0
:10E0600000000000000000000000000000000000B0
:10E0700000000000000000000000000000000000A0
:10E080000000000000000000000000000000000090
:10E090000000000000000000000000000000008000
:10E0A000B0B4B6B636363636363636363636363618
:10E0B00036360600000000F0F0F0F0F0F0F0F0F07E
:10E0C000F0E0C00000F0F0F00000C0E0F0F0F0F090
:10E0D000F0F0F0E0C00000F0F0F00000F0F0F00030
:10E0E00000000000000000F0F0F0F0F0F0F0F0F0C0
:10E0F000E0C00000F0F0F0000000000000000000B0
:10E10000000000606C6D6D6D0D01000000000000EE
:10E1100000000000C0C0C0C0C0C0C0C000FFFFFF02
:10E12000000000000000FFFFFF0000F8F8F800000A
:10E13000FFFFFFC0C0C0C0C0FFFFFF0000F8F8F83D
:10E140000000FFFFFF1E1E1E1E1E1E0000F0F8FC3A
:10E150003C3C3C3C3CFCFFFF0000FFFFFF0000009C
:10E16000000000000000C0D8DBDBDBDBC3C0C0C0A8
:10E17000C0C0C0C0C0C0C0C0000001010101010199
:10E18000010100FFFFFFF0F0F0F0F0F0FF7F3F0033
:10E1900000FFFFFF0000F0F1F3F3F3F3F3F3FF7F71
:10E1A0003F0000FFFFFF00003F7FFFF0F0F0F0F0C6
:10E1B000F000003F7FFFF0F0F0F0F0FF7F3F000045
:10E1C0003F7FFFF0F0F0F0F0F000000206060606D8
:10E1D00006060606060606060606060606000000F1
:10E1E000000000000000000000000000000000002F
:10E1F000000000000000000000000000000000001F
:10E20000000000000000000000000000000000000E
:10E2100000000000000000000000000000000000FE
:10E2200000000000000000000000000000000000EE
:10E230000000000000000080F8FE7E0600000000E4
:10E24000000080F8FE7E060080F8FE7E0E0E0E0EA8
:10E250000E0E0E0ECEFEFC380000000E7EFEF0808C
:10E26000000000000080E0F07C1E0F0301000000B1
:10E27000000000000000000000000000000000009E
:10E28000000000000000000000000000000000008E
:10E290000000000000000000000000C0F8FFFFC701
:10E2A000C0C0C0C0C0C0C0F8FF3F0700C0F8FFFF3B
:10E2B000C7C0C0C0C0C0C0C0F0FE7F0F01000000DA
:10E2C000000000037FFFFCF0783E0F070100000014
:10E2D000000000000000000000000000000000003E
:10E2E000000000000000000000000000000000002E
:10E2F000000000000000000000000000000000E03E
:10E30000FCFF1F03030303030303E3FFFF1F0300DB
:10E31000E0FCFF1F070F3FFDF1C1010101010100FA
:10E3200000000000000080E0F07C1E0F0F3FFFF0B7
:10E33000C00000000000000000000000000000001D
:10E3400000000000000000000000000000000000CD
:10E3500000000000000000000000000000000000BD
:10E36000000000607E7F1F01000000000000607E52
:10E370007F1F0100607E7F1F010000000000030F6F
:10E380003F7C7040000080C0F0783E0F0701000025
:10E3900000000000010F7F7E700000000000000000
:10E3A000000000000000000000000000000000006D
:10E3B000000000000000000000000000000000005D
:10E3C000000000000000000000000000000000004D
:10E3D000000000000000000000000000000000003D
:10E3E000000000000000000000000000000000002D
:10E3F000000000000000000000000000000000001D
:10E40000000000000000000000000000000000000C
:10E4100000000000000000000000000000000000FC
:10E4200000000000000000000000000000000000EC
:10E4300000000000000000000000000000000000DC
:10E4400000000000000000000000000000000000CC
:10E4500000000000000000000000000000000000BC
:10E4600000000000000000000000000000000000AC
:10E47000000000000000000000000000000000009C
:10E48000000000000000000000000000000000008C
:10E49000000000000000000080808080808080807C
:10E4A000808080808080808080808080808080806C
:10E4B000808080808080808080808080808080805C
:10E4C000808080808080808080808080808080804C
:10E4D000808080808080808080808080808080803C
:10E4E000808080808080808080808080808080802C
:10E4F000808080808080808080000030F0F0F17922
:10E500003D3F3733F1F1F1793D3F3733F1F1F179A7
:10E510003D3F3733F1F1F1793D3F3733F1F1F17997
:10E520003D3F3733F1F1F1793D3F3733F1F1F17987
:10E530003D3F3733F1F1F1793D3F3733F1F1F17977
:10E540003D3F3733F1F1F1793D3F3733F1F1F17967
:10E550003D3F3733F1F1F1793D3F373301010100A0
:10E5600000000000000000000000000000000000AB
:10E57000FCFC00000000000D0D000000001C3C0031
:10E58000001C3C000000000000002020F02C20F0C7
:10E590002C120F02120F0202F0F898FE9898100841
:10E5A00019197F191F0F18242498E0380C301C0704
:10E5B000192424181834C48404040006091010090E
:10E5C000061B00003C1C00000000000000000000D2
:10E5D00000E0F81C0C000000071F383000000000AD
:10E5E0000C1CF8E000000030381F0700000080809D
:10E5F000000000000001010000008080E0E0808059
:10E6000000010107070101000000000000000000F8
:10E61000301E0E000000808080808080800101011B
:10E6200001010101000000000000000000181800B6
:10E63000000000000000C0300C00300C030000009F
:10E64000F0F87C840CF8F00F1F30213E1F0F30389B
:10E650001CFCFC00000030303F3F303030381C0CD8
:10E660009CF8F0383C3E37333130181C0C8C8CFC55
:10E67000F818383031313F1FFCFC808080FCFC00F2
:10E68000010101013F3FFCFCCCCCCC8C0C18383094
:10E6900030391F0FC0E0F0B89C8C041F3F3131317E
:10E6A0003F1F0C0C0C8CCCFC78003E3F030100009B
:10E6B000F8FC8C8C8CFCF81F3F3131313F1FF8FC8B
:10E6C0008C8C8CFCF818393131313F1F00006060B0
:10E6D000000000000006060000000000006060006E
:10E6E000000020301E0E000080C06030180C0401B5
:10E6F00003060C18302060606060606060060606EB
:10E7000006060606040C183060C0802030180C067F
:10E710000301181C0C8CCCFC78000037370100007A
:10E72000E0108848C810E007081112131209F0F829
:10E730009C8C9CF8F01F1F0101011F1FFCFCCCCC1E
:10E74000CCFC381F1F1818181F0FF8FC0C0C0C3CC1
:10E75000380F1F1818181E0EFCFC0C0C1CF8F01FAC
:10E760001F18181C0F07FCFCCCCCCC0C0C1F1F185E
:10E7700018181818FCFC8C8C8C0C0C1F1F01010144
:10E780000000F8FC0C8C8C9C980F1F1819191F0F97
:10E79000FCFCC0C0C0FCFC1F1F0000001F1F00FCD1
:10E7A000FC00000000001F1F000000000C0C0C0CFF
:10E7B0000CFCFC0E1E3830381F0FFCFCC0E070381B
:10E7C0001C1F1F0103070E1CFCFC00000000001FA3
:10E7D0001F1818181818FCFC70E070FCFC1F1F00B4
:10E7E00000001F1FFCFC3CF000FCFC1F1F00031E70
:10E7F0001F1FF0F81C0C1CF8F0070F1C181C0F074B
:10E80000FCFC8C8C8CFCF81F1F0101010100F0F84E
:10E810000C0C0CF8F0070F181A1C0F13FCFCCCCCD6
:10E82000CCFC781F1F0103071E1C70F8DCCC9C98E1
:10E8300030060C1C191D0F070C0C0CFC0C0C0C00EA
:10E8400000001F000000FCFC000000FCFC0F1F1873
:10E85000180C1F1FFCFC800080FCFC00030F1E0F27
:10E860000300FCFC00F800FCFC0F1F1C0F1C1F0F1A
:10E870000C3CF0C0F03C0C181E0701071E187CFC75
:10E88000C0C0FC7C0000001F1F0000000C0C8CCCE2
:10E89000EC7C3C1E1F1B19181818FCFC0C0C0C0CF3
:10E8A000003F3F30303030000C30C000000000002E
:10E8B0000000030C3000000C0C0C0CFCFC00303091
:10E8C00030303F3F6030180C18306000000000000E
:10E8D00000000000000000000030303030303030E8
:10E8E00000000C3C00000000000000000000006080
:10E8F000606060E0C00E1F1B1B0F1F1FFCFC80C070
:10E90000C0C0801F1F0D18181F0F80C0E06060E09E
:10E91000C0070F1C18181C0C80C0C0C080FCFC0F66
:10E920001F18180D1F1FC0E0606060E0C00F1F1BA4
:10E930001B1B1B0BC0C0F8FCCCCC0C00003F3F00E5
:10E940000000C0E0606060E0C001333636363F1F33
:10E95000FCFCC0C0C0C0801F1F0000001F1F00CCF7
:10E96000CC00000000001F1F00000000000000009D
:10E97000ECEC001C3C30303F3F00FCFC0080C0E071
:10E98000601F1F03070F1C18FCFC0000000000079D
:10E990000F1C181C0C00E0E060C060E0C01F1F00EE
:10E9A0001F001F1FE0E0C0E0E0E0C01F1F010000EB
:10E9B0001F1F80C0E060E0C080070F1C181C0F07FD
:10E9C000E0E0606060E0C03F3F0606060703C0E08D
:10E9D000606060E0E003070606063F3FE0E080C0BD
:10E9E000C060601F1F0101000000C0E06060606047
:10E9F0004008191B1B1B1E0CC0C0FCFCC0C0C00083
:10EA0000000F1F181818E0E0000000E0E0070F18E2
:10EA1000180C1F1FE0E0000000E0E000030F1C0FD7
:10EA20000300E0E0000000E0E0070F1C0F1C0F07F0
:10EA300060E0800080E060181C0703071C18E0E01D
:10EA4000000000E0E001333333333F1F606060E0DB
:10EA5000E0E0601C1E1F1B19181880C070080C0C09
:10EA60000001030E103030000000FCFC000000002C
:10EA7000003F3F000000000C0C0870C080003030E8
:10EA8000100E0301C0E0E0C00080C00301000307D6
:10EA90000703FCF8F0E0C080007F3F1F0F07030171
:10EAA000FCFE1F6183FEFC43474C484F47430C0E5E
:10EAB00007FFFF0000404C4C4F4F4C4C0C0E87C3DF
:10EAC000E77E3C4E4F4F4D4C4C4C0607036363FFB3
:10EAD000FE464E4C4C4C4F473F7F606060FFFF400E
:10EAE000404040404F4F3F3F333373E3C3464E4CAB
:10EAF0004C4E4743F0F87C6E67E3C1474F4C4C4C9B
:10EB00004F470383C3E3733F1E404F4F4040404095
:10EB1000FEFF636363FFFE474F4C4C4C4F473E7F05
:10EB2000636363FFFE464E4C4C4C4F4760F0B0B001
:10EB3000B03020444C4D4D4D4F460080C0E0F0F8C1
:10EB4000FC0103070F1F3F7F000000000000004092
:10EB50004040404040400000000000000000000035
:10EB600000000000000000000000000000000000A5
:10EB70000000000000000000000000000000000095
:10EB80000000000000000000000000000000000085
:10EB90000000000000000000000000000000000075
:10EBA0000000000000000000000000000000000065
:10EBB0000000000000000000000000000000000055
:10EBC0000000000000000000000000000000000045
:10EBD0000000000000000000000000000000000035
:10EBE000000000000000000010284444C404040495
:10EBF000C444442810000000000000000000000091
:10EC000000F008040404F4F404040484C4E4670079
:10EC10000000078484848484848404040404040835
:10EC2000F00000FF00000000FFFF1C3E77E3C18002
:10EC30000000003E7FE3C1C1C1C1C163FFFE00000F
:10EC40000000FF00003F2020202023232020202040
:10EC5000212323202020282C2C2C2C2C2C2C2F273B
:10EC6000202020203F0000000000000000000000E5
:10EC700010284444C4040404C44444281000000080
:10EC8000000000000000000000F008040404F4F498
:10EC900004040484C4E4670000000784848484843A
:10ECA0008484040404040408F00000FF0000000051
:10ECB000FFFF1C3E77E3C1800000003E7FE3C1C13F
:10ECC000C1C1C163FFFE00000000FF00003F3F3FE5
:10ECD0003F3F3C3C3F3F3F3F3E3C3C3F3F3F373365
:10ECE00033333333333330383F3F3F3F3F0000004F
:10ECF000000000000000000010284444C404040484
:10ED0000C44444281000000000000000000000007F
:10ED100000F008040404F4F404040484C4E4670068
:10ED20000000078484848484848404040404040824
:10ED3000F00000FFF8F8F8F80707E4C68F1B3978F1
:10ED4000F8F8F8C6873B39393939399B0706F8F89E
:10ED5000F8F8FF00003F3F3F3F3F3C3C3F3F3F3F15
:10ED60003E3C3C3F3F3F373333333333333330382C
:10ED70003F3F3F3F3F000000000000000000000058
:10ED800010284444C4040404C4444428100000006F
:10ED9000000000000000000000F0C8C4C4C4343407
:10EDA000C4C4C4440424A7C0C0C0C74444444444A9
:10EDB0004444C4C4C4C4C4C8F00000FFFFFFFFFF44
:10EDC0000000E3C1881C3E7FFFFFFFC1803C3E3E48
:10EDD0003E3E3E9C0001FFFFFFFFFF00003F3F3F24
:10EDE0003F3F3C3C3F3F3F3F3E3C3C3F3F3F373354
:10EDF00033333333333330383F3F3F3F3F0000003E
:10EE0000000000000000000010387C7CFCFCFCFCD2
:10EE1000FC7C7C38100000000000000000000000B6
:10EE200000F0F8FCFCFC0C0CFCFCFC7C3C1C9FFF88
:10EE3000FFFFFF7C7C7C7C7C7C7CFCFCFCFCFCF88D
:10EE4000F00000FFFFFFFFFF0000E3C1881C3E7FD2
:10EE5000FFFFFFC1803C3E3E3E3E3E9C0001FFFF67
:10EE6000FFFFFF00003F3F3F3F3F3C3C3F3F3F3FF6
:10EE70003E3C3C3F3F3F373333333333333330381B
:10EE80003F3F3F3F3F000000000000000000000047
:10EE90000000000000000000000000000000000072
:10EEA0000000000000000000000000000000000062
:10EEB0000000000000000000000000000000000052
:10EEC0000000000000000000000000000000000042
:10EED0000000000000000000000000000000000032
:10EEE00000000000000000000000FCFA0606060614
:10EEF0000606066696961626060686F68606060612
:10EF000086464686C60606C606864646060686F631
:10EF1000860606060606060606FAFC003F5F6060E7
:10EF200060606060606468696966606060676868A6
:10EF30006060676868646F60606F61606060606097
:10EF400060676868606060606060605F3F00FCFAF6
:10EF500006E6C6860606066696961626060686F611
:10EF60008606060686464686C60606C606864646C1
:10EF7000060686F6860606060686C6E606FAFCFE3F
:10EF80003F5FE0EFE7E3E1E0E0E4E8E9E9E6E0E065
:10EF9000E0E7E8E8E0E0E7E8E8E4EFE0E0EFE1E020
:10EFA000E0E0E0E0E0E7E8E8E0E0E1E3E7EFE0DF31
:10EFB000BF7FFF0305F9F9F9F9F9F9996969E9D909
:10EFC000F9F9790979F9F9F979B9B97939F9F939A1
:10EFD000F979B9B9F9F9790979F9F9F9F9F9F9F991
:10EFE000F90503FFFFC0A09F9F9F9F9F9F9B979640
:10EFF00096999F9F9F9897979F9F9897979B909F71
:10F000009F909E9F9F9F9F9F9F9897979F9F9F9F37
:10F010009F9F9FA0C0FFFCFA06060606060606068E
:10F0200006066696961626060686F68606060606E0
:10F030008686860606068606868606060606060670
:10F040000606060606FAFC003F5F606060606060CE
:10F050006060606064686969666060606768686075
:10F0600060676868686760607F656464636060604B
:10F07000606060606060605F3F00FCFA06E6C68624
:10F080000606060606066696961626060686F68680
:10F090000606060686868606060686068686060610
:10F0A000060606060686C6E606FAFCFE3F5FE0EFA9
:10F0B000E7E3E1E0E0E0E0E0E4E8E9E9E6E0E0E021
:10F0C000E7E8E8E0E0E7E8E8E8E7E0E0FFE5E4E4D7
:10F0D000E3E0E0E0E0E0E1E3E7EFE0DFBF7FFF0354
:10F0E00005F9F9F9F9F9F9F9F9F9996969E9D9F934
:10F0F000F9790979F9F9F9F9797979F9F9F979F970
:10F100007979F9F9F9F9F9F9F9F9F9F9F90503FF53
:10F11000FFC0A09F9F9F9F9F9F9F9F9F9B9796969B
:10F12000999F9F9F9897979F9F98979797989F9F32
:10F13000809A9B9B9C9F9F9F9F9F9F9F9F9F9FA00D
:10F14000C0FFF0F8FC1E0E0E1EFCF8F0FFFFFF00E3
:10F15000000000FFFFFF070F1F3C38383C1F0F0760
:10F1600080C0E0F0783C1EFEFEFE030301000000BC
:10F1700000FFFFFF000000000000003F3F3FF8FCE1
:10F18000FE1E0E0E9EFEFCF8000080E0F8FE3F0F13
:10F1900003003C3E3F3F3B38383838381C1E1E0EBB
:10F1A0000E0E1EFEFCF80000001C1C1C3EFFF7E3C8
:10F1B0001C3C3C3838383C3F1F0FFEFEFE00000070
:10F1C00000FEFEFE070F1F1C1C1C1CFFFFFF0000A3
:10F1D00000000000003F3F3FFEFEFE0E0E0E0E0E32
:10F1E0000E0E0F0F0F0E0E0E1EFEFCF838383838BC
:10F1F00038383C3F1F0FFCFEFE0E0E0E0E1E1E1C6E
:10F20000FFFFFF1C1C1C1CFCFCF81F3F3F3838385C
:10F21000383F3F1F0E0E0E0E0E0E0EFEFEFC0000BF
:10F2200000C0F0FC3F0F030100003F3F3F00000023
:10F230000000F8FCFE1E0E0E1EFEFCF8E3F7FF3E7B
:10F240001C1C3EFFF7E30F1F3F3C38383C3F1F0FAD
:10F25000FCFEFE0E0E0E0EFEFEFC0F1F1F1C1C1CE5
:10F260001CFFFFFF183838383838383F3F1FF8FC8C
:10F27000FE1E0E0E1EFEFCF8FFFFFF80000080FF4A
:10F28000FFFF0103070707070707030180C0E0F03E
:10F29000783C1EFEFEFE03030100000000FFFFFF9E
:10F2A00000000000000000070707F8FCFE1E0E0E1D
:10F2B0001EFEFCF8C0E0F0783C1E0F0703010707B4
:10F2C00007070707070707071C1E1E0E0E0E1EFE68
:10F2D000FEFC8080800006068FFFFFF9030707070A
:10F2E000070707070703FEFEFE00000000FEFEFE04
:10F2F00003070F0E0E0E0EFFFFFF000000000000C0
:10F3000000070707FEFEFE0E0E0E0E0E0E0E07077E
:10F310000707070707FFFFFE070707070707070796
:10F320000703FCFEFE0E0E0E0E1E1E1CFFFFFF0747
:10F33000070707FFFFFE030707070707070707037E
:10F340000E0E0E0E0E0ECEFEFE3C0000C0F0FC3F78
:10F350000F03000000000707070000000000F8FC92
:10F36000FE1E0E0E1EFEFCF8F9FFFF8F06068FFF35
:10F37000FFF901030707070707070301FCFEFE0E5D
:10F380000E0E0EFEFEFC03070707070707FFFFFF31
:10F39000030707070707070707030000000000002F
:10F3A000000000000000000000000000000000005D
:10F3B00000000000000000000080808080808080CD
:10F3C000808080808080808080808080808080803D
:10F3D000808080808080808080808080808080802D
:10F3E0008080808080808080808080FF808080809E
:10F3F0008482BE80808080FF80808080B2AAAAA4A0
:10F40000808080FF80808080A2A2AA94808080FF7C
:10F4100080808080868888BE808080FF80FF80809A
:10F4200080AEAAAA9280808080FF808080BCAAAA39
:10F43000BA80808080FF80808082B28A86808080CF
:10F4400080FF808080BEAAAABE80808080FF80FF6F
:10F45000808080AEAAAA9E80808080FF808084BE4B
:10F46000809CA2A29C8080FF80808084BE8084BE1D
:10F47000808080FF808084BE80A4B2AAA48080FFA8
:10F4800080FF808084BE80A2A2AA948080FF8080BA
:10F4900084BE80868888BE8080FF808084BE80AEE7
:10F4A000AAAA928080FF808084BE80BCAAAABA806B
:10F4B00080FF80FF808084BE8082B28A868080FF49
:10F4C000808084BE80BEAAAABE8080FF808084BE69
:10F4D00080AEAAAA9E8080FF80A2B2AAA4809CA22D
:10F4E000A29C80FF80FF80B2AAAAA480808482BEF2
:10F4F00080FF80B2AAAAA480B2AAAAA480FF80B288
:10F50000AAAAA480A2A2AA9480FF80B2AAAAA480D8
:10F51000868888BE80FF80FF80B2AAAAA480AEAA97
:10F52000AA9280FF80B2AAAAA480BCAAAABA80FF2D
:10F5300080B2AAAAA48082B28A8680FF80B2AAAAD8
:10F54000A480BEAAAABE80FF80FF80B2AAAAA4801F
:10F55000AEAAAA9E80FF80A2A2AA94809CA2A29C8E
:10F5600080FF80A2A2AA94808084BE8080FF80A2B7
:10F57000A2AA9480B2AAAAA480FF80FF80A2A2AA15
:10F580009480A2A2AA9480FF80A2A2AA94808688D6
:10F5900088BE80FF80A2A2AA9480AEAAAA9280FF11
:10F5A00080A2A2AA9480BCAAAABA80FF8000000010
:10F5B000000000002F00000003000300543F147EF1
:10F5C000152E2A7F2A3A22152A5422122D29112873
:10F5D0000003000000001C2241000041221C00002A
:10F5E0000C0C000008083E08080040300000080825
:10F5F000080808004000000040300806013E474966
:10F60000713E0402017F0062514946002241493E99
:10F61000000708087F004F494931003C4A49300043
:10F62000016119070036494936002649497E000024
:10F63000001200000040340000081422410014149D
:10F64000141414004122140802290502000E152B7F
:10F650002D123E0909093E3F2525251A1E2121218B
:10F66000123F2121211E3F252525213F090909019E
:10F670001E2121293A3F0404043F3F0000000021DD
:10F680004141413F3F0C1221003F202020003F0616
:10F690000C063F3F030E183F1E2121211E3F090982
:10F6A00009061E2129112E3F0909192612252912A2
:10F6B0000001013F01011F2020203F030C300C03FB
:10F6C0001F301C301F221408142203043804033195
:10F6D00029252321007F41410001060830400041D7
:10F6E000417F00040201020440404040400001020A
:10F6F0000000102A2A2A3C3F242424181C222222FB
:10F7000022182424243F1C2A2A2A2C087E090100BE
:10F710004C5252523C3F040404383D00000000208B
:10F7200040403D003F081422001F202020003C02E2
:10F730003C023C3E0402023C1C2222221C7E12128D
:10F74000120C0C1212127E3E0404020214262A32FB
:10F7500014041F2424001E2020203E061820180612
:10F760001E201C201E24181824004E5050503E22EB
:10F77000322A2622083641410000007F0000414124
:10F780003E0800180408100C0000000000000000F3
:10F790000000000000000000000000000000000069
:10F7A00000000000000000C02010D012151D111D27
:10F7B0001512101020C0FF80809F848A918086A936
:10F7C000A9BE8080FFC02010D012151D111D15127A
:10F7D000101020C0FFF0F0EFF4FAE1F0F6D9D9CE26
:10F7E000F0F0FFC02010D012151D111D15121010C1
:10F7F00020C0FFFEFEE1FAF4EFFEF8D7D7C0FEFE10
:10F80000FFC0E0D010D2D5DDD1DDD5D2D0D0E0C060
:10F81000FFFFFFE0FBF5EEFFF9D6D6C1FFFFFFC00B
:10F82000E0F030F2F7FFFFFFF7F2F0F0E0C0FFFF8B
:10F83000FFE0FBF5EEFFF9D6D6C1FFFFFF0F3FFF5C
:10F84000FCF0C00000C0F0FCFF3F0F000000000310
:10F850000F3F7E7E3F0F03000000005500810081B6
:10F86000008100412214000000006A000000000036
:10F870000001020468000000000316504000000070
:10F880000000004050160300000000010514404035
:10F8900014050100000000FFFFFFC7C7C7C7C7EF7F
:10F8A000FFFE7C0000007F7F7F01010103071F7FB7
:10F8B0007C780000000080404020202040408000F4
:10F8C000000000000E31404E9191914040310E00F9
:10F8D0000000008060100808E42424C408081060B8
:10F8E000800007182040409F8385984040201807DB
:10F8F0000000000000000000000000000000000008
:10F9000000000000000000000000000000000000F7
:10F9100000000000000000000000000000000000E7
:10F9200000000000000000000000000000000000D7
:10F9300000000000000000000000000000000000C7
:10F9400000000000000000000000000000000000B7
:10F9500000000000000000000000000000000000A7
:10F960000000000000000000000000000000000097
:10F970000000000000000000000000000000000087
:10F980000000000000000000000000000000000077
:10F99000000000000000000000000000000000FE69
:10F9A00002FA0A0A0A0A0A0A0A0A0A0A0A0A0A0ACF
:10F9B0000A0A0A0A0A0A0A0A0A0A0A0A0A0A0A0AA7
:10F9C0000A0A0A0A0A0A0A0A0A0A8A8A8A8A8A8A97
:10F9D0008A8A8A8A8A8ACACACACACACACACACACA07
:10F9E000CAEAEAEAEAEAEAEAEAEAEAEAEAFAFAFA67
:10F9F000FAFAFAFA02FE7F405F5858585858585C95
:10FA00005C5C5C5C5C5C5C5C5C5C5C5E5E5E5E5E2C
:10FA10005E5E5E5E5E5E5F5F5F5F5F5F5F5F5F5FFC
:10FA20005F5F5F5F5F5F5F5F5F5F5F5F5F5F5F5FE6
:10FA30005F5F5F5F5F5F5F5F5F5F5F5F5F5F5F5FD6
:10FA40005F5F5F5F5F5F5F5F5F5F5F407F80808062
:10FA500080808080808080808C8C8C9EBFBFBFBF68
:10FA60009292928482898595B595858982848080D9
:10FA7000888494B494848880808080808090B090C2
:10FA8000808080808080808080A080808080809F37
:10FA9000909F80969589809F958A8080BFA1A1A123
:10FAA000A1A18780808080BFA1A1A181819F80804A
:10FAB0008080BFA1818181A1BF808080809F818162
:10FAC000A1A1A1BF8080808087A1A1A1A1A1BF80A9
:10FAD000808080B1A1A1A1A1A1BF80808080BCA0B5
:10FAE000A1A1A1A1BF80808080BFA0A0A0A1A1BF33
:10FAF00080808080BFA1A1A0A0A0BF80808080BFA7
:10FB0000A1A1A1A1A0BC80808080BFA1A1A1A1A131
:10FB1000B18080808C92A1A1A181828C8080808C18
:10FB200092A18181A1928C8080808C8281A1A1A1EF
:10FB3000928C8080808092A1A1A1A1928C808080F3
:10FB40008C90A0A1A1A1928C8080808C92A1A0A079
:10FB5000A1928C8080808C92A1A1A1A0908C8080A9
:10FB6000808C92A1A1A1A192808080BE8989BE8053
:10FB7000B8A8BF80B888406070787C7E7C78706060
:10FB80004002060E1E3E7E3E1E0E060200000000D3
:10FB900000000000000000808080808080808080E5
:10FBA0008080808080808080808080809E9EBFBF9B
:10FBB000AFB7BBBDAFB7BBBDAFB7BBBDAFB7BBBDCD
:10FBC000BF9E92A1A1A1B1B9BDAFB7BBBDAFB7BB3D
:10FBD000BDAFB7BBBDBF9E92A1A1A1A1A1A1A1B183
:10FBE000B9BDAFB7BBBDAFB7BBBDBF9E92A1A1A111
:10FBF000A1A1A1A1A1A1A1A1B1B9BDAFB7BBBDBF39
:10FC00009E92A1A1A1A1A1A1A1A1A1A1A1A1A1A1F6
:10FC1000A1B1B9BDBF9E92A1A1A1A1A1A1A1A1A184
:10FC2000A1A1A1A1A1A1A1A1A1BF9E92A1A1B1A9A0
:10FC3000A5A3B1A9A5A3B1A9A5A3B1A9A5A3BFFCDB
:10FC4000FE9393FEFC8098BCE6E6BCFFFF8080FE3E
:10FC5000FE988C8698BEB7B3B3B383B0BCBFB7B3BE
:10FC6000BB9F86B0BBBBBFB7870000000000000091
:10FC70000000000000000000000000000000000084
:10FC80000000000000000000000000000000000074
:10FC90000000000000000000000000000000000064
:10FCA0000000000000000000000000000000000054
:10FCB0000000000000000000000000000000000044
:10FCC0000000000000000000000000000000000034
:10FCD000000000000000007EFFC3FF7E000607FF5B
:10FCE000FFE7F3FBDFCEC3DBDBFF7E0F1F18FFFF59
:10FCF000DFDFDBFB737EFFDBFB7103F3FB1F0F66B4
:10FD0000FFDBFF660EDFDBFFFE00000000000000EF
:10FD100000000000000000000000000406FF0604D0
:10FD200000E3F3FBDFCFC70406FF060400FFFF1864
:10FD300018FFFF0406FF0604000303FFFF03030090
:10FD4000000000000000111B1511110A04111B1FF7
:10FD50001F1F0E0446756E6B2D5369676E616C3AFA
:10FD60000050726F66692F45636F2F4E5A004465CD
:10FD7000636F64657235362F35370048656C6C6982
:10FD8000676B6569743A00416B6B756C6164756E85
:10FD9000673A00525353492D4261636B3A00486100
:10FDA0006E647265676C6572005A77656974652068
:10FDB0004C6F6B004C6F6B616472657373650046CA
:10FDC000756E6B74696F6E656E00FEFF01FFFE7FDE
:10FDD000FF80FF7F536F6674776172653A004164FC
:10FDE000722D46756E6B3A0056657262696E646577
:10FDF0006E004C6F6B2D5375636865002D2D2D2D96
:10FE00002D2D2D2D004B6F6E74726173740056652D
:10FE10007273696F6E0050726F6772616D004C6F24
:10FE20006B7761686C00537461747573005265730D
:10FE3000657400536574757000413A00200020001D
:10FE400020002000200056657262696E64756E673E
:10FE5000206D69742043445A002020206E6575206F
:10FE6000617566626175656E2E00204C6173742049
:10FE700065696E7374656C6C656E00447265686B61
:10FE80006E6F706620647275652D006475726368AC
:10FE90007A756675656872656E2E004C6F6B61646D
:10FEA00072657373652050726F67004465636F6499
:10FEB00065722050726F6772616D00636B656E2CA6
:10FEC00020756D2065696E656E0048616E647265AF
:10FED000676C65722D5479700049324320616B74F0
:10FEE00075656C6C3A200050726F6772616D6D6958
:10FEF0006572656E002020202020202020202020F8
:10FF000020004932432D416472657373653A0041A4
:10FF1000647265737365206E65753A004C6F6B6132
:10FF20006472657373653A0048617570746D656ECF
:10FF30007565005A7765697465204C6F6B004C6F6E
:10FF40006B7765636873656C004C6F6B20737563CA
:10FF500068656E0046756E6B74696F6E656E0049FC
:10FF600032432D5374617475730056657262696E05
:10FF700064656E0052616E67696572656E004175F9
:10FF8000746F66616872740043445A2D49443A2084
:10FF9000005A656E7472616C65004B6F6E747261AD
:10FFA000737400426567696E6E3A004C6F6B7761DF
:10FFB000686C004272656D736500204F4B20200015
:10FFC0004164723A2000585858582000456E6465C4
:10FFD0003A00436F64653A00576572743A005245BF
:10FFE000534554005365747570004572726F72000A
:10FFF0005265736574004164723A003F3F3F0000F0
:020000040001F9
:100000000401116F0A0E04011119D8A40DD20001C8
:100010009F05D8A4A8D0000E9F6F070ED66F600072
:10002000D8F3D7F0010E06EC1AF0C00ED66FFF0E13
:10003000D76F060ED86F000ED96F010EDA6F000E63
:10004000DB6F000EDC6F000EDD6F000EDE6F000E4A
:10005000DF6FE1EC0BF0010E0101546F00019A0516
:10006000D8A404D0010E0101526F74D0600EC26F8B
:10007000E50EC36F070EC46F020EC56F000EC66F8C
:10008000000EC76F050EC86F000EC96F000ECA6F55
:10009000000ECB6F000ECC6F000ECD6F6000D8F35A
:1000A000CEF0C0EC06F0600EC26FE50EC36F070E17
:1000B000C46F020EC56F000EC66F090EC76F050E26
:1000C000C86F000EC96F000ECA6F000ECB6F000E16
:1000D000CC6F000ECD6F6000D8F3CEF0C0EC06F010
:1000E000600EC26FE50EC36F070EC46F020EC56FC0
:1000F000000EC66F120EC76F050EC86F000EC96FD7
:10010000000ECA6F000ECB6F000ECC6F000ECD6FCD
:100110006000D8F3CEF0C0EC06F0600EC26FE50EC2
:10012000C36F070EC46F020EC56F000EC66F1A0EA6
:10013000C76F050EC86F000EC96F000ECA6F000EA4
:10014000CB6F000ECC6F000ECD6F6000D8F3CEF0F9
:10015000C0EC06F0010E01015A6F010E576F010E3F
:10016000566FB8EC0DF001017405D8A431D0010E22
:10017000C56F295104E1320E285DD8A013D0460482
:10018000D8A410D0000E466E000E296F000E286F06
:10019000010E546F00019A05D8A421D0010E01016F
:1001A000526F1DD0295104E11E0E285DD8A017D032
:1001B0004650D8A414D0010E466E000E296F000ED2
:1001C000286F010E546F00019A05D8B4E7D707D005
:1001D000000E296F000E286F000EC56FF2D70101C7
:1001E0007305D8A41DD0010EC46F275104E1460E3B
:1001F000265DD8A005D07205D8A402D0000E0AD082
:10020000275104E1140E265DD8A012D07251D8A453
:100210000FD0010E726F000E276F000E266F06D0F2
:10022000000E276F000E266F000EC46F010E5A6F6E
:1002300000018751D8B403D03E04D8A46BD08651B6
:10024000D8B404D001014305D8A464D0000185517D
:10025000D8B404D001014105D8A45CD001015405F3
:10026000D8A424D000019A05D8A409D06000D8F100
:10027000D6F06000DCF1D7F045ECD1F008D060009A
:10028000D8F1D6F06000DCF1D7F0EFECDDF076C00D
:1002900078F077C079F06000E0F1BCF06000E4F144
:1002A000BDF05FEC0BF0000E0101546F5205D8A4B5
:1002B0000FD06000C0F1D6F06000C4F1D7F045EC7B
:1002C000D1F070C072F071C073F0000E0101526F76
:1002D0005A05D8A40AD000018F5110EC00F060003C
:1002E0003CF240F0000E01015A6F5705D8A406D029
:1002F000585176EC13F0000E0101576F5605D8A443
:1003000009D000018D51FDEC13F08DC08EF0000E70
:100310000101566F01014805D8A42BD049510001B5
:100320008719D8B423D001014905D8A410D0000EF4
:100330000001D76F000ED66F100ED86F020ED96F66
:10034000080ECCECD7F0010E0101C66F08D0010EEB
:1003500000019F6F000E0101C66F000E3E6E000E81
:1003600002016A6F000E696F49C187F0000E01013A
:10037000486F4205D8A429D03D5000018519D8B452
:1003800021D03D04D8A40FD0000ED76F000ED66F39
:10039000100ED86F020ED96F070ECCECD7F0010EFD
:1003A0000101C66F07D0010E9F6F000E0101C66FDD
:1003B000000E416F000E02016A6F000E696F60004F
:1003C000F4F085F0000E0101426F4405D8A412003C
:1003D000455100018619D8B423D001014505D8A4A0
:1003E00010D0000E0001D76F000ED66F100ED86F20
:1003F000020ED96F090ECCECD7F0010E0101C66FC9
:1004000008D0010E00019F6F000E0101C66F000EA3
:10041000436F000E02016A6F000E696F45C186F0DE
:10042000000E0101446F12000B0E1119D8A42CD03C
:1004300000019F05D8A414D0070ED66F6000D8F332
:10044000D7F0010E06EC1AF06A0EEA6FFE0EEB6FA3
:10045000110EEC6F32EC13F0000E9F6F010E9E6FC9
:1004600001015605D8B404D000019E05D8A412009D
:1004700000018D5140EC14F08DC08EF0000E9E6F87
:10048000000E0101566F12000C0E1119D8A40BD2E8
:10049000100E0F6F030E106F6C0E006F6C0E016F5D
:1004A0006C0E026F6C0E036F00019F05D8A4D8D0AC
:1004B0001E0EC26FAF0EC36F440EC46F050EC56F24
:1004C000000EC66F61003CF0C7F0610040F0C8F05C
:1004D000000EC96F000ECA6F010ECB6F000ECC6FFD
:1004E000000ECD6F6000D8F3CEF0C0EC06F01E0E0B
:1004F000C26FAF0EC36F440EC46F050EC56F0E0EF4
:10050000C66F61003CF0C7F0610040F0C8F0000E1B
:10051000C96F000ECA6F010ECB6F000ECC6F000EBC
:10052000CD6F6000D8F3CEF0C0EC06F0600EC26F65
:10053000E50EC36F070EC46F020EC56F6C0EC66F5B
:1005400004010F510C0F0001C76F04011051030F7C
:100550000001C86F000EC96F000ECA6F010ECB6F8D
:10056000000ECC6F000ECD6F6000D8F3CEF0C0EC63
:1005700006F0600EC26FE50EC36F070EC46F020E69
:10058000C56F6C0EC66F04010F51150F0001C76FC8
:1005900004011051030F0001C86F000EC96F000E57
:1005A000CA6F010ECB6F000ECC6F000ECD6F6000D6
:1005B000D8F3CEF0C0EC06F0600EC26FE50EC36F4C
:1005C000070EC46F020EC56F6C0EC66F04010F518B
:1005D0001E0F0001C76F04011051030F0001C86F07
:1005E000000EC96F000ECA6F010ECB6F000ECC6FEC
:1005F000000ECD6F6000D8F3CEF0C0EC06F0600EB8
:10060000C26FE50EC36F070EC46F020EC56F6C0E8E
:10061000C66F04010F51270F0001C76F040110516D
:10062000030F0001C86F000EC96F000ECA6F010EE4
:10063000CB6F000ECC6F000ECD6F6000D8F3CEF004
:10064000C0EC06F03E0EEA6FFF0EEB6F0B0EEC6F88
:1006500032EC13F0000E9F6F010E9E6F010E986F2B
:1006600001015405D8B404D000019E05D8A410D1CE
:10067000E80E0001765D030E7759D8A01CD0270E36
:10068000BF6F100EBE6F6000D8F1BCF06000DCF1EF
:10069000BDF0EFEC1AF06000F0F2C2F06000F4F28E
:1006A000C3F0030EC56FE80EC46FB0EC19F0C25171
:1006B000600F0401006F0001775104E1640E765D64
:1006C000D8A01CD0030EBF6FE80EBE6F6000D8F13B
:1006D000BCF06000DCF1BDF0EFEC1AF06000F0F26D
:1006E000C2F06000F4F2C3F0000EC56F640EC46F78
:1006F000B0EC19F0C251600F0401016F0001775195
:1007000004E10A0E765DD8A01CD0000EBF6F640E07
:10071000BE6F6000D8F1BCF06000DCF1BDF0EFEC22
:100720001AF06000F0F2C2F06000F4F2C3F0000EC4
:10073000C56F0A0EC46FB0EC19F0C251600F04010E
:10074000026F6000D8F1BCF06000DCF1BDF0000E7B
:100750000001BF6F0A0EBE6FEFEC1AF0BC51600FC4
:100760000401036F600E0001C26FE50EC36F070E38
:10077000C46F020EC56F610000F0C6F004010F5196
:100780000C0F0001C76F04011051030F0001C86F67
:10079000000EC96F000ECA6F010ECB6F000ECC6F3A
:1007A000000ECD6F6000D8F3CEF0C0EC06F0600E06
:1007B000C26FE50EC36F070EC46F020EC56F6100F6
:1007C00004F0C6F004010F51150F0001C76F0401BA
:1007D0001051030F0001C86F000EC96F000ECA6FE1
:1007E000010ECB6F000ECC6F000ECD6F6000D8F302
:1007F000CEF0C0EC06F0600EC26FE50EC36F070EC0
:10080000C46F020EC56F610008F0C6F004010F51FD
:100810001E0F0001C76F04011051030F0001C86FC4
:10082000000EC96F000ECA6F010ECB6F000ECC6FA9
:10083000000ECD6F6000D8F3CEF0C0EC06F0600E75
:10084000C26FE50EC36F070EC46F020EC56F610065
:100850000CF0C6F004010F51270F0001C76F04010F
:100860001051030F0001C86F000EC96F000ECA6F50
:10087000010ECB6F000ECC6F000ECD6F6000D8F371
:10088000CEF0C0EC06F0000E9E6F000E0101546F1A
:10089000410E0001BC6F140EBD6F9851BAEC13F0FD
:1008A0000101546F1200640E1119D8A4B0D30001D5
:1008B0009F05D8A416D0070ED66F6000D8F3D7F0E6
:1008C000010E06EC1AF0280EEA6FFF0EEB6F0B0E0E
:1008D000EC6F32EC13F0000E9F6F010E9E6F010E55
:1008E000946F9605D8B47CD39E05D8A4120078D313
:1008F0001E0EE96FFE0EEA6F080EEB6F600094F2B9
:10090000ECF0020E83ECF7F0690EC26FFC0EC36FC1
:100910005A0EC46F010EC56F000EC66F000EC76F72
:10092000040EC86F000EC96F000ECA6F000ECB6FA9
:10093000000ECC6F000ECD6F6000D8F3CEF0C0EC8F
:1009400006F0160ED66FFE0ED76F080ED86F030E88
:10095000D96F040EDA6F000EDB6F000EDC6F000E35
:10096000DD6F000EDE6F010EDF6FABECEBF0690E9A
:10097000C26FFC0EC36F660EC46F010EC56F000E12
:10098000C66F000EC76F050EC86F000EC96F000E50
:10099000CA6F000ECB6F000ECC6F000ECD6F6000E3
:1009A000D8F3CEF0C0EC06F0BF0ED66FFD0ED76FB9
:1009B0000B0ED86F030ED96F050EDA6F000EDB6FCA
:1009C000000EDC6F000EDD6F000EDE6F010EDF6FBC
:1009D000ABECEBF0690EC26FFC0EC36F660EC46F1A
:1009E000010EC56F000EC66F000EC76F060EC86FF2
:1009F000000EC96F000ECA6F000ECB6F000ECC6FD9
:100A0000000ECD6F6000D8F3CEF0C0EC06F0330ED0
:100A1000D66FFE0ED76F060ED86F030ED96F060E77
:100A2000DA6F000EDB6F000EDC6F000EDD6F000E64
:100A3000DE6F010EDF6FABECEBF0690EC26FFC0EE8
:100A4000C36F660EC46F010EC56F000EC66F000E39
:100A5000C76F070EC86F000EC96F000ECA6F000E79
:100A6000CB6F000ECC6F000ECD6F6000D8F3CEF0D0
:100A7000C0EC06F0260ED66FFE0ED76F070ED86FAD
:100A8000030ED96F070EDA6F000EDB6F000EDC6FFE
:100A9000000EDD6F000EDE6F010EDF6FABECEBF0D2
:100AA000AFD2160EE96FFE0EEA6F080EEB6F600014
:100AB00094F2ECF0030E83ECF7F0690EC26FFC0EBB
:100AC000C36F5A0EC46F010EC56F000EC66F000EC5
:100AD000C76F020EC86F000EC96F000ECA6F000EFE
:100AE000CB6F000ECC6F000ECD6F6000D8F3CEF050
:100AF000C0EC06F01E0ED66FFE0ED76F080ED86F34
:100B0000030ED96F020EDA6F000EDB6F000EDC6F82
:100B1000000EDD6F000EDE6F010EDF6FABECEBF051
:100B2000690EC26FFC0EC36F5A0EC46F010EC56F03
:100B3000000EC66F000EC76F050EC86F000EC96F9E
:100B4000000ECA6F000ECB6F000ECC6F000ECD6F83
:100B50006000D8F3CEF0C0EC06F0BF0ED66FFD0EED
:100B6000D76F0B0ED86F030ED96F050EDA6F000E1C
:100B7000DB6F000EDC6F000EDD6F000EDE6F010E0E
:100B8000DF6FABECEBF026D7BF0EE96FFD0EEA6F1F
:100B90000B0EEB6F600094F2ECF0040E83ECF7F0B8
:100BA000690EC26FFC0EC36F5A0EC46F010EC56F83
:100BB000000EC66F000EC76F020EC86F000EC96F21
:100BC000000ECA6F000ECB6F000ECC6F000ECD6F03
:100BD0006000D8F3CEF0C0EC06F01E0ED66FFE0E0D
:100BE000D76F080ED86F030ED96F020EDA6F000EA2
:100BF000DB6F000EDC6F000EDD6F000EDE6F010E8E
:100C0000DF6FABECEBF0690EC26FFC0EC36F5A0ED8
:100C1000C46F010EC56F000EC66F000EC76F030EC6
:100C2000C86F000EC96F000ECA6F000ECB6F000EAA
:100C3000CC6F000ECD6F6000D8F3CEF0C0EC06F0A4
:100C4000160ED66FFE0ED76F080ED86F030ED96F33
:100C5000030EDA6F000EDB6F000EDC6F000EDD6F2F
:100C6000000EDE6F010EDF6FABECEBF0690EC26FB2
:100C7000FC0EC36F5A0EC46F010EC56F000EC66F17
:100C8000000EC76F060EC86F000EC96F000ECA6F48
:100C9000000ECB6F000ECC6F000ECD6F6000D8F34E
:100CA000CEF0C0EC06F0B3D6330EE96FFE0EEA6F5D
:100CB000060EEB6F600094F2ECF0050E83ECF7F09B
:100CC000690EC26FFC0EC36F5A0EC46F010EC56F62
:100CD000000EC66F000EC76F020EC86F000EC96F00
:100CE000000ECA6F000ECB6F000ECC6F000ECD6FE2
:100CF0006000D8F3CEF0C0EC06F01E0ED66FFE0EEC
:100D0000D76F080ED86F030ED96F020EDA6F000E80
:100D1000DB6F000EDC6F000EDD6F000EDE6F010E6C
:100D2000DF6FABECEBF0690EC26FFC0EC36F5A0EB7
:100D3000C46F010EC56F000EC66F000EC76F030EA5
:100D4000C86F000EC96F000ECA6F000ECB6F000E89
:100D5000CC6F000ECD6F6000D8F3CEF0C0EC06F083
:100D6000160ED66FFE0ED76F080ED86F030ED96F12
:100D7000030EDA6F000EDB6F000EDC6F000EDD6F0E
:100D8000000EDE6F010EDF6FABECEBF0690EC26F91
:100D9000FC0EC36F5A0EC46F010EC56F000EC66FF6
:100DA000000EC76F040EC86F000EC96F000ECA6F29
:100DB000000ECB6F000ECC6F000ECD6F6000D8F32D
:100DC000CEF0C0EC06F0BF0ED66FFD0ED76F0B0E47
:100DD000D86F030ED96F040EDA6F000EDB6F000EB2
:100DE000DC6F000EDD6F000EDE6F010EDF6FABEC0F
:100DF000EBF0690EC26FFC0EC36F5A0EC46F010E8A
:100E0000C56F000EC66F000EC76F070EC86F000ECD
:100E1000C96F000ECA6F000ECB6F000ECC6F000EB4
:100E2000CD6F6000D8F3CEF0C0EC06F023D6260ECE
:100E3000E96FFE0EEA6F070EEB6F600094F2ECF0C4
:100E4000060E83ECF7F0690EC26FFC0EC36F5A0EEC
:100E5000C46F010EC56F000EC66F000EC76F020E85
:100E6000C86F000EC96F000ECA6F000ECB6F000E68
:100E7000CC6F000ECD6F6000D8F3CEF0C0EC06F062
:100E80001E0ED66FFE0ED76F080ED86F030ED96FE9
:100E9000020EDA6F000EDB6F000EDC6F000EDD6FEE
:100EA000000EDE6F010EDF6FABECEBF0690EC26F70
:100EB000FC0EC36F5A0EC46F010EC56F000EC66FD5
:100EC000000EC76F030EC86F000EC96F000ECA6F09
:100ED000000ECB6F000ECC6F000ECD6F6000D8F30C
:100EE000CEF0C0EC06F0160ED66FFE0ED76F080ED1
:100EF000D86F030ED96F030EDA6F000EDB6F000E92
:100F0000DC6F000EDD6F000EDE6F010EDF6FABECED
:100F1000EBF0690EC26FFC0EC36F5A0EC46F010E68
:100F2000C56F000EC66F000EC76F040EC86F000EAF
:100F3000C96F000ECA6F000ECB6F000ECC6F000E93
:100F4000CD6F6000D8F3CEF0C0EC06F0BF0ED66FC8
:100F5000FD0ED76F0B0ED86F030ED96F040EDA6F2C
:100F6000000EDB6F000EDC6F000EDD6F000EDE6F1B
:100F7000010EDF6FABECEBF0690EC26FFC0EC36FBE
:100F80005A0EC46F010EC56F000EC66F000EC76FFC
:100F9000050EC86F000EC96F000ECA6F000ECB6F32
:100FA000000ECC6F000ECD6F6000D8F3CEF0C0EC19
:100FB00006F0330ED66FFE0ED76F060ED86F030EF7
:100FC000D96F050EDA6F000EDB6F000EDC6F000EBE
:100FD000DD6F000EDE6F010EDF6FABECEBF010D0BB
:100FE0009451010AD8B484D4030AD8B45AD5010A5A
:100FF000D8B4CAD5070AD8B457D6010AD8B417D777
:1010000094C095F0000E966F000E9E6F1200650E54
:101010001119D8A474D000019F05D8A448D0070E98
:10102000D66F6000D8F3D7F0010E06EC1AF0AB0EC5
:10103000EA6FFF0EEB6F080EEC6F32EC13F01C0E34
:10104000D66FFF0ED76F0C0ED86F000ED96F020E41
:10105000DA6F000EDB6F000EDC6F000EDD6F000E2E
:10106000DE6F000EDF6FE1EC0BF0B105D8A406D007
:101070005A0ED66F480EB9EC01F013D0020EB1191A
:10108000D8A406D05A0ED66F200EB9EC01F009D0C4
:10109000030EB119D8A405D05A0ED66F200EB9ECA4
:1010A00001F0000E9F6F010E9E6F010E986F0101FF
:1010B0005405D8B404D000019E05D8A415D0600012
:1010C000D8F1D6F06000DCF1D7F00A0E0001D86F3D
:1010D000040ED96F600094F2DAF068ECCAF0000EEA
:1010E0009E6F000E0101546F410E0001BC6F140E83
:1010F000BD6F9851BAEC13F00101546F12006D0EE0
:101100001119D8A453D300019F05D8A495D1070E77
:10111000D66F6000D8F3D7F0010E06EC1AF0630E1C
:10112000EA6FFF0EEB6F070EEC6F32EC13F090518D
:10113000D8B459D0870ED66FFD0ED76F0C0ED86F6E
:10114000000ED96F020EDA6F000EDB6F000EDC6F3F
:10115000000EDD6F000EDE6F010EDF6FABECEBF00B
:10116000540ED66FFD0ED76F0D0ED86F000ED96FCF
:10117000030EDA6F000EDB6F000EDC6F000EDD6F0A
:10118000000EDE6F010EDF6FABECEBF0DE0ED66F04
:10119000FD0ED76F0A0ED86F000ED96F040EDA6FEE
:1011A000000EDB6F000EDC6F000EDD6F000EDE6FD9
:1011B000010EDF6FABECEBF0930ED66FFD0ED76F29
:1011C0000B0ED86F000ED96F050EDA6F000EDB6FB5
:1011D000000EDC6F000EDD6F000EDE6F010EDF6FA4
:1011E000ABECEBF058D0880ED66FFF0ED76F090E20
:1011F000D86F000ED96F020EDA6F000EDB6F000E93
:10120000DC6F000EDD6F000EDE6F010EDF6FABECEA
:10121000EBF0D90ED66FFE0ED76F0E0ED86F000E04
:10122000D96F030EDA6F000EDB6F000EDC6F000E5D
:10123000DD6F000EDE6F010EDF6FABECEBF0020E28
:10124000D66FFF0ED76F0D0ED86F000ED96F040E3C
:10125000DA6F000EDB6F000EDC6F000EDD6F000E2C
:10126000DE6F010EDF6FABECEBF05F0ED66FFF0EA3
:10127000D76F0B0ED86F000ED96F050EDA6F000E08
:10128000DB6F000EDC6F000EDD6F000EDE6F010EF7
:10129000DF6FABECEBF07B0ED66FFD0ED76F0C0E55
:1012A000D86F000ED96F060EDA6F000EDB6F000EDE
:1012B000DC6F000EDD6F000EDE6F010EDF6FABEC3A
:1012C000EBF0D40ED66FFD0ED76F0A0ED86F000E5E
:1012D000D96F070EDA6F000EDB6F000EDC6F000EA9
:1012E000DD6F000EDE6F010EDF6FABECEBF0C70EB3
:1012F000D66FFF0ED76F050ED86F4F0ED96F020E47
:10130000DA6F000EDB6F000EDC6F000EDD6F000E7B
:10131000DE6F010EDF6FABECEBF0C70ED66FFF0E8A
:10132000D76F050ED86F4F0ED96F030EDA6F000E10
:10133000DB6F000EDC6F000EDD6F000EDE6F010E46
:10134000DF6FABECEBF0C70ED66FFF0ED76F050E5D
:10135000D86F4F0ED96F040EDA6F000EDB6F000EE0
:10136000DC6F000EDD6F000EDE6F010EDF6FABEC89
:10137000EBF0C70ED66FFF0ED76F050ED86F4F0E6E
:10138000D96F050EDA6F000EDB6F000EDC6F000EFA
:10139000DD6F000EDE6F010EDF6FABECEBF0C70E02
:1013A000D66FFF0ED76F050ED86F4F0ED96F060E92
:1013B000DA6F000EDB6F000EDC6F000EDD6F000ECB
:1013C000DE6F010EDF6FABECEBF0390ED66FFE0E69
:1013D000D76F030ED86F420ED96F070EDA6F000E6B
:1013E000DB6F000EDC6F000EDD6F000EDE6F010E96
:1013F000DF6FABECEBF0EF0ED66F020ED76F050E82
:10140000D86F4F0ED96F070EDA6F000EDB6F000E2C
:10141000DC6F000EDD6F000EDE6F010EDF6FABECD8
:10142000EBF0000E9F6F010E0101656F010EB46FAE
:10143000010EB26F010EAD6F00019051D8B4B8D05B
:1014400001015D05D8A42CD0FC0E0001D66FFE0E64
:10145000D76F060ED86F430ED96F020EDA6F000EEB
:10146000DB6F000EDC6F000EDD6F000EDE6F000E16
:10147000DF6FABECEBF0600030F4D6F0600034F4DA
:10148000D7F04F0ED86F020ED96F000EDA6F000E34
:10149000DB6F000EDC6F89ECD4F0000E01015D6F94
:1014A0006205D8A42AD0FC0E0001D66FFE0ED76FBD
:1014B000060ED86F430ED96F030EDA6F000EDB6F86
:1014C000000EDC6F000EDD6F000EDE6F000EDF6FB2
:1014D000ABECEBF060008CF5D6F0D76B4F0ED86F0D
:1014E000030ED96F000EDA6F000EDB6F000EDC6F9B
:1014F00089ECD4F0000E0101626FB405D8A42AD0A3
:10150000FC0E0001D66FFE0ED76F060ED86F430E8D
:10151000D96F040EDA6F000EDB6F000EDC6F000E69
:10152000DD6F000EDE6F000EDF6FABECEBF06000E6
:101530006CF1D6F0D76B4F0ED86F040ED96F000E3A
:10154000DA6F000EDB6F000EDC6F89ECD4F0000E5A
:101550000101B46F9F05D8A4F9D0FC0E0001D66F2D
:10156000FE0ED76F060ED86F430ED96F050EDA6FD9
:10157000000EDB6F000EDC6F000EDD6F000EDE6F05
:10158000000EDF6FABECEBF060008CF6D6F0D76BA3
:101590004F0ED86F050ED96F000EDA6F000EDB6F9D
:1015A000000EDC6F89ECD4F0000E01019F6FCED0ED
:1015B00001016505D8A42AD0FC0E0001D66FFE0EED
:1015C000D76F060ED86F430ED96F020EDA6F000E7A
:1015D000DB6F000EDC6F000EDD6F000EDE6F000EA5
:1015E000DF6FABECEBF0600008F1D6F0D76B4F0E7D
:1015F000D86F020ED96F000EDA6F000EDB6F000E8F
:10160000DC6F89ECD4F0000E0101656FB205D8A43F
:1016100050D0FC0E0001D66FFE0ED76F060ED86FAD
:10162000430ED96F030EDA6F000EDB6F000EDC6F16
:10163000000EDD6F000EDE6F000EDF6FABECEBF027
:101640006000D4F2D6F0D76B4F0ED86F030ED96F6F
:10165000000EDA6F000EDB6F000EDC6F89ECD4F049
:10166000FC0ED66FFE0ED76F060ED86F430ED96FE5
:10167000040EDA6F000EDB6F000EDC6F000EDD6F04
:10168000000EDE6F000EDF6FABECEBF06000C8F217
:10169000D6F0D76B4F0ED86F040ED96F000EDA6FED
:1016A000000EDB6F000EDC6F89ECD4F0000E010140
:1016B000B26FAD05D8A44AD0FC0E0001D66FFE0E65
:1016C000D76F060ED86F430ED96F050EDA6F000E76
:1016D000DB6F000EDC6F000EDD6F000EDE6F000EA4
:1016E000DF6FABECEBF0AF05D8A417D0BA0ED66F16
:1016F000FF0ED76F060ED86F4A0ED96F050EDA6F40
:10170000000EDB6F000EDC6F000EDD6F000EDE6F73
:10171000010EDF6FABECEBF016D0EA0ED66FFF0ECA
:10172000D76F060ED86F490ED96F050EDA6F000E0F
:10173000DB6F000EDC6F000EDD6F000EDE6F010E42
:10174000DF6FABECEBF0000E0101AD6F7D05D8A4AF
:101750001200FC0E0001D66FFE0ED76F060ED86F7A
:10176000430ED96F060EDA6F000EDB6F000EDC6FD2
:10177000000EDD6F000EDE6F000EDF6FABECEBF0E6
:10178000600068F4D6F060006CF4D7F04F0ED86FAC
:10179000060ED96F000EDA6F000EDB6F000EDC6FE5
:1017A00089ECD4F0000E01017D6F12006E0E11194C
:1017B000D8A4ADD300019F05D8A416D0070ED66FCC
:1017C0006000D8F3D7F0010E06EC1AF0E70EEA6FCE
:1017D000FE0EEB6F0E0EEC6F32EC13F0000E9F6FEF
:1017E000010E9E6F010E946F9605D8B47ED39E05B0
:1017F000D8A412007AD36E0EE96FFD0EEA6F0D0EBB
:10180000EB6F600094F2ECF0020E83ECF7F0690EDF
:10181000C26FFC0EC36F5A0EC46F010EC56F000E6F
:10182000C66F000EC76F040EC86F000EC96F000EA2
:10183000CA6F000ECB6F000ECC6F000ECD6F600034
:10184000D8F3CEF0C0EC06F0610ED66FFD0ED76F68
:101850000D0ED86F030ED96F040EDA6F000EDB6F1A
:10186000000EDC6F000EDD6F000EDE6F010EDF6F0D
:10187000ABECEBF0690EC26FFC0EC36F660EC46F6B
:10188000010EC56F000EC66F000EC76F050EC86F44
:10189000000EC96F000ECA6F000ECB6F000ECC6F2A
:1018A000000ECD6F6000D8F3CEF0C0EC06F0B40EA1
:1018B000D66FFD0ED76F0B0ED86F030ED96F050EC6
:1018C000DA6F000EDB6F000EDC6F000EDD6F000EB6
:1018D000DE6F010EDF6FABECEBF0690EC26FFC0E3A
:1018E000C36F660EC46F010EC56F000EC66F000E8B
:1018F000C76F060EC86F000EC96F000ECA6F000ECC
:10190000CB6F000ECC6F000ECD6F6000D8F3CEF021
:10191000C0EC06F0440ED66FFE0ED76F020ED86FE5
:10192000030ED96F060EDA6F000EDB6F000EDC6F50
:10193000000EDD6F000EDE6F010EDF6FABECEBF023
:10194000690EC26FFC0EC36F660EC46F010EC56FC9
:10195000000EC66F000EC76F070EC86F000EC96F6E
:10196000000ECA6F000ECB6F000ECC6F000ECD6F55
:101970006000D8F3CEF0C0EC06F0420ED66FFE0E3B
:10198000D76F020ED86F030ED96F070EDA6F000EF5
:10199000DB6F000EDC6F000EDD6F000EDE6F010EE0
:1019A000DF6FABECEBF000EF88F0610EE96FFD0E3E
:1019B000EA6F0D0EEB6F600094F2ECF0030E83EC17
:1019C000F7F0690EC26FFC0EC36F5A0EC46F010EA2
:1019D000C56F000EC66F000EC76F020EC86F000EF7
:1019E000C96F000ECA6F000ECB6F000ECC6F000ED9
:1019F000CD6F6000D8F3CEF0C0EC06F06E0ED66F5F
:101A0000FD0ED76F0D0ED86F030ED96F020EDA6F71
:101A1000000EDB6F000EDC6F000EDD6F000EDE6F60
:101A2000010EDF6FABECEBF0690EC26FFC0EC36F03
:101A30005A0EC46F010EC56F000EC66F000EC76F41
:101A4000050EC86F000EC96F000ECA6F000ECB6F77
:101A5000000ECC6F000ECD6F6000D8F3CEF0C0EC5E
:101A600006F0B40ED66FFD0ED76F0B0ED86F030EB7
:101A7000D96F050EDA6F000EDB6F000EDC6F000E03
:101A8000DD6F000EDE6F010EDF6FABECEBF025D7E4
:101A9000B40EE96FFD0EEA6F0B0EEB6F600094F26F
:101AA000ECF0040E83ECF7F0690EC26FFC0EC36F0E
:101AB0005A0EC46F010EC56F000EC66F000EC76FC1
:101AC000020EC86F000EC96F000ECA6F000ECB6FFA
:101AD000000ECC6F000ECD6F6000D8F3CEF0C0ECDE
:101AE00006F06E0ED66FFD0ED76F0D0ED86F030E7B
:101AF000D96F020EDA6F000EDB6F000EDC6F000E86
:101B0000DD6F000EDE6F010EDF6FABECEBF0690EE8
:101B1000C26FFC0EC36F5A0EC46F010EC56F000E6C
:101B2000C66F000EC76F030EC86F000EC96F000EA0
:101B3000CA6F000ECB6F000ECC6F000ECD6F600031
:101B4000D8F3CEF0C0EC06F0610ED66FFD0ED76F65
:101B50000D0ED86F030ED96F030EDA6F000EDB6F18
:101B6000000EDC6F000EDD6F000EDE6F010EDF6F0A
:101B7000ABECEBF0690EC26FFC0EC36F5A0EC46F74
:101B8000010EC56F000EC66F000EC76F060EC86F40
:101B9000000EC96F000ECA6F000ECB6F000ECC6F27
:101BA000000ECD6F6000D8F3CEF0C0EC06F0B2D6D8
:101BB000440EE96FFE0EEA6F020EEB6F600094F2C6
:101BC000ECF0050E83ECF7F0690EC26FFC0EC36FEC
:101BD0005A0EC46F010EC56F000EC66F000EC76FA0
:101BE000020EC86F000EC96F000ECA6F000ECB6FD9
:101BF000000ECC6F000ECD6F6000D8F3CEF0C0ECBD
:101C000006F06E0ED66FFD0ED76F0D0ED86F030E59
:101C1000D96F020EDA6F000EDB6F000EDC6F000E64
:101C2000DD6F000EDE6F010EDF6FABECEBF0690EC7
:101C3000C26FFC0EC36F5A0EC46F010EC56F000E4B
:101C4000C66F000EC76F030EC86F000EC96F000E7F
:101C5000CA6F000ECB6F000ECC6F000ECD6F600010
:101C6000D8F3CEF0C0EC06F0610ED66FFD0ED76F44
:101C70000D0ED86F030ED96F030EDA6F000EDB6FF7
:101C8000000EDC6F000EDD6F000EDE6F010EDF6FE9
:101C9000ABECEBF0690EC26FFC0EC36F5A0EC46F53
:101CA000010EC56F000EC66F000EC76F040EC86F21
:101CB000000EC96F000ECA6F000ECB6F000ECC6F06
:101CC000000ECD6F6000D8F3CEF0C0EC06F0B40E7D
:101CD000D66FFD0ED76F0B0ED86F030ED96F040EA3
:101CE000DA6F000EDB6F000EDC6F000EDD6F000E92
:101CF000DE6F010EDF6FABECEBF0690EC26FFC0E16
:101D0000C36F5A0EC46F010EC56F000EC66F000E72
:101D1000C76F070EC86F000EC96F000ECA6F000EA6
:101D2000CB6F000ECC6F000ECD6F6000D8F3CEF0FD
:101D3000C0EC06F022D6420EE96FFE0EEA6F020EEC
:101D4000EB6F600094F2ECF0060E83ECF7F0690E96
:101D5000C26FFC0EC36F5A0EC46F010EC56F000E2A
:101D6000C66F000EC76F020EC86F000EC96F000E5F
:101D7000CA6F000ECB6F000ECC6F000ECD6F6000EF
:101D8000D8F3CEF0C0EC06F06E0ED66FFD0ED76F16
:101D90000D0ED86F030ED96F020EDA6F000EDB6FD7
:101DA000000EDC6F000EDD6F000EDE6F010EDF6FC8
:101DB000ABECEBF0690EC26FFC0EC36F5A0EC46F32
:101DC000010EC56F000EC66F000EC76F030EC86F01
:101DD000000EC96F000ECA6F000ECB6F000ECC6FE5
:101DE000000ECD6F6000D8F3CEF0C0EC06F0610EAF
:101DF000D66FFD0ED76F0D0ED86F030ED96F030E81
:101E0000DA6F000EDB6F000EDC6F000EDD6F000E70
:101E1000DE6F010EDF6FABECEBF0690EC26FFC0EF4
:101E2000C36F5A0EC46F010EC56F000EC66F000E51
:101E3000C76F040EC86F000EC96F000ECA6F000E88
:101E4000CB6F000ECC6F000ECD6F6000D8F3CEF0DC
:101E5000C0EC06F0B40ED66FFD0ED76F0B0ED86F28
:101E6000030ED96F040EDA6F000EDB6F000EDC6F0D
:101E7000000EDD6F000EDE6F010EDF6FABECEBF0DE
:101E8000690EC26FFC0EC36F5A0EC46F010EC56F90
:101E9000000EC66F000EC76F050EC86F000EC96F2B
:101EA000000ECA6F000ECB6F000ECC6F000ECD6F10
:101EB0006000D8F3CEF0C0EC06F0440ED66FFE0EF4
:101EC000D76F020ED86F030ED96F050EDA6F000EB2
:101ED000DB6F000EDC6F000EDD6F000EDE6F010E9B
:101EE000DF6FABECEBF000EF88F09451010AD8B44F
:101EF00082D4030AD8B459D5010AD8B4C9D5070A7F
:101F0000D8B456D6010AD8B416D700EF88F06F0EB1
:101F10001119D8A4D1D200019F05D8A4F2D0070E80
:101F2000D66F6000D8F3D7F0010E06EC1AF0AB0EB6
:101F3000EA6FFE0EEB6F100EEC6F32EC13F0B5D0C3
:101F4000D20ED66FFF0ED76F060ED86F000ED96F68
:101F5000020EDA6F000EDB6F000EDC6F000EDD6F1D
:101F6000000EDE6F000EDF6FE1EC0BF0D80ED66FC7
:101F7000FF0ED76F060ED86F000ED96F040EDA6F02
:101F8000000EDB6F000EDC6F000EDD6F000EDE6FEB
:101F9000000EDF6FE1EC0BF04704D8A40AD0010E6D
:101FA000D66F020ED76F000ED86F6E519CECE5F025
:101FB00016D0C70ED66FFF0ED76F050ED86F460E20
:101FC000D96F020EDA6F000EDB6F000EDC6F000EB1
:101FD000DD6F000EDE6F000EDF6FE1EC0BF0010134
:101FE0007505D8A410D06000A8F1D6F06000ACF15F
:101FF000D7F0010E0001D86F040ED96F000EDA6F12
:10200000EBECDAF059D0C60E0001D66FFF0ED76F99
:10201000060ED86F3E0ED96F040EDA6F000EDB6F1E
:10202000000EDC6F000EDD6F000EDE6F000EDF6F46
:10203000E1EC0BF041D0D20ED66FFF0ED76F060E3B
:10204000D86F000ED96F020EDA6F000EDB6F000E34
:10205000DC6F000EDD6F000EDE6F000EDF6FE1EC57
:102060000BF04704D8A40AD0010ED66F020ED76F2A
:10207000000ED86F6E519CECE5F01ED0C70ED66FE7
:10208000FF0ED76F050ED86F460ED96F020EDA6FAE
:10209000000EDB6F000EDC6F000EDD6F000EDE6FDA
:1020A000000EDF6FE1EC0BF007D09D51010AD8B4B0
:1020B000C2D7020AD8B444D70A0EC26FC30EC36F88
:1020C000440EC46F020EC56F010EC66F100EC76FAF
:1020D000060EC86F000EC96F000ECA6F000ECB6FE0
:1020E000000ECC6F000ECD6F6000D8F3CEF0C0ECC8
:1020F00006F0000E9F6F010E9E6F010E946F010E91
:10210000966F9605D8B42AD13AD1600EC26FE50E0B
:10211000C36F070EC46F020EC56F000EC66F250E8B
:10212000C76F040EC86F000EC96F000ECA6F000E95
:10213000CB6F000ECC6F000ECD6F6000D8F3CEF0E9
:10214000C0EC06F00A0EC26FC30EC36F440EC46F1C
:10215000020EC56F010EC66F100EC76F060EC86F58
:10216000000EC96F000ECA6F000ECB6F000ECC6F51
:10217000000ECD6F6000D8F3CEF0C0EC06F0600E1C
:10218000C26FE50EC36F070EC46F020EC56F5F0E00
:10219000C66F250EC76F020EC86F000EC96F000E06
:1021A000CA6F000ECB6F000ECC6F000ECD6F6000BB
:1021B000D8F3CEF0C0EC06F0DBD0600EC26FE50EB7
:1021C000C36F070EC46F020EC56F000EC66F250EDB
:1021D000C76F020EC86F000EC96F000ECA6F000EE7
:1021E000CB6F000ECC6F000ECD6F6000D8F3CEF039
:1021F000C0EC06F09D05D8B43BD00A0EC26FC30EEA
:10220000C36F440EC46F020EC56F010EC66F100E71
:10221000C76F060EC86F000EC96F000ECA6F000EA2
:10222000CB6F000ECC6F000ECD6F6000D8F3CEF0F8
:10223000C0EC06F0600EC26FE50EC36F070EC46FF0
:10224000020EC56F5F0EC66F250EC76F040EC86FF6
:10225000000EC96F000ECA6F000ECB6F000ECC6F60
:10226000000ECD6F6000D8F3CEF0C0EC06F080D049
:102270000A0EC26FC30EC36F440EC46F020EC56F49
:10228000020EC66F100EC76F060EC86F000EC96F24
:10229000000ECA6F000ECB6F000ECC6F000ECD6F1C
:1022A0006000D8F3CEF0C0EC06F062D0600EC26FD2
:1022B000E50EC36F070EC46F020EC56F000EC66F2A
:1022C000250EC76F020EC86F000EC96F000ECA6FD1
:1022D000000ECB6F000ECC6F000ECD6F6000D8F3F8
:1022E000CEF0C0EC06F0600EC26FE50EC36F070EB5
:1022F000C46F020EC56F000EC66F250EC76F040EA9
:10230000C86F000EC96F000ECA6F000ECB6F000EB3
:10231000CC6F000ECD6F6000D8F3CEF0C0EC06F0AD
:102320000A0EC26FC30EC36F440EC46F020EC56F98
:10233000020EC66F100EC76F060EC86F000EC96F73
:10234000000ECA6F000ECB6F000ECC6F000ECD6F6B
:102350006000D8F3CEF0C0EC06F00AD09451010A28
:10236000D8B4D3D6030AD8B428D7010AD8B49ED794
:1023700094C095F0000E966F000E9E6F29D001015B
:102380003E05D8A40FD0010E0001D66F020ED76F04
:10239000600094F2D8F06C519CECE5F0000E010165
:1023A0003E6F16D03D05D8A413D06000A0F1D6F042
:1023B0006000A4F1D7F0010E0001D86F040ED96FB0
:1023C000600094F2DAF0EBECDAF0000E01013D6F00
:1023D00000019E05D8A456D09C05D8A40AD0010EB1
:1023E000D66F020ED76F010ED86F6C519CECE5F0E2
:1023F00046D09B05D8A40FD06000A0F1D6F06000B5
:10240000A4F1D7F0010ED86F040ED96F010EDA6F68
:10241000EBECDAF034D04704D8A431D09D05D8A431
:1024200004D0020E9519D8B40DD001017505D8A4B9
:1024300026D0030E00019519D8A421D0030E9D19B2
:10244000D8A41DD00A0EC26FC30EC36F440EC46F52
:10245000020EC56F030EC66F100EC76F060EC86F53
:10246000000EC96F000ECA6F000ECB6F000ECC6F4E
:10247000000ECD6F6000D8F3CEF0C0EC06F0000E79
:1024800000019E6F9C05D8A40AD0410EBC6F140EAB
:10249000BD6F9851BAEC13F001013E6F12009B051D
:1024A000D8A41200410EBC6F140EBD6F9851BAEC47
:1024B00013F001013D6F1200700E1119D8A472D0F3
:1024C00000019F05D8A446D0070ED66F6000D8F350
:1024D000D7F0010E06EC1AF09B0EEA6FFE0EEB6FC2
:1024E000100EEC6F32EC13F00F0ED66FFF0ED76F9D
:1024F0000D0ED86F000ED96F020EDA6F000EDB6F73
:10250000000EDC6F000EDD6F000EDE6F000EDF6F61
:10251000E1EC0BF0B105D8A406D05A0ED66F480EE8
:10252000B9EC01F013D0020EB119D8A406D05A0E9E
:10253000D66F200EB9EC01F009D0030EB119D8A462
:1025400005D05A0ED66F200EB9EC01F0000E9F6F29
:10255000010E9E6F01013C05D8B404D000019E0518
:10256000D8A415D0600098F1D6F060009CF1D7F0A7
:102570000A0E0001D86F040ED96F600094F2DAF0F1
:1025800068ECCAF0000E9E6F000E01013C6F410E18
:102590000001BC6F140EBD6F9851BAEC13F001012D
:1025A0003C6F1200780E1119D8A4ADD300019F051D
:1025B000D8A416D0070ED66F6000D8F3D7F0010E5E
:1025C00006EC1AF0E40EEA6FFF0EEB6F060EEC6FEE
:1025D00032EC13F0000E9F6F010E9E6F010E946F90
:1025E0009605D8B47ED39E05D8A412007AD3050EE2
:1025F000E96FFE0EEA6F090EEB6F600094F2ECF0EB
:10260000020E83ECF7F0690EC26FFC0EC36F5A0E18
:10261000C46F010EC56F000EC66F000EC76F040EAB
:10262000C86F000EC96F000ECA6F000ECB6F000E90
:10263000CC6F000ECD6F6000D8F3CEF0C0EC06F08A
:102640009E0ED66FFD0ED76F0B0ED86F030ED96F8F
:10265000040EDA6F000EDB6F000EDC6F000EDD6F14
:10266000000EDE6F010EDF6FABECEBF0690EC26F98
:10267000FC0EC36F660EC46F010EC56F000EC66FF1
:10268000000EC76F050EC86F000EC96F000ECA6F2F
:10269000000ECB6F000ECC6F000ECD6F6000D8F334
:1026A000CEF0C0EC06F0FC0ED66FFD0ED76F090E13
:1026B000D86F030ED96F050EDA6F000EDB6F000EB8
:1026C000DC6F000EDD6F000EDE6F010EDF6FABEC16
:1026D000EBF0690EC26FFC0EC36F660EC46F010E85
:1026E000C56F000EC66F000EC76F060EC86F000ED6
:1026F000C96F000ECA6F000ECB6F000ECC6F000EBC
:10270000CD6F6000D8F3CEF0C0EC06F0E80ED66FC7
:10271000FD0ED76F0A0ED86F030ED96F060EDA6F53
:10272000000EDB6F000EDC6F000EDD6F000EDE6F43
:10273000010EDF6FABECEBF0690EC26FFC0EC36FE6
:10274000660EC46F010EC56F000EC66F000EC76F18
:10275000070EC86F000EC96F000ECA6F000ECB6F58
:10276000000ECC6F000ECD6F6000D8F3CEF0C0EC41
:1027700006F02D0ED66FFE0ED76F060ED86F030E25
:10278000D96F070EDA6F000EDB6F000EDC6F000EE4
:10279000DD6F000EDE6F010EDF6FABECEBF000EFD4
:1027A00088F09E0EE96FFD0EEA6F0B0EEB6F600076
:1027B00094F2ECF0030E83ECF7F0690EC26FFC0E9E
:1027C000C36F5A0EC46F010EC56F000EC66F000EA8
:1027D000C76F020EC86F000EC96F000ECA6F000EE1
:1027E000CB6F000ECC6F000ECD6F6000D8F3CEF033
:1027F000C0EC06F0050ED66FFE0ED76F090ED86F2F
:10280000030ED96F020EDA6F000EDB6F000EDC6F65
:10281000000EDD6F000EDE6F010EDF6FABECEBF034
:10282000690EC26FFC0EC36F5A0EC46F010EC56FE6
:10283000000EC66F000EC76F050EC86F000EC96F81
:10284000000ECA6F000ECB6F000ECC6F000ECD6F66
:102850006000D8F3CEF0C0EC06F0FC0ED66FFD0E93
:10286000D76F090ED86F030ED96F050EDA6F000E01
:10287000DB6F000EDC6F000EDD6F000EDE6F010EF1
:10288000DF6FABECEBF025D7FC0EE96FFD0EEA6FC6
:10289000090EEB6F600094F2ECF0040E83ECF7F09D
:1028A000690EC26FFC0EC36F5A0EC46F010EC56F66
:1028B000000EC66F000EC76F020EC86F000EC96F04
:1028C000000ECA6F000ECB6F000ECC6F000ECD6FE6
:1028D0006000D8F3CEF0C0EC06F0050ED66FFE0E09
:1028E000D76F090ED86F030ED96F020EDA6F000E84
:1028F000DB6F000EDC6F000EDD6F000EDE6F010E71
:10290000DF6FABECEBF0690EC26FFC0EC36F5A0EBB
:10291000C46F010EC56F000EC66F000EC76F030EA9
:10292000C86F000EC96F000ECA6F000ECB6F000E8D
:10293000CC6F000ECD6F6000D8F3CEF0C0EC06F087
:102940009E0ED66FFD0ED76F0B0ED86F030ED96F8C
:10295000030EDA6F000EDB6F000EDC6F000EDD6F12
:10296000000EDE6F010EDF6FABECEBF0690EC26F95
:10297000FC0EC36F5A0EC46F010EC56F000EC66FFA
:10298000000EC76F060EC86F000EC96F000ECA6F2B
:10299000000ECB6F000ECC6F000ECD6F6000D8F331
:1029A000CEF0C0EC06F0B2D6E80EE96FFD0EEA6F8D
:1029B0000A0EEB6F600094F2ECF0050E83ECF7F07A
:1029C000690EC26FFC0EC36F5A0EC46F010EC56F45
:1029D000000EC66F000EC76F020EC86F000EC96FE3
:1029E000000ECA6F000ECB6F000ECC6F000ECD6FC5
:1029F0006000D8F3CEF0C0EC06F0050ED66FFE0EE8
:102A0000D76F090ED86F030ED96F020EDA6F000E62
:102A1000DB6F000EDC6F000EDD6F000EDE6F010E4F
:102A2000DF6FABECEBF0690EC26FFC0EC36F5A0E9A
:102A3000C46F010EC56F000EC66F000EC76F030E88
:102A4000C86F000EC96F000ECA6F000ECB6F000E6C
:102A5000CC6F000ECD6F6000D8F3CEF0C0EC06F066
:102A60009E0ED66FFD0ED76F0B0ED86F030ED96F6B
:102A7000030EDA6F000EDB6F000EDC6F000EDD6FF1
:102A8000000EDE6F010EDF6FABECEBF0690EC26F74
:102A9000FC0EC36F5A0EC46F010EC56F000EC66FD9
:102AA000000EC76F040EC86F000EC96F000ECA6F0C
:102AB000000ECB6F000ECC6F000ECD6F6000D8F310
:102AC000CEF0C0EC06F0FC0ED66FFD0ED76F090EEF
:102AD000D86F030ED96F040EDA6F000EDB6F000E95
:102AE000DC6F000EDD6F000EDE6F010EDF6FABECF2
:102AF000EBF0690EC26FFC0EC36F5A0EC46F010E6D
:102B0000C56F000EC66F000EC76F070EC86F000EB0
:102B1000C96F000ECA6F000ECB6F000ECC6F000E97
:102B2000CD6F6000D8F3CEF0C0EC06F022D62D0EAB
:102B3000E96FFE0EEA6F060EEB6F600094F2ECF0A8
:102B4000060E83ECF7F0690EC26FFC0EC36F5A0ECF
:102B5000C46F010EC56F000EC66F000EC76F020E68
:102B6000C86F000EC96F000ECA6F000ECB6F000E4B
:102B7000CC6F000ECD6F6000D8F3CEF0C0EC06F045
:102B8000050ED66FFE0ED76F090ED86F030ED96FE4
:102B9000020EDA6F000EDB6F000EDC6F000EDD6FD1
:102BA000000EDE6F010EDF6FABECEBF0690EC26F53
:102BB000FC0EC36F5A0EC46F010EC56F000EC66FB8
:102BC000000EC76F030EC86F000EC96F000ECA6FEC
:102BD000000ECB6F000ECC6F000ECD6F6000D8F3EF
:102BE000CEF0C0EC06F09E0ED66FFD0ED76F0B0E2A
:102BF000D86F030ED96F030EDA6F000EDB6F000E75
:102C0000DC6F000EDD6F000EDE6F010EDF6FABECD0
:102C1000EBF0690EC26FFC0EC36F5A0EC46F010E4B
:102C2000C56F000EC66F000EC76F040EC86F000E92
:102C3000C96F000ECA6F000ECB6F000ECC6F000E76
:102C4000CD6F6000D8F3CEF0C0EC06F0FC0ED66F6E
:102C5000FD0ED76F090ED86F030ED96F040EDA6F11
:102C6000000EDB6F000EDC6F000EDD6F000EDE6FFE
:102C7000010EDF6FABECEBF0690EC26FFC0EC36FA1
:102C80005A0EC46F010EC56F000EC66F000EC76FDF
:102C9000050EC86F000EC96F000ECA6F000ECB6F15
:102CA000000ECC6F000ECD6F6000D8F3CEF0C0ECFC
:102CB00006F0E80ED66FFD0ED76F0A0ED86F030E22
:102CC000D96F050EDA6F000EDB6F000EDC6F000EA1
:102CD000DD6F000EDE6F010EDF6FABECEBF000EF8F
:102CE00088F09451010AD8B482D4030AD8B459D5D3
:102CF000010AD8B4C9D5070AD8B456D6010AD8B43F
:102D000016D700EF88F0790E1119D8A45BD0000116
:102D10009F05D8A430D0070ED66F6000D8F3D7F047
:102D2000010E06EC1AF09A0EEA6FFF0EEB6F090E19
:102D3000EC6F32EC13F0000E9F6F000E986FF80EE0
:102D40009225D66FD76BFF0ED7232E0ED86F020EAB
:102D5000D96F000EDA6F000EDB6F000EDC6FD7EC60
:102D6000CDF0050ED66F9251F80FD76F070E3EECDF
:102D700011F0080F926F01016905D8A41200F80E36
:102D80006A250001D66FD76BFF0ED7232E0ED86FA2
:102D9000020ED96F000EDA6F000EDB6F000EDC6FD3
:102DA000D7ECCDF0050ED66F01016A51F80F000186
:102DB000D76F070E3EEC11F0080F926F000E010165
:102DC000696F12007A0E1119D8A46CEF9CF0000103
:102DD0009F05D8A416D0070ED66F6000D8F3D7F0A1
:102DE000010E06EC1AF0CA0EEA6FFE0EEB6F0F0E24
:102DF000EC6F32EC13F0000E9F6F010E946F010E1A
:102E0000966F9605D8B445EF9BF054EF9BF0B00554
:102E1000D8A458D00A0EC26FC30EC36F440EC46F3D
:102E2000020EC56F110EC66F080EC76F020EC86F77
:102E3000000EC96F000ECA6F000ECB6F000ECC6F74
:102E4000000ECD6F6000D8F3CEF0C0EC06F00A0E95
:102E5000C26FC30EC36F440EC46F020EC56F160E51
:102E6000C66F080EC76F040EC86F000EC96F000E44
:102E7000CA6F000ECB6F000ECC6F000ECD6F6000DE
:102E8000D8F3CEF0C0EC06F00A0EC26FC30EC36FCB
:102E9000440EC46F020EC56F120EC66F080EC76FC8
:102EA000060EC86F000EC96F000ECA6F000ECB6F02
:102EB000000ECC6F000ECD6F6000D8F3CEF0C0ECEA
:102EC00006F0B7D0020EB019D8A458D00A0EC26FBF
:102ED000C30EC36F440EC46F020EC56F0F0EC66FD4
:102EE000080EC76F020EC86F000EC96F000ECA6FC2
:102EF000000ECB6F000ECC6F000ECD6F6000D8F3CC
:102F0000CEF0C0EC06F00A0EC26FC30EC36F440EC3
:102F1000C46F020EC56F180EC66F080EC76F040E81
:102F2000C86F000EC96F000ECA6F000ECB6F000E87
:102F3000CC6F000ECD6F6000D8F3CEF0C0EC06F081
:102F40000A0EC26FC30EC36F440EC46F020EC56F6C
:102F5000120EC66F080EC76F060EC86F000EC96F3F
:102F6000000ECA6F000ECB6F000ECC6F000ECD6F3F
:102F70006000D8F3CEF0C0EC06F05BD0030EB019C1
:102F8000D8A457D00A0EC26FC30EC36F440EC46FCD
:102F9000020EC56F0F0EC66F080EC76F020EC86F08
:102FA000000EC96F000ECA6F000ECB6F000ECC6F03
:102FB000000ECD6F6000D8F3CEF0C0EC06F00A0E24
:102FC000C26FC30EC36F440EC46F020EC56F160EE0
:102FD000C66F080EC76F040EC86F000EC96F000ED3
:102FE000CA6F000ECB6F000ECC6F000ECD6F60006D
:102FF000D8F3CEF0C0EC06F00A0EC26FC30EC36F5A
:10300000440EC46F020EC56F140EC66F080EC76F54
:10301000060EC86F000EC96F000ECA6F000ECB6F90
:10302000000ECC6F000ECD6F6000D8F3CEF0C0EC78
:1030300006F0600EC26FE50EC36F070EC46F020E7E
:10304000C56F000EC66F500EC76F040EC86F000E1E
:10305000C96F000ECA6F000ECB6F000ECC6F000E52
:10306000CD6F6000D8F3CEF0C0EC06F0600EC26FFA
:10307000E50EC36F070EC46F020EC56F000EC66F5C
:10308000500EC76F060EC86F000EC96F000ECA6FD4
:10309000000ECB6F000ECC6F000ECD6F6000D8F32A
:1030A000CEF0C0EC06F0600EC26FE50EC36F070EE7
:1030B000C46F020EC56F6B0EC66F500EC76F020E47
:1030C000C86F000EC96F000ECA6F000ECB6F000EE6
:1030D000CC6F000ECD6F6000D8F3CEF0C0EC06F0E0
:1030E000DFD2020EB019D8A458D00A0EC26FC30E98
:1030F000C36F440EC46F020EC56F0E0EC66F080E6E
:10310000C76F020EC86F000EC96F000ECA6F000EA7
:10311000CB6F000ECC6F000ECD6F6000D8F3CEF0F9
:10312000C0EC06F00A0EC26FC30EC36F440EC46F2C
:10313000020EC56F190EC66F080EC76F040EC86F5A
:10314000000EC96F000ECA6F000ECB6F000ECC6F61
:10315000000ECD6F6000D8F3CEF0C0EC06F00A0E82
:10316000C26FC30EC36F440EC46F020EC56F120E42
:10317000C66F080EC76F060EC86F000EC96F000E2F
:10318000CA6F000ECB6F000ECC6F000ECD6F6000CB
:10319000D8F3CEF0C0EC06F0B6D0B005D8A458D025
:1031A0000A0EC26FC30EC36F440EC46F020EC56F0A
:1031B000100EC66F080EC76F020EC86F000EC96FE3
:1031C000000ECA6F000ECB6F000ECC6F000ECD6FDD
:1031D0006000D8F3CEF0C0EC06F00A0EC26FC30E4A
:1031E000C36F440EC46F020EC56F170EC66F080E74
:1031F000C76F040EC86F000EC96F000ECA6F000EB5
:10320000CB6F000ECC6F000ECD6F6000D8F3CEF008
:10321000C0EC06F00A0EC26FC30EC36F440EC46F3B
:10322000020EC56F120EC66F080EC76F060EC86F6E
:10323000000EC96F000ECA6F000ECB6F000ECC6F70
:10324000000ECD6F6000D8F3CEF0C0EC06F05BD07E
:10325000030EB019D8A457D00A0EC26FC30EC36FA5
:10326000440EC46F020EC56F0E0EC66F080EC76FF8
:10327000020EC86F000EC96F000ECA6F000ECB6F32
:10328000000ECC6F000ECD6F6000D8F3CEF0C0EC16
:1032900006F00A0EC26FC30EC36F440EC46F020E57
:1032A000C56F170EC66F080EC76F040EC86F000EED
:1032B000C96F000ECA6F000ECB6F000ECC6F000EF0
:1032C000CD6F6000D8F3CEF0C0EC06F00A0EC26FEE
:1032D000C30EC36F440EC46F020EC56F140EC66FCB
:1032E000080EC76F060EC86F000EC96F000ECA6FBA
:1032F000000ECB6F000ECC6F000ECD6F6000D8F3C8
:10330000CEF0C0EC06F0600EC26FE50EC36F070E84
:10331000C46F020EC56F000EC66F500EC76F020E4F
:10332000C86F000EC96F000ECA6F000ECB6F000E83
:10333000CC6F000ECD6F6000D8F3CEF0C0EC06F07D
:10334000600EC26FE50EC36F070EC46F020EC56F2D
:10335000000EC66F500EC76F060EC86F000EC96F05
:10336000000ECA6F000ECB6F000ECC6F000ECD6F3B
:103370006000D8F3CEF0C0EC06F0600EC26FE50E30
:10338000C36F070EC46F020EC56F6B0EC66F500E73
:10339000C76F040EC86F000EC96F000ECA6F000E13
:1033A000CB6F000ECC6F000ECD6F6000D8F3CEF067
:1033B000C0EC06F075D1030EB019D8A458D00A0E8F
:1033C000C26FC30EC36F440EC46F020EC56F0E0EE4
:1033D000C66F080EC76F020EC86F000EC96F000ED1
:1033E000CA6F000ECB6F000ECC6F000ECD6F600069
:1033F000D8F3CEF0C0EC06F00A0EC26FC30EC36F56
:10340000440EC46F020EC56F160EC66F080EC76F4E
:10341000040EC86F000EC96F000ECA6F000ECB6F8E
:10342000000ECC6F000ECD6F6000D8F3CEF0C0EC74
:1034300006F00A0EC26FC30EC36F440EC46F020EB5
:10344000C56F150EC66F080EC76F060EC86F000E4B
:10345000C96F000ECA6F000ECB6F000ECC6F000E4E
:10346000CD6F6000D8F3CEF0C0EC06F0B6D0B0055A
:10347000D8A458D00A0EC26FC30EC36F440EC46FD7
:10348000020EC56F100EC66F080EC76F020EC86F12
:10349000000EC96F000ECA6F000ECB6F000ECC6F0E
:1034A000000ECD6F6000D8F3CEF0C0EC06F00A0E2F
:1034B000C26FC30EC36F440EC46F020EC56F160EEB
:1034C000C66F080EC76F040EC86F000EC96F000EDE
:1034D000CA6F000ECB6F000ECC6F000ECD6F600078
:1034E000D8F3CEF0C0EC06F00A0EC26FC30EC36F65
:1034F000440EC46F020EC56F130EC66F080EC76F61
:10350000060EC86F000EC96F000ECA6F000ECB6F9B
:10351000000ECC6F000ECD6F6000D8F3CEF0C0EC83
:1035200006F05BD0020EB019D8A457D00A0EC26FB5
:10353000C30EC36F440EC46F020EC56F0E0EC66F6E
:10354000080EC76F020EC86F000EC96F000ECA6F5B
:10355000000ECB6F000ECC6F000ECD6F6000D8F365
:10356000CEF0C0EC06F00A0EC26FC30EC36F440E5D
:10357000C46F020EC56F180EC66F080EC76F040E1B
:10358000C86F000EC96F000ECA6F000ECB6F000E21
:10359000CC6F000ECD6F6000D8F3CEF0C0EC06F01B
:1035A0000A0EC26FC30EC36F440EC46F020EC56F06
:1035B000130EC66F080EC76F060EC86F000EC96FD8
:1035C000000ECA6F000ECB6F000ECC6F000ECD6FD9
:1035D0006000D8F3CEF0C0EC06F0600EC26FE50ECE
:1035E000C36F070EC46F020EC56F000EC66F500E7C
:1035F000C76F020EC86F000EC96F000ECA6F000EB3
:10360000CB6F000ECC6F000ECD6F6000D8F3CEF004
:10361000C0EC06F0600EC26FE50EC36F070EC46FFC
:10362000020EC56F000EC66F500EC76F040EC86F36
:10363000000EC96F000ECA6F000ECB6F000ECC6F6C
:10364000000ECD6F6000D8F3CEF0C0EC06F0600E37
:10365000C26FE50EC36F070EC46F020EC56F6B0E0F
:10366000C66F500EC76F060EC86F000EC96F000EF2
:10367000CA6F000ECB6F000ECC6F000ECD6F6000D6
:10368000D8F3CEF0C0EC06F00BD09451010AD8B4B8
:1036900007EF97F0030AD8B424D5010AD8B48BD623
:1036A00094C095F0000E966F9E05D8A41200950563
:1036B000D8A458D00A0EC26FC30EC36F440EC46F95
:1036C000020EC56F110EC66F080EC76F020EC86FCF
:1036D000000EC96F000ECA6F000ECB6F000ECC6FCC
:1036E000000ECD6F6000D8F3CEF0C0EC06F00A0EED
:1036F000C26FC30EC36F440EC46F020EC56F160EA9
:10370000C66F080EC76F040EC86F000EC96F000E9B
:10371000CA6F000ECB6F000ECC6F000ECD6F600035
:10372000D8F3CEF0C0EC06F00A0EC26FC30EC36F22
:10373000440EC46F020EC56F120EC66F080EC76F1F
:10374000060EC86F000EC96F000ECA6F000ECB6F59
:10375000000ECC6F000ECD6F6000D8F3CEF0C0EC41
:1037600006F0B7D0020E9519D8A458D00A0EC26F31
:10377000C30EC36F440EC46F020EC56F0E0EC66F2C
:10378000080EC76F020EC86F000EC96F000ECA6F19
:10379000000ECB6F000ECC6F000ECD6F6000D8F323
:1037A000CEF0C0EC06F00A0EC26FC30EC36F440E1B
:1037B000C46F020EC56F190EC66F080EC76F040ED8
:1037C000C86F000EC96F000ECA6F000ECB6F000EDF
:1037D000CC6F000ECD6F6000D8F3CEF0C0EC06F0D9
:1037E0000A0EC26FC30EC36F440EC46F020EC56FC4
:1037F000120EC66F080EC76F060EC86F000EC96F97
:10380000000ECA6F000ECB6F000ECC6F000ECD6F96
:103810006000D8F3CEF0C0EC06F05BD0030E951933
:10382000D8A457D00A0EC26FC30EC36F440EC46F24
:10383000020EC56F0E0EC66F080EC76F020EC86F60
:10384000000EC96F000ECA6F000ECB6F000ECC6F5A
:10385000000ECD6F6000D8F3CEF0C0EC06F00A0E7B
:10386000C26FC30EC36F440EC46F020EC56F160E37
:10387000C66F080EC76F040EC86F000EC96F000E2A
:10388000CA6F000ECB6F000ECC6F000ECD6F6000C4
:10389000D8F3CEF0C0EC06F00A0EC26FC30EC36FB1
:1038A000440EC46F020EC56F150EC66F080EC76FAB
:1038B000060EC86F000EC96F000ECA6F000ECB6FE8
:1038C000000ECC6F000ECD6F6000D8F3CEF0C0ECD0
:1038D00006F0000E9E6F12007B0E1119D8A41BD0AB
:1038E00000019F05D8A41200070ED66F6000D8F320
:1038F000D7F0010E06EC1AF0910EEA6FFF0EEB6F97
:10390000090EEC6F32EC13F0000E9F6F010E9E6FEC
:10391000010E946F12007C0E1119D8A411D1000170
:103920009F05D8A442D0070ED66F6000D8F3D7F019
:10393000010E06EC1AF06A0EEA6FFF0EEB6F0A0E2C
:10394000EC6F32EC13F0460ED66FFE0ED76F130EEF
:10395000D86F000ED96F020EDA6F000EDB6F000E0B
:10396000DC6F000EDD6F000EDE6F010EDF6FABEC63
:10397000EBF0590ED66FFE0ED76F110ED86F000EFA
:10398000D96F030EDA6F000EDB6F000EDC6F000ED6
:10399000DD6F000EDE6F010EDF6FABECEBF0000EA3
:1039A0009F6F020E946F010E966F9605D8B4BFD02C
:1039B0009E05D8A41200BBD09E05D8A41ED00A0E26
:1039C000C26FC30EC36F440EC46F020EC56F090EE3
:1039D000C66F100EC76F040EC86F000EC96F000EC1
:1039E000CA6F000ECB6F000ECC6F000ECD6F600063
:1039F000D8F3CEF0C0EC06F01DD00A0EC26FC30E95
:103A0000C36F440EC46F020EC56F080EC66F100E52
:103A1000C76F040EC86F000EC96F000ECA6F000E8C
:103A2000CB6F000ECC6F000ECD6F6000D8F3CEF0E0
:103A3000C0EC06F00A0EC26FC30EC36F440EC46F13
:103A4000020EC56F1D0EC66F100EC76F060EC86F33
:103A5000000EC96F000ECA6F000ECB6F000ECC6F48
:103A6000000ECD6F6000D8F3CEF0C0EC06F000EF92
:103A700088F00A0EC26FC30EC36F440EC46F020EED
:103A8000C56F070EC66F100EC76F040EC86F000E0D
:103A9000C96F000ECA6F000ECB6F000ECC6F000E08
:103AA000CD6F6000D8F3CEF0C0EC06F09E05D8A430
:103AB0001FD00A0EC26FC30EC36F440EC46F020E36
:103AC000C56F1F0EC66F100EC76F060EC86F000EB3
:103AD000C96F000ECA6F000ECB6F000ECC6F000EC8
:103AE000CD6F6000D8F3CEF0C0EC06F000EF88F0A8
:103AF0000A0EC26FC30EC36F440EC46F020EC56FB1
:103B00001E0EC66F100EC76F060EC86F000EC96F6F
:103B1000000ECA6F000ECB6F000ECC6F000ECD6F83
:103B20006000D8F3CEF0C0EC06F000EF88F09451BE
:103B3000010AD8B441D7030AD8B49BD700EF88F064
:103B4000810E1119D8A46DD000019F05D8A41200D0
:103B5000070ED66F6000D8F3D7F0010E06EC1AF00E
:103B6000F00EEA6FFF0EEB6F060EEC6F32EC13F007
:103B70007B0ED66FFE0ED76F100ED86F060ED96F64
:103B8000030EDA6F000EDB6F000EDC6F000EDD6FD0
:103B9000000EDE6F000EDF6FABECEBF0BB0ED66FEE
:103BA000FE0ED76F0F0ED86F0A0ED96F040EDA6FA4
:103BB000000EDB6F000EDC6F000EDD6F000EDE6F9F
:103BC000000EDF6FABECEBF0DE0ED66FFF0ED76FA3
:103BD000060ED86F240ED96F050EDA6F000EDB6F5C
:103BE000000EDC6F000EDD6F000EDE6F000EDF6F6B
:103BF000ABECEBF08B0ED66FFE0ED76F100ED86FBE
:103C0000080ED96F060EDA6F000EDB6F000EDC6F48
:103C1000000EDD6F000EDE6F000EDF6FABECEBF021
:103C200073D6820E1119D8A4ADD300019F05D8A474
:103C300016D0070ED66F6000D8F3D7F0010E06EC51
:103C40001AF0540EEA6FFF0EEB6F0B0EEC6F32ECB6
:103C500013F0000E9F6F010E9E6F010E946F96057C
:103C6000D8B47ED39E05D8A412007AD3A90EE96FEA
:103C7000FD0EEA6F0B0EEB6F600094F2ECF0020E9B
:103C800083ECF7F0690EC26FFC0EC36F5A0EC46F5F
:103C9000010EC56F000EC66F000EC76F040EC86F11
:103CA000000EC96F000ECA6F000ECB6F000ECC6FF6
:103CB000000ECD6F6000D8F3CEF0C0EC06F0F20E2F
:103CC000D66FFD0ED76F0A0ED86F030ED96F040E94
:103CD000DA6F000EDB6F000EDC6F000EDD6F000E82
:103CE000DE6F010EDF6FABECEBF0690EC26FFC0E06
:103CF000C36F660EC46F010EC56F000EC66F000E57
:103D0000C76F050EC86F000EC96F000ECA6F000E98
:103D1000CB6F000ECC6F000ECD6F6000D8F3CEF0ED
:103D2000C0EC06F0400ED66FFE0ED76F020ED86FB5
:103D3000030ED96F050EDA6F000EDB6F000EDC6F1D
:103D4000000EDD6F000EDE6F010EDF6FABECEBF0EF
:103D5000690EC26FFC0EC36F660EC46F010EC56F95
:103D6000000EC66F000EC76F060EC86F000EC96F3B
:103D7000000ECA6F000ECB6F000ECC6F000ECD6F21
:103D80006000D8F3CEF0C0EC06F03E0ED66FFE0E0B
:103D9000D76F020ED86F030ED96F060EDA6F000EC2
:103DA000DB6F000EDC6F000EDD6F000EDE6F010EAC
:103DB000DF6FABECEBF0690EC26FFC0EC36F660EEB
:103DC000C46F010EC56F000EC66F000EC76F070EE1
:103DD000C86F000EC96F000ECA6F000ECB6F000EC9
:103DE000CC6F000ECD6F6000D8F3CEF0C0EC06F0C3
:103DF0003C0ED66FFE0ED76F020ED86F030ED96F32
:103E0000070EDA6F000EDB6F000EDC6F000EDD6F49
:103E1000000EDE6F010EDF6FABECEBF000EF88F011
:103E2000F20EE96FFD0EEA6F0A0EEB6F600094F27E
:103E3000ECF0030E83ECF7F0690EC26FFC0EC36F5B
:103E40005A0EC46F010EC56F000EC66F000EC76F0D
:103E5000020EC86F000EC96F000ECA6F000ECB6F46
:103E6000000ECC6F000ECD6F6000D8F3CEF0C0EC2A
:103E700006F0A90ED66FFD0ED76F0B0ED86F030E8E
:103E8000D96F020EDA6F000EDB6F000EDC6F000ED2
:103E9000DD6F000EDE6F010EDF6FABECEBF0690E35
:103EA000C26FFC0EC36F5A0EC46F010EC56F000EB9
:103EB000C66F000EC76F050EC86F000EC96F000EEB
:103EC000CA6F000ECB6F000ECC6F000ECD6F60007E
:103ED000D8F3CEF0C0EC06F0400ED66FFE0ED76FD2
:103EE000020ED86F030ED96F050EDA6F000EDB6F6E
:103EF000000EDC6F000EDD6F000EDE6F010EDF6F57
:103F0000ABECEBF025D7400EE96FFE0EEA6F020E28
:103F1000EB6F600094F2ECF0040E83ECF7F0690EA6
:103F2000C26FFC0EC36F5A0EC46F010EC56F000E38
:103F3000C66F000EC76F020EC86F000EC96F000E6D
:103F4000CA6F000ECB6F000ECC6F000ECD6F6000FD
:103F5000D8F3CEF0C0EC06F0A90ED66FFD0ED76FE9
:103F60000B0ED86F030ED96F020EDA6F000EDB6FE7
:103F7000000EDC6F000EDD6F000EDE6F010EDF6FD6
:103F8000ABECEBF0690EC26FFC0EC36F5A0EC46F40
:103F9000010EC56F000EC66F000EC76F030EC86F0F
:103FA000000EC96F000ECA6F000ECB6F000ECC6FF3
:103FB000000ECD6F6000D8F3CEF0C0EC06F0F20E2C
:103FC000D66FFD0ED76F0A0ED86F030ED96F030E92
:103FD000DA6F000EDB6F000EDC6F000EDD6F000E7F
:103FE000DE6F010EDF6FABECEBF0690EC26FFC0E03
:103FF000C36F5A0EC46F010EC56F000EC66F000E60
:10400000C76F060EC86F000EC96F000ECA6F000E94
:10401000CB6F000ECC6F000ECD6F6000D8F3CEF0EA
:10402000C0EC06F0B2D63E0EE96FFE0EEA6F020E4D
:10403000EB6F600094F2ECF0050E83ECF7F0690E84
:10404000C26FFC0EC36F5A0EC46F010EC56F000E17
:10405000C66F000EC76F020EC86F000EC96F000E4C
:10406000CA6F000ECB6F000ECC6F000ECD6F6000DC
:10407000D8F3CEF0C0EC06F0A90ED66FFD0ED76FC8
:104080000B0ED86F030ED96F020EDA6F000EDB6FC6
:10409000000EDC6F000EDD6F000EDE6F010EDF6FB5
:1040A000ABECEBF0690EC26FFC0EC36F5A0EC46F1F
:1040B000010EC56F000EC66F000EC76F030EC86FEE
:1040C000000EC96F000ECA6F000ECB6F000ECC6FD2
:1040D000000ECD6F6000D8F3CEF0C0EC06F0F20E0B
:1040E000D66FFD0ED76F0A0ED86F030ED96F030E71
:1040F000DA6F000EDB6F000EDC6F000EDD6F000E5E
:10410000DE6F010EDF6FABECEBF0690EC26FFC0EE1
:10411000C36F5A0EC46F010EC56F000EC66F000E3E
:10412000C76F040EC86F000EC96F000ECA6F000E75
:10413000CB6F000ECC6F000ECD6F6000D8F3CEF0C9
:10414000C0EC06F0400ED66FFE0ED76F020ED86F91
:10415000030ED96F040EDA6F000EDB6F000EDC6FFA
:10416000000EDD6F000EDE6F010EDF6FABECEBF0CB
:10417000690EC26FFC0EC36F5A0EC46F010EC56F7D
:10418000000EC66F000EC76F070EC86F000EC96F16
:10419000000ECA6F000ECB6F000ECC6F000ECD6FFD
:1041A0006000D8F3CEF0C0EC06F022D63C0EE96FEA
:1041B000FE0EEA6F020EEB6F600094F2ECF0060E5A
:1041C00083ECF7F0690EC26FFC0EC36F5A0EC46F1A
:1041D000010EC56F000EC66F000EC76F020EC86FCE
:1041E000000EC96F000ECA6F000ECB6F000ECC6FB1
:1041F000000ECD6F6000D8F3CEF0C0EC06F0A90E33
:10420000D66FFD0ED76F0B0ED86F030ED96F020E4F
:10421000DA6F000EDB6F000EDC6F000EDD6F000E3C
:10422000DE6F010EDF6FABECEBF0690EC26FFC0EC0
:10423000C36F5A0EC46F010EC56F000EC66F000E1D
:10424000C76F030EC86F000EC96F000ECA6F000E55
:10425000CB6F000ECC6F000ECD6F6000D8F3CEF0A8
:10426000C0EC06F0F20ED66FFD0ED76F0A0ED86FB7
:10427000030ED96F030EDA6F000EDB6F000EDC6FDA
:10428000000EDD6F000EDE6F010EDF6FABECEBF0AA
:10429000690EC26FFC0EC36F5A0EC46F010EC56F5C
:1042A000000EC66F000EC76F040EC86F000EC96FF8
:1042B000000ECA6F000ECB6F000ECC6F000ECD6FDC
:1042C0006000D8F3CEF0C0EC06F0400ED66FFE0EC4
:1042D000D76F020ED86F030ED96F040EDA6F000E7F
:1042E000DB6F000EDC6F000EDD6F000EDE6F010E67
:1042F000DF6FABECEBF0690EC26FFC0EC36F5A0EB2
:10430000C46F010EC56F000EC66F000EC76F050E9D
:10431000C86F000EC96F000ECA6F000ECB6F000E83
:10432000CC6F000ECD6F6000D8F3CEF0C0EC06F07D
:104330003E0ED66FFE0ED76F020ED86F030ED96FEA
:10434000050EDA6F000EDB6F000EDC6F000EDD6F06
:10435000000EDE6F010EDF6FABECEBF000EF88F0CC
:104360009451010AD8B482D4030AD8B459D5010AA9
:10437000D8B4C9D5070AD8B456D6010AD8B416D7C6
:1043800000EF88F0830E1119D8A4D3D300019F0544
:10439000D8A43DD0070ED66F6000D8F3D7F0010E39
:1043A00006EC1AF0330EEA6FFF0EEB6F0B0EEC6F9C
:1043B00032EC13F0F60ED66FFF0ED76F050ED86FE6
:1043C000000ED96F020EDA6F000EDB6F000EDC6F8D
:1043D000000EDD6F000EDE6F000EDF6FE1EC0BF004
:1043E0009A05D8A404D0000E916F030E03D0010EDD
:1043F000916F010E946F000E9F6F35503610D8A448
:1044000004D0000E366E010E356E010E966F9605C5
:10441000D8B482D292D2600EC26FE50EC36F070E7F
:10442000C46F020EC56F000EC66F450EC76F040E37
:10443000C86F000EC96F000ECA6F000ECB6F000E62
:10444000CC6F000ECD6F6000D8F3CEF0C0EC06F05C
:10445000600EC26FE50EC36F070EC46F020EC56F0C
:104460006B0EC66F450EC76F020EC86F000EC96F88
:10447000000ECA6F000ECB6F000ECC6F000ECD6F1A
:104480006000D8F3CEF0C0EC06F06000C8F1D6F0C2
:104490006000CCF1D7F01E0ED86F020ED96F000E5F
:1044A000DA6F000EDB6F000EDC6FD7ECCDF0B7518A
:1044B000D8A41ED00A0EC26FC30EC36F440EC46FC1
:1044C000020EC56F0A0EC66F000EC76F040EC86FCE
:1044D000000EC96F000ECA6F000ECB6F000ECC6FBE
:1044E000000ECD6F6000D8F3CEF0C0EC06F01DD00A
:1044F0000A0EC26FC30EC36F440EC46F020EC56FA7
:104500000C0EC66F000EC76F040EC86F000EC96F89
:10451000000ECA6F000ECB6F000ECC6F000ECD6F79
:104520006000D8F3CEF0C0EC06F09105D8A41ED000
:104530000A0EC26FC30EC36F440EC46F020EC56F66
:10454000040EC66F000EC76F060EC86F000EC96F4F
:10455000000ECA6F000ECB6F000ECC6F000ECD6F39
:104560006000D8F3CEF0C0EC06F01DD00A0EC26F8A
:10457000C30EC36F440EC46F020EC56F1A0EC66F12
:10458000000EC76F060EC86F000EC96F000ECA6F0F
:10459000000ECB6F000ECC6F000ECD6F6000D8F315
:1045A000CEF0C0EC06F0B105D8A406D05A0ED66FF6
:1045B000200EB9EC01F0BAD1020EB119D8A406D080
:1045C0005A0ED66F200EB9EC01F0B0D1030EB1191E
:1045D000D8A4ACD15A0ED66F200EB9EC01F0A6D1FA
:1045E000600EC26FE50EC36F070EC46F020EC56F7B
:1045F000000EC66F450EC76F020EC86F000EC96F62
:10460000000ECA6F000ECB6F000ECC6F000ECD6F88
:104610006000D8F3CEF0C0EC06F0600EC26FE50E7D
:10462000C36F070EC46F020EC56F6B0EC66F450ECB
:10463000C76F040EC86F000EC96F000ECA6F000E60
:10464000CB6F000ECC6F000ECD6F6000D8F3CEF0B4
:10465000C0EC06F06000C8F1D6F06000CCF1D7F0F5
:104660001E0ED86F020ED96F000EDA6F000EDB6FD0
:10467000000EDC6FD7ECCDF0B751D8A41ED00A0ED7
:10468000C26FC30EC36F440EC46F020EC56F0B0E14
:10469000C66F000EC76F040EC86F000EC96F000E04
:1046A000CA6F000ECB6F000ECC6F000ECD6F600096
:1046B000D8F3CEF0C0EC06F01DD00A0EC26FC30EC8
:1046C000C36F440EC46F020EC56F0D0EC66F000E91
:1046D000C76F040EC86F000EC96F000ECA6F000EC0
:1046E000CB6F000ECC6F000ECD6F6000D8F3CEF014
:1046F000C0EC06F09105D8A41ED00A0EC26FC30EFE
:10470000C36F440EC46F020EC56F040EC66F000E59
:10471000C76F060EC86F000EC96F000ECA6F000E7D
:10472000CB6F000ECC6F000ECD6F6000D8F3CEF0D3
:10473000C0EC06F01DD00A0EC26FC30EC36F440E4C
:10474000C46F020EC56F1A0EC66F000EC76F060E3D
:10475000C86F000EC96F000ECA6F000ECB6F000E3F
:10476000CC6F000ECD6F6000D8F3CEF0C0EC06F039
:10477000780ED66F780EB9EC01F0D8D0600EC26F0B
:10478000E50EC36F070EC46F020EC56F000EC66F35
:10479000450EC76F020EC86F000EC96F000ECA6FBC
:1047A000000ECB6F000ECC6F000ECD6F6000D8F303
:1047B000CEF0C0EC06F0600EC26FE50EC36F070EC0
:1047C000C46F020EC56F000EC66F450EC76F040E94
:1047D000C86F000EC96F000ECA6F000ECB6F000EBF
:1047E000CC6F000ECD6F6000D8F3CEF0C0EC06F0B9
:1047F0006000C8F1D6F06000CCF1D7F01E0ED86F83
:10480000020ED96F000EDA6F000EDB6F000EDC6F48
:10481000D7ECCDF0B751D8A41ED00A0EC26FC30E8C
:10482000C36F440EC46F020EC56F0A0EC66F000E32
:10483000C76F040EC86F000EC96F000ECA6F000E5E
:10484000CB6F000ECC6F000ECD6F6000D8F3CEF0B2
:10485000C0EC06F01DD00A0EC26FC30EC36F440E2B
:10486000C46F020EC56F0C0EC66F000EC76F040E2C
:10487000C86F000EC96F000ECA6F000ECB6F000E1E
:10488000CC6F000ECD6F6000D8F3CEF0C0EC06F018
:104890009105D8A41ED00A0EC26FC30EC36F440E7A
:1048A000C46F020EC56F050EC66F000EC76F060EF1
:1048B000C86F000EC96F000ECA6F000ECB6F000EDE
:1048C000CC6F000ECD6F6000D8F3CEF0C0EC06F0D8
:1048D0001DD00A0EC26FC30EC36F440EC46F020E0A
:1048E000C56F1B0EC66F000EC76F060EC86F000E99
:1048F000C96F000ECA6F000ECB6F000ECC6F000E9A
:10490000CD6F6000D8F3CEF0C0EC06F0780ED66F15
:10491000780EB9EC01F00AD09451010AD8B47BD5D5
:10492000030AD8B45DD6010AD8B428D794C095F04C
:10493000000E966F000E9E6F22D001015205D8A482
:104940001ED0000170517111D8A404D0000E716FF7
:10495000010E706F6000C0F1D6F06000C4F1D7F0B6
:104960001E0ED86F020ED96F000EDA6F000EDB6FCD
:10497000000EDC6FD7ECCDF0000E0101526F00018C
:104980009E05D8A4CCD08C05D8A439D06000C0F145
:10499000D6F06000C4F1D7F01E0ED86F020ED96FAA
:1049A000000EDA6F000EDB6F000EDC6FD7ECCDF07F
:1049B00070C072F071C073F09151D8A4AED00A0EDD
:1049C000C26FC30EC36F440EC46F020EC56F040ED8
:1049D000C66F000EC76F060EC86F000EC96F000EBF
:1049E000CA6F000ECB6F000ECC6F000ECD6F600053
:1049F000D8F3CEF0C0EC06F0010E916F8ED0020E0F
:104A00009519D8A448D001015105D8A420D00A0E88
:104A10000001C26FC30EC36F440EC46F020EC56F98
:104A20000D0EC66F000EC76F040EC86F000EC96F63
:104A3000000ECA6F000ECB6F000ECC6F000ECD6F54
:104A40006000D8F3CEF0C0EC06F0010E1FD00A0EC5
:104A50000001C26FC30EC36F440EC46F020EC56F58
:104A60000B0EC66F000EC76F040EC86F000EC96F25
:104A7000000ECA6F000ECB6F000ECC6F000ECD6F14
:104A80006000D8F3CEF0C0EC06F0000EB76F915185
:104A9000D8B495D742D0030E9519D8A43ED091052D
:104AA000D8A41ED00A0EC26FC30EC36F440EC46FCB
:104AB000020EC56F060EC66F000EC76F060EC86FDA
:104AC000000EC96F000ECA6F000ECB6F000ECC6FC8
:104AD000000ECD6F6000D8F3CEF0C0EC06F01DD014
:104AE0000A0EC26FC30EC36F440EC46F020EC56FB1
:104AF0001C0EC66F000EC76F060EC86F000EC96F82
:104B0000000ECA6F000ECB6F000ECC6F000ECD6F83
:104B10006000D8F3CEF0C0EC06F0000E9E6F410EA0
:104B2000BC6F140EBD6F9851BAEC13F00101526FB7
:104B30001200840E1119D8A47DD2360E0A6F1B0EF6
:104B40000E6F5F0E0D6F00019F05D8A449D0070EB0
:104B5000D66F6000D8F3D7F0010E06EC1AF0490EBC
:104B6000EA6FFF0EEB6F0B0EEC6F32EC13F0A30E3F
:104B7000D66FFF0ED76F080ED86F000ED96F020EDA
:104B8000DA6F000EDB6F000EDC6F000EDD6F000EC3
:104B9000DE6F000EDF6FE1EC0BF0CC0ED66FFF0E78
:104BA000D76F060ED86F000ED96F040EDA6F000EA5
:104BB000DB6F000EDC6F000EDD6F000EDE6F000E8F
:104BC000DF6FE1EC0BF0000E9F6F010E9E6F010E88
:104BD000946F010E966F010E0101406F010E3F6F41
:104BE00000019605D8B43BD14BD1600EC26FE50EE3
:104BF000C36F070EC46F020EC56F000EC66F610053
:104C000034F0C7F0040EC86F000EC96F000ECA6FF3
:104C1000000ECB6F000ECC6F000ECD6F6000D8F38E
:104C2000CEF0C0EC06F0600EC26FE50EC36F070E4B
:104C3000C46F020EC56F6B0EC66F610034F0C7F013
:104C4000020EC86F000EC96F000ECA6F000ECB6F48
:104C5000000ECC6F000ECD6F6000D8F3CEF0C0EC2C
:104C600006F08451D8A41FD0860EC26FEE0EC36F1B
:104C7000320EC46F020EC56F010EC66F610038F0B0
:104C8000C7F0060EC86F000EC96F000ECA6F000E87
:104C9000CB6F000ECC6F000ECD6F6000D8F3CEF05E
:104CA000C0EC06F0E6D0860EC26FEE0EC36F320E79
:104CB000C46F020EC56F040EC66F610038F0C7F0F6
:104CC000060EC86F000EC96F000ECA6F000ECB6FC4
:104CD000000ECC6F000ECD6F6000D8F3CEF0C0ECAC
:104CE00006F0C7D0600EC26FE50EC36F070EC46F2B
:104CF000020EC56F000EC66F610034F0C7F0020EE1
:104D0000C86F000EC96F000ECA6F000ECB6F000E89
:104D1000CC6F000ECD6F6000D8F3CEF0C0EC06F083
:104D2000600EC26FE50EC36F070EC46F020EC56F33
:104D30006B0EC66F610034F0C7F0040EC86F000E32
:104D4000C96F000ECA6F000ECB6F000ECC6F000E45
:104D5000CD6F6000D8F3CEF0C0EC06F08451D8B42B
:104D600083D7A1D7600EC26FE50EC36F070EC46F65
:104D7000020EC56F000EC66F610034F0C7F0020E60
:104D8000C86F000EC96F000ECA6F000ECB6F000E09
:104D9000CC6F000ECD6F6000D8F3CEF0C0EC06F003
:104DA000600EC26FE50EC36F070EC46F020EC56FB3
:104DB000000EC66F610034F0C7F0040EC86F000E1D
:104DC000C96F000ECA6F000ECB6F000ECC6F000EC5
:104DD000CD6F6000D8F3CEF0C0EC06F08451D8A4BB
:104DE0001FD0860EC26FEE0EC36F320EC46F020E5E
:104DF000C56F020EC66F610038F0C7F0060EC86FAF
:104E0000000EC96F000ECA6F000ECB6F000ECC6F84
:104E1000000ECD6F6000D8F3CEF0C0EC06F029D0C4
:104E2000860EC26FEE0EC36F320EC46F020EC56FD8
:104E3000050EC66F610038F0C7F0060EC86F000E91
:104E4000C96F000ECA6F000ECB6F000ECC6F000E44
:104E5000CD6F6000D8F3CEF0C0EC06F00AD09451CC
:104E6000010AD8B4C2D6030AD8B43CD7010AD8B4D0
:104E700079D794C095F0000E966F000E9E6F46D0C5
:104E800001014005D8A420D031503210D8A404D05C
:104E9000000E326E010E316E6000C4F0D6F060007C
:104EA000C8F0D7F0610028F0D8F0020E0001D96FE9
:104EB000000EDA6F000EDB6F000EDC6FD7ECCDF06A
:104EC000000E0101406F22D03F05D8A41FD02F5003
:104ED0003010D8A404D0000E306E010E2F6E60008A
:104EE000BCF0D6F06000C0F0D7F0610028F0D8F038
:104EF000040E0001D96F000EDA6F000EDB6F000E9A
:104F0000DC6FD7ECCDF0000E01013F6F00019E0574
:104F1000D8A476D08305D8A416D06000C4F0D6F00B
:104F20006000C8F0D7F0610028F0D8F0020ED96F09
:104F3000000EDA6F000EDB6F000EDC6FD7ECCDF0E9
:104F4000000E986F5BD08205D8A414D06000BCF02E
:104F5000D6F06000C0F0D7F0610028F0D8F0040E61
:104F6000D96F000EDA6F000EDB6F000EDC6FD7EC2E
:104F7000CDF0E6D7030E9519D8A440D08451D8A41B
:104F80001FD0860EC26FEE0EC36F320EC46F020EBC
:104F9000C56F030EC66F610038F0C7F0060EC86F0C
:104FA000000EC96F000ECA6F000ECB6F000ECC6FE3
:104FB000000ECD6F6000D8F3CEF0C0EC06F01ED02E
:104FC000860EC26FEE0EC36F320EC46F020EC56F37
:104FD000060EC66F610038F0C7F0060EC86F000EEF
:104FE000C96F000ECA6F000ECB6F000ECC6F000EA3
:104FF000CD6F6000D8F3CEF0C0EC06F0000E9E6FCF
:105000008305D8A40AD0410EBC6F140EBD6F985111
:10501000BAEC13F00101406F12008205D8A412000F
:10502000410EBC6F140EBD6F9851BAEC13F0010124
:105030003F6F12001105D8A4E0D000019F05D8A44D
:1050400028D0000EC26FDF0EC36F660EC46F040E51
:10505000C56F010EC66F650EC76F000EC86F000EDC
:10506000C96F000ECA6F000ECB6F000ECC6F000E22
:10507000CD6F6000D8F3CEF0C0EC06F0010E446EA8
:10508000000E0201A36F010E0101C26F000E0001AC
:105090009F6F060E0101C1651200650E446002D0CB
:1050A000442A40D0000E0001C26FDF0EC36F660EAF
:1050B000C46F040EC56F020EC66F160EC76F040EC6
:1050C000C86F000EC96F000ECA6F000ECB6F000EC6
:1050D000CC6F000ECD6F6000D8F3CEF0C0EC06F0C0
:1050E000890EC26FF70EC36F0F0EC46F020EC56F2D
:1050F0000A0EC66F590EC76F060EC86F000EC96F35
:10510000000ECA6F000ECB6F000ECC6F000ECD6F7D
:105110006000D8F3CEF0C0EC06F0000E0101C26FC3
:10512000010EC06F3A0E446419D0EF0E0001D66F25
:10513000020ED76F050ED86F44506508D96F040E64
:10514000DA6F000EDB6F000EDC6F000EDD6F000EFD
:10515000DE6F010EDF6FABECEBF02DD00E0E000119
:10516000D66FFE0ED76F080ED86F000ED96F040EE3
:10517000DA6F000EDB6F000EDC6F000EDD6F000ECD
:10518000DE6F010EDF6FABECEBF0EF0ED66F020EB1
:10519000D76F050ED86F2A0ED96F040EDA6F000E86
:1051A000DB6F000EDC6F000EDD6F000EDE6F010E98
:1051B000DF6FABECEBF0000EC26FDF0EC36F660E5D
:1051C000C46F040EC56F010EC66F44506508C76FEB
:1051D000000EC86F000EC96F000ECA6F000ECB6FB5
:1051E000000ECC6F000ECD6F6000D8F3CEF0C0EC97
:1051F00006F0000E0101C16F1200030E1119D8A4B0
:105200004DD000019F05D8A41CD08105D8A40CD096
:10521000600014F1D6F0D76B100ED86F020ED96F64
:10522000020ECCECD7F00BD0000ED76F000ED66F6D
:10523000100ED86F020ED96F050ECCECD7F0000E11
:105240009F6F01017005D8A4120000018105D8A448
:105250001200600EC26FE50EC36F070EC46F020E20
:10526000C56F4550600FC66F290EC76F050EC86F1A
:10527000000EC96F000ECA6F010ECB6F000ECC6F0F
:10528000000ECD6F6000D8F3CEF0C0EC06F06000E9
:1052900014F171F1000E0101706F1200040E11196A
:1052A000D8A446D0100E056F020E066F00019F05B0
:1052B000D8A40FD060004CF2D6F0D76B610014F088
:1052C000D8F0610018F0D9F0040ECCECD7F0000E45
:1052D0009F6F01016E05D8A41200600E0001C26F1D
:1052E000E50EC36F070EC46F020EC56F9351600FBA
:1052F000C66F04010551190F0001C76F0401065163
:10530000030F0001C86F000EC96F000ECA6F010EB7
:10531000CB6F000ECC6F000ECD6F6000D8F3CEF0D7
:10532000C0EC06F093C06FF1000E01016E6F120029
:10533000050E1119D8A4A4D0100E0B6F020E0C6F1D
:10534000020E096F090E046F00019F05D8A40FD04B
:10535000000ED76F1E0ED66F61002CF0D8F06100E2
:1053600030F0D9F0030ECCECD7F0000E9F6F0101A6
:105370006E05D8A412000A0E0001C06F93518FEC85
:105380001CF0600F0401096F0A0E0001BC6F9351FD
:10539000A2EC1DF0600F0401046F600E0919D8B46F
:1053A00026D0600E0001C26FE50EC36F070EC46FFA
:1053B000020EC56F610024F0C6F004010B51150FF9
:1053C0000001C76F04010C51030F0001C86F000EEC
:1053D000C96F000ECA6F010ECB6F000ECC6F000EAE
:1053E000CD6F6000D8F3CEF0C0EC06F024D0600E94
:1053F0000001C26FE50EC36F070EC46F020EC56FCA
:105400006C0EC66F04010B51150F0001C76F04012C
:105410000C51030F0001C86F000EC96F000ECA6F58
:10542000010ECB6F000ECC6F000ECD6F6000D8F375
:10543000CEF0C0EC06F0600EC26FE50EC36F070E33
:10544000C46F020EC56F610010F0C6F004010B516D
:105450001E0F0001C76F04010C51030F0001C86F3C
:10546000000EC96F000ECA6F010ECB6F000ECC6F1D
:10547000000ECD6F6000D8F3CEF0C0EC06F052D72E
:10548000060E1119D8A41200100E076F020E086F35
:1054900000019F05D8A40FD060000CF1D6F0D76BA7
:1054A00061001CF0D8F0610020F0D9F00D0ECCECBA
:1054B000D7F0000E9F6F01016705D8A41200600E9F
:1054C0000001C26FE50EC36F070EC46F020EC56FF9
:1054D0004350600FC66F04010751190F0001C76FD9
:1054E00004010851030F0001C86F000EC96F000EC0
:1054F000CA6F010ECB6F000ECC6F000ECD6F600037
:10550000D8F3CEF0C0EC06F060000CF168F1000EAC
:105510000101676F1200C6EC14F013ECF5F0000EF9
:105520000001BD6F000EBC6FFBEC1EF09F0AD8B4EB
:1055300009D0000E0001BD6F000EBC6F9F0EBE6F44
:1055400097EC1BF09F0E57EC19F0A6EC1FF0210E04
:105550003A01136F3D017399D28ED28C010E59EC32
:105560001AF0F66FF651FDEC0FF0010E0001A26F7C
:10557000010E516EC682200EA7EC1EF00101E56FF0
:10558000A4EC1FF057ECE3F0CBEC1CF0000E000194
:10559000CC6F6000E4F0CDF06000E8F0CEF0020ED9
:1055A000D06F020ECF6F040ED26F040ED16F090EB2
:1055B000DAECE0F0600030F339F0600034F33AF0F8
:1055C000010E0101BA6F0101AF05D8A403D0020199
:1055D000614B622B00019051D8A46EEC18F00001D1
:1055E0009051D8A43DEC16F020EC1EF082EC1FF098
:1055F000E5EC00F000019051D8A456EC0AF0FDEC67
:1056000018F0A7EC12F0DBEC0AF0D2ECFBF0F8ECAF
:105610001BF001015B05D8A422D0040E0001A219E1
:10562000D8B41DD0030EA219D8B419D0A205D8B48D
:1056300016D0050EA219D8B412D09051D8B40FD0FC
:10564000B451D8A40CD0AD51D8A409D0A2C0A1F0B7
:10565000050EA26F010E9F6F010E0101C76F515021
:10566000D8B4B4EC16F00101AD51D8B40FD000019C
:105670009051D8A40BD0010E0101766F6D0E000180
:10568000A219D8B403D0000E0101AD6F0201495137
:105690004A11D8B403D04907D8A04A0701017605BA
:1056A000D8A42BD00001A205D8B427D002014951BB
:1056B0004A11D8A422D0000E4A6F400E496F6000F4
:1056C000B4F2EAF06000D0F2EBF06000B8F2ECF077
:1056D000600084F5EDF0600064F2EEF060000CF91B
:1056E000EFF0600010F9F0F0600000F6F1F0010159
:1056F0005F51CEECFAF00101766F0A0E0001A2199B
:10570000D8A487D39905D8A40BD0000E996F7AC07E
:1057100043F27BC044F2010E0101766F000E476F29
:105720000001AE05D8B403D0AF05D8A4DED0010186
:105730004F51D8A46DD0000178517A1904E1795104
:105740007B19D8B458D0000E0101236F000E226FD0
:10575000010E0001B36F4AD082EC1FF000017851B6
:105760007A1910E179517B19D8A40CD0000E0101EF
:10577000AA6F000E236F000E226F000E0001B36FA0
:10578000010E9F6F0101235104E1C80E225DD8A0D4
:105790002DD0000E0001D76F000ED66F100ED86FFF
:1057A000020ED96F060ECCECD7F07A51351806E10F
:1057B0007B513618D8A402D0000E9A6F010E010159
:1057C000AA6F000E236F000E226F000E0001B36F50
:1057D000010E9F6F410E0001F46FF00EF36F330E58
:1057E000E82EFED7F32FFCD7F42FFAD70001B3052C
:1057F000D8A406D0B1D7000E0101AA6F000E506FD9
:1058000000017A517B11D8A403D0010E01014F6F22
:1058100001014E51D8A469D035503610D8A402D019
:10582000010E4E6F00017251351804E173513618A4
:10583000D8B45BD0000E0101236F000E226F010E61
:105840000001B36F4ED082EC1FF000017251351889
:1058500017E173513618D8A413D078517A1910E192
:1058600079517B19D8A40CD0000E0101AA6F000E4B
:10587000236F000E226F000E0001B36F010E9F6FA9
:105880000101235104E1640E225DD8A02AD0000E4C
:105890000001D76F000ED66F100ED86F020ED96FB1
:1058A000060ECCECD7F0000E9A6F6000C8F135F010
:1058B0006000CCF136F0000E0101236F000E226F64
:1058C000000E0001B36F010E9F6F410E0001F46FD7
:1058D000F00EF36F330EE82EFED7F32FFCD7F42F24
:1058E000FAD70001B305D8B4AED70101AA05D8B4E0
:1058F00004D000018605D8A402D0010E09D0010110
:10590000AA51D8A407D000018651D8A403D0000E14
:105910000101746F5A0E0001A619D8B404D05A0EB2
:1059200007EC15F0A66FB051B119D8B404D0B0513E
:1059300086EC02F0B16F4950D8B436D0A551D8A446
:1059400031D0000ECA6F100EC96F8CEC1DF000092B
:10595000D8A428D06000E0F2BCF04050F3EC10F086
:105960008F6F8505D8A41AD0120E8F6502D0120E43
:1059700007D0030E8F6105D0010E406402D0020EE5
:105980008F6F050E8F610AD0020E8E6107D0020E56
:105990008D6F8DC08EF0010E0101566F010E010159
:1059A0005A6F02D0000E496E010158510001B8191A
:1059B000D8B411D00101585198EC1FF0B86F010E06
:1059C0000101576F0001B851B7190101596F000E5D
:1059D000496F010E486F0001A505D8A416D0010E2D
:1059E0000101CE6F2F5104E13D0E2E5DD8A00DD0E8
:1059F0000B0E0001A26F000E0101CE6F000E2F6F83
:105A0000000E2E6F010E00019F6F0001A405D8A4A7
:105A100023D001012F5120E13D0E2E5DD8B01CD0C6
:105A2000000ECE6F000E2F6F000E2E6F48A006D016
:105A3000000E00018F6F010E01015A6F48A20CD0B9
:105A40004050D8A409D00001B851010A0101586F93
:105A5000000E496F010E486F000E0001CA6F100E54
:105A6000C96F55EC1BF00009D8B406D0AA51D8A4D0
:105A700003D0010E0101C96F000E0001CA6F100EA4
:105A8000C96F76EC1BF00009D8B408D0000E0101F4
:105A9000C96F000E02016E6F000E6D6F0001A90547
:105AA000D8A415D002016E5104E1330E6D5DD8A06B
:105AB0000ED00C0E0001A26F000E0101C96F000E86
:105AC00002016E6F000E6D6F010E00019F6F0201EB
:105AD0006A5104E1960E695DD8A01ED0010E000146
:105AE0009F6F000E0101C66F000E02016A6F000E6B
:105AF000696F00018705D8A402D0010E3E6E8505AE
:105B0000D8A403D0010E0101416F00018605D8A47D
:105B100003D0010E0101436F32ECEFF001017E5121
:105B2000D8B402D0000E7E6F000E0001CA6F100EB6
:105B3000C96F55EC1BF0E806D8B409D0000ECA6F47
:105B4000100EC96F76EC1BF0E806D8A422D0AA513B
:105B5000D8A410D06000A4F2CCF0600050F6CDF0D4
:105B6000600010F6CEF0000ECF6F0A0ECFECE7F01B
:105B7000A96F0FD0600030F1CCF0600048F6CDF096
:105B8000600008F6CEF0000ECF6F0C0ECFECE7F001
:105B90004C6E000ECA6F200EC96F55EC1BF0E80664
:105BA000D8B409D0000ECA6F200EC96F76EC1BF076
:105BB000E806D8A422D0AA51D8A410D06000A0F240
:105BC000CCF060004CF6CDF060000CF6CEF0000E8C
:105BD000CF6F0B0ECFECE7F0A86F0FD060009CF2F8
:105BE000CCF0600044F6CDF0600004F6CEF0000E7C
:105BF000CF6F0D0ECFECE7F0A76FA705D8A40BD0A1
:105C000065EC05F005D082EC1FF08FECFEF0506ED5
:105C10005050D8B4F8D70001B005D8A404D0A7518B
:105C2000B8EC1DF007D0020EB019D8A405D0A851C9
:105C3000B8EC1DF03D6E18D0030EB019D8A414D0E6
:105C40008851B8EC1DF03D6E8905D8A402D0010E34
:105C500001D0000E0101456F000186510101451977
:105C6000D8B402D0010E446F000185513D18D8B45C
:105C700011D03D04D8A405D08EC055F1010E8D6F12
:105C800002D055C18DF08DC08EF0010E0101566F0E
:105C9000010E426F000E01017F6F0001A005D8A424
:105CA00013D0600080F2CCF0000ECD6F000ECE6FEE
:105CB000000ECF6F140ECFECE7F0A06FA051D8A468
:105CC0001AD0A1C0A2F00BD0000ECA6F800EC96F0F
:105CD00076EC1BF0E806D8A406D0640EA26F010E85
:105CE0009F6F010E06D0000ECA6F800EC96F8CEC3C
:105CF0001DF001017F6F020E0001CA6F000EC96F17
:105D000076EC1BF0E806D8B409D0020ECA6F000E7C
:105D1000C96F55EC1BF0E806D8A415D06000A8F2B6
:105D2000CCF0010ECD6F010ECE6F000ECF6F0E0EB8
:105D3000CFECE7F0AA6F030EB119D8A4AAC080F186
:105D4000010E0101766F01013251D8A48FECFEF0F3
:105D5000000E0001CA6F400EC96F55EC1BF0E8063B
:105D6000D8A40BD0010E0101CD6F000E00017F6F92
:105D7000000E7E6F010E0101476F000E0001CA6F19
:105D8000400EC96F8CEC1DF0E806D8A416D07F51E8
:105D900004E1320E7E5DD8A010D0000E0101476FE5
:105DA00000019051D8B409D065EC05F0A2C0A1F073
:105DB000040E0001A26F010E9F6F000ECA6F400E0D
:105DC000C96F76EC1BF0E806D8A416D07F5114E119
:105DD000320E7E5DD8B010D0000E0101CD6F000EE6
:105DE00000017F6F000E7E6F01014705D8A404D02B
:105DF000010E491B010E486F87C073F10001800539
:105E0000D8A430EFC5F0A2C0A1F0030EA26F00EF3E
:105E1000C4F00B0EA219D8A434D09951D8A409D03B
:105E2000010E996F7AC043F27BC044F2010E01016A
:105E3000766F1E0E0001A619D8B404D01E0E07EC12
:105E400015F0A66F4950D8B407D08E51CCEC1AF09B
:105E50008D6F010E0101566F0001A405D8A40CD06E
:105E60000A0EA26F000E0101CE6F000E2F6F000E02
:105E70002E6F010E00019F6F8005D8B4C4D730EF9C
:105E8000C5F00C0EA219D8A425D19951D8A417D0C9
:105E9000010E996F7AC043F27BC044F2010E0101FA
:105EA000766F000E0001CA6F100EC96F8CEC1DF0EA
:105EB0000009D8A404D00A0EA26F010E9F6FDC0E59
:105EC000A619D8B404D0DC0E07EC15F0A66F495023
:105ED000D8B411D06000D8F1BCF06000DCF1BDF0A6
:105EE00089EC11F06000F0F276F06000F4F277F0E7
:105EF000010E0101546F00017651335C7751345823
:105F0000D8B009D06000CCF076F06000D0F077F027
:105F1000010E0101546F000176517711D8A407D00A
:105F2000000E776F010E766F010E0101546F000EA7
:105F30000001CC6F000ECD6F000ECE6F000ECF6F44
:105F4000120ECFECE7F0E806D8A407D074C076F0C4
:105F500075C077F0010E0101546F000E0001CC6F87
:105F6000000ECD6F000ECE6F000ECF6F130ECFEC74
:105F7000E7F0E806D8A409D06000DCF076F0600015
:105F8000E0F077F0010E0101546F000E0001CA6FBE
:105F9000100EC96F76EC1BF00009D8B457D0000E74
:105FA000A96F000E986F76517A1904E177517B1929
:105FB000D8B434D06000D0F137F06000D4F138F0BC
:105FC0007AC074F07BC075F0000E8B6F000E8A6F84
:105FD000000E896F000E886F000E01014D6F000EDC
:105FE0004C6F000E4B6F000E4A6F00018705D8A45E
:105FF00005D0000E0101496F010E486F000E00012F
:106000008F6F010E01015A6F010E00018D6F010E9D
:106010000101566F000E506F000E4F6F78C043F2B3
:1060200079C044F2355000017A1906E136507B19E7
:10603000D8A402D0000E9A6F0A0EA26F010E9F6FB5
:106040009051D8A403D0050EC2ECF9F0000E000167
:10605000CA6F100EC96F55EC1BF0E806D8B409D012
:10606000000ECA6F100EC96F76EC1BF0E806D8A4BC
:106070000FD06000A4F2CCF0600050F6CDF06000CC
:1060800010F6CEF0000ECF6F0A0ECFECE7F0A96F3E
:10609000000ECA6F200EC96F55EC1BF0E806D8B48D
:1060A00009D0000ECA6F200EC96F76EC1BF0E8060F
:1060B000D8A4E2D66000A0F2CCF060004CF6CDF09F
:1060C00060000CF6CEF0000ECF6F0B0ECFECE7F0B9
:1060D000A86FD2D6640EA219D8A489D09951D8A499
:1060E00009D0010E996F7AC043F27BC044F2010ED1
:1060F0000101766F1E0E0001A619D8B404D01E0E41
:1061000007EC15F0A66F4950D8B409D0600088F2AA
:10611000BCF09551D3EC11F0946F010E966FA3056E
:10612000D8A402D0010E9E6FA405D8B40ED020D002
:10613000650E09D06E0E07D0820E05D0780E03D002
:106140006D0E01D0640EA26F11D09551010AD8B422
:10615000EFD7030AD8B4EED7010AD8B4EDD7070AAF
:10616000D8B4ECD7010AD8B4EBD7ECD7010E9F6FA7
:10617000000ECA6F400EC96F55EC1BF0E806D8A49C
:1061800008D0010E0101CD6F000E00017F6F000EDF
:106190007E6F000ECA6F400EC96F8CEC1DF0E806D2
:1061A000D8A412D07F5104E1510E7E5DD8A00CD04E
:1061B0000A0EA26F010E9F6F000E0101CD6F000E3F
:1061C00000017F6F000E7E6F000ECA6F400EC96F18
:1061D00076EC1BF0E806D8A44FD67F5107E1510EAC
:1061E0007E5DD8B049D60A0E39EFC3F045D6650EAC
:1061F000A219D8A4DFD19951D8A409D0010E996F62
:106200007AC043F27BC044F2010E0101766FDC0ECE
:106210000001A619D8B404D0DC0E07EC15F0A66F67
:106220004950D8B411D06000D8F1BCF06000DCF166
:10623000BDF089EC11F06000F0F276F06000F4F24D
:1062400077F0010E0101546F0001A305D8A404D01A
:10625000010E9E6F000E986FA405D8A453D07651FE
:106260007A1904E177517B19D8B434D06000D0F1A9
:1062700037F06000D4F138F07AC074F07BC075F06C
:10628000000E8B6F000E8A6F000E896F000E886FF4
:10629000000E01014D6F000E4C6F000E4B6F000E93
:1062A0004A6F00018705D8A405D0000E0101496F8F
:1062B000010E486F000E00018F6F010E01015A6F31
:1062C000010E00018D6F010E0101566F000E506F1F
:1062D000000E4F6F78C043F279C044F23550000190
:1062E0007A1906E136507B19D8A402D0000E9A6FB5
:1062F0000A0EA26F010E9F6F9051D8A403D0050E15
:10630000C2ECF9F0000E0001CC6F000ECD6F000E54
:10631000CE6F000ECF6F120ECFECE7F0E806D8A4D8
:1063200007D074C076F075C077F0010E0101546F8C
:10633000000E0001CC6F000ECD6F000ECE6F000E70
:10634000CF6F130ECFECE7F0E806D8A409D06000B9
:10635000DCF076F06000E0F077F0010E0101546FA0
:10636000000E0001CC6F000ECD6F000ECE6F000E40
:10637000CF6F0F0ECFECE7F0E806D8A471D0030E74
:10638000B119D8A425D06000D8F1C9F06000DCF1C3
:10639000CAF05A0ECB6FABEC08F0F36F060EF36148
:1063A00005D00A0E7627000E772304D03C0E765FC8
:1063B000000E775B775104E13E0E765DD8A004D0E5
:1063C000000E776F3D0E766F010E0101546F48D0BD
:1063D000020EB119D8A415D06000D8F1C9F0600040
:1063E000DCF1CAF05A0ECB6FABEC08F0F36F090E7C
:1063F000F36105D00A0E7627000E7723E5D75A0EF3
:106400002BD0B105D8A42CD06000D8F1C9F0600021
:10641000DCF1CAF0540ECB6FABEC08F00009D8A445
:106420000BD06000D8F1C9F06000DCF1CAF05A0E60
:10643000CB6FABEC08F0DAD76000D8F1C9F06000A0
:10644000DCF1CAF05A0ECB6FABEC08F0F36F020E22
:10645000F36101D0CFD7140E765F000E775BB4D70F
:10646000000E0001CC6F000ECD6F000ECE6F000E3F
:10647000CF6F100ECFECE7F0E806D8A430D0020EB4
:10648000B119D8B42CD0B105D8A429D06000D8F166
:10649000C9F06000DCF1CAF0540ECB6FABEC08F031
:1064A0000009D8A415D06000D8F1C9F06000DCF173
:1064B000CAF0480ECB6FABEC08F0F36F090EF36136
:1064C00005D0640E7627000E772306D0840E01D007
:1064D000E80E765F030E775B010E0101546F000139
:1064E0007651335C77513458D8B009D06000CCF085
:1064F00076F06000D0F077F0010E0101546F0001DA
:1065000076517711D8A407D0000E776F010E766F01
:10651000010E0101546F000E0001CA6F400EC96FD9
:1065200055EC1BF0E806D8A40ED0000E986F010EB3
:106530000101CD6F000E00017F6F000E7E6F7AC0EB
:1065400076F07BC077F0000ECA6F400EC96F8CECFE
:106550001DF0E806D8A412D07F5104E1510E7E5DF3
:10656000D8A00CD00A0EA26F010E9F6F000E010181
:10657000CD6F000E00017F6F000E7E6F000ECA6FA0
:10658000400EC96F76EC1BF0E806D8A475D47F5195
:1065900010E1510E7E5DD8B06FD4640EA26F000E74
:1065A0000101CD6F000E00017F6F000E7E6F010EA6
:1065B00062D462D46E0EA219D8A489D09951D8A4FD
:1065C00009D0010E996F7AC043F27BC044F2010EEC
:1065D0000101766F1E0E0001A619D8B404D01E0E5C
:1065E00007EC15F0A66F4950D8B409D0600088F2C6
:1065F000BCF09551D3EC11F0946F010E966FA3058A
:10660000D8A402D0010E9E6FA405D8B412D023D016
:106610006F0EA26F030E93EC1FF01AD06F0EA26FD5
:10662000010E93EC1FF014D0700E01D0640EA26F17
:106630000FD09551010AD8B4EBD7030AD8B4EED7DE
:10664000010AD8B4F1D7070AD8B4F0D7010AEED7B7
:10665000010E00019F6F000ECA6F400EC96F55EC0E
:106660001BF0E806D8A408D0010E0101CD6F000E82
:1066700000017F6F000E7E6F000ECA6F400EC96F63
:106680008CEC1DF0E806D8A412D07F5104E1510E25
:106690007E5DD8A00CD00A0EA26F010E9F6F000E77
:1066A0000101CD6F000E00017F6F000E7E6F000EA6
:1066B000CA6F400EC96F76EC1BF0E806D8A43CEF19
:1066C000AFF07F5102E133EFC3F03CEFAFF06F0E5C
:1066D000A219D8A41DD39951D8A409D0010E996F3D
:1066E0007AC043F27BC044F2010E0101766F080EBE
:1066F000406405D0080E00018F6F080E406E010E39
:1067000000018D6F010E8E6F9C51D8A40BD09B5150
:10671000D8A408D01E0EA619D8B404D01E0E07ECBB
:1067200015F015D09C05D8A408D0A00EA619D8B491
:1067300004D0A00E07EC15F00AD09B05D8A408D011
:10674000DC0EA619D8B404D0DC0E07EC15F0A66F49
:106750004950D8B43AD09C51D8A415D09B51D8A454
:1067600012D0600088F2BCF09551D3EC11F0946F18
:106770009D05D8A405D0020E946502D0020E946F38
:10678000010E966F22D09C05D8A40BD06C5181ECE1
:106790001AF0F36FF3516C6F6D6B010E01013E6FD8
:1067A00014D09B05D8A411D06000A0F1BCF060000B
:1067B000A4F1BDF048EC15F06000F0F268F0600064
:1067C000F4F269F0010E01013D6F0001A305D8A4A8
:1067D00004D0000E986F010E9E6FA405D8A46ED051
:1067E0009C51D8A461D09B51D8B43DD05DD0010E4E
:1067F0009C6F000E476E000E9B6F0BD09D05D8B4AA
:106800000BD0010E9B6F000E0101756F000E000191
:106810009C6F010E986F52D04704D8A44FD0010E40
:1068200001019D6F000E000114D04704D8A446D08A
:1068300001017505D8A442D000019D05D8B40AD045
:106840006E5101EC16F001019D6F00016E51DDECFF
:106850000CF0AC6F000E0101A96F6F0E0001A26F6A
:10686000010E9F6F2BD09551010AD8B4C0D7030AEF
:10687000D8B4C4D7010AD8B4D8D720D0000E9C6FA2
:10688000010E476E6CC06EF06DC06FF014D09D05A8
:10689000D8B411D0000E9B6F010E0101756F68C056
:1068A0006AF069C06BF007D09551010AD8B4E6D7F9
:1068B000030AD8B4ECD7010E0001966F01019D05C3
:1068C000D8B404D00001AC05D8A407D00101A95167
:1068D000D8A403D0010E0001B36F0001B305D8B4F2
:1068E00056D059D082EC1FF000016E5102013B19C5
:1068F0001DE100016F5102013C19D8A417D000011D
:106900006A510201391912E100016B5102013A1971
:10691000D8A40CD0000E0101A96F000E236F000E49
:10692000226F000E0001B36F010E9F6F0101235112
:1069300004E1C80E225DD8A02AD0000E0001D76F56
:10694000000ED66F100ED86F020ED96F0B0ECCEC66
:10695000D7F0010E0101A96F000E9D6F000E00011E
:10696000AC6F000E0101236F000E226F000E0001BC
:10697000B36F010E9F6F410E0001F46FF00EF36FC5
:10698000330EE82EFED7F32FFCD7F42FFAD70001F1
:10699000B305D8B4A7D7600080F2CCF0000ECD6F5D
:1069A000000ECE6F000ECF6F140ECFECE7F0A06F8D
:1069B000A005D8A406D0A2C0A1F00A0EA26F010EB5
:1069C0009F6F000ECC6F000ECD6F000ECE6F000ECD
:1069D000CF6F0F0ECFECE7F0E806D8A4DCD0030EA3
:1069E000B119D8A426D09B05D8A405D0000E696F94
:1069F000010E686F5BD09C51D8B4CDD06000B0F16F
:106A0000C9F06000B4F1CAF05A0ECB6FABEC08F0DD
:106A1000F36F070EF36105D00A0E6C27000E6D238D
:106A200004D0460E6C5F000E6D5B010E01013E6FDF
:106A3000B2D0020EB119D8A451D09B05D8A43AD037
:106A40006000A0F1C9F06000A4F1CAF0480ECB6F5D
:106A5000ABEC08F0F36F020EF36115D06000A0F10B
:106A6000C9F06000A4F1CAF05A0ECB6FABEC08F08D
:106A7000F36F090EF36105D00A0E6827000E692333
:106A800015D05A0E10D06000A0F1C9F06000A4F13A
:106A9000CAF05A0ECB6FABEC08F0F36F030EF36144
:106AA00001D0EAD71E0E685F000E695B010E01017E
:106AB0003D6F71D09C51D8B46ED06000B0F1C9F078
:106AC0006000B4F1CAF05A0ECB6FABEC08F0F36F74
:106AD000090EF36101D0A0D75A0EA4D7B105D8A4EE
:106AE0005AD09B05D8A42AD06000A0F1C9F060005C
:106AF000A4F1CAF0480ECB6FABEC08F0F36F020EB6
:106B0000F3610BD06000A0F1C9F06000A4F1CAF0FD
:106B10005A0ECB6FABEC08F0ABD76000A0F1C9F018
:106B20006000A4F1CAF05A0ECB6FABEC08F0F36F23
:106B3000050EF36101D0A0D7320EB5D79C51D8B461
:106B40002AD06000B0F1C9F06000B4F1CAF0480E7C
:106B5000CB6FABEC08F0F36F020EF3610BD060006B
:106B6000B0F1C9F06000B4F1CAF05A0ECB6FABECD3
:106B700008F0ADD76000B0F1C9F06000B4F1CAF020
:106B80005A0ECB6FABEC08F0F36F050EF36101D03A
:106B900043D7320E47D7000E0001CC6F000ECD6FE9
:106BA000000ECE6F000ECF6F100ECFECE7F0E806B0
:106BB000D8A451D0B105D8A43CD09B05D8A41BD0F3
:106BC0006000A0F1C9F06000A4F1CAF0480ECB6FDC
:106BD000ABEC08F0F36F020EF36105D0640E68278A
:106BE000000E692304D0C80E685F000E695B010EB9
:106BF00001013D6F30D09C51D8B42DD06000B0F170
:106C0000C9F06000B4F1CAF0480ECB6FABEC08F0ED
:106C1000F36F020EF36105D0640E6C27000E6D2336
:106C200004D0C80E6C5F000E6D5B010E01013E6F5B
:106C300012D0020EB119D8A40ED09B05D8A40BD047
:106C40006000A0F1C9F06000A4F1CAF0480ECB6F5B
:106C5000ABEC08F0BFD73F500001F36FF46B6C5101
:106C6000F35D6D51F459D8B004D06000FCF06CF0C5
:106C70006D6B68510101085D0001695101010959FD
:106C8000D8B004D008C168F009C169F0000E000155
:106C9000CA6F400EC96F55EC1BF0E806D8A40ED0A1
:106CA000000E986F010E0101CD6F000E00017F6F85
:106CB000000E7E6F000E9B6F000E9C6F000ECA6F61
:106CC000400EC96F8CEC1DF0E806D8A412D07F519D
:106CD00004E1510E7E5DD8A00CD00A0EA26F010E09
:106CE0009F6F000E0101CD6F000E00017F6F000E3F
:106CF0007E6F000ECA6F400EC96F76EC1BF0E8067F
:106D0000D8A43CEFAFF07F5101E11FD23CEFAFF0D0
:106D1000700EA219D8A423D29951D8A409D0010E7B
:106D2000996F7AC043F27BC044F2010E0101766F85
:106D3000000E00018F6F000E406EDC0EA619D8B455
:106D400004D0DC0E07EC15F0A66F4950D8B411D072
:106D5000600098F1BCF060009CF1BDF089EC11F08E
:106D60006000F0F266F06000F4F267F0010E0101DD
:106D70003C6F0001A305D8A404D0000E986F010E4B
:106D80009E6FA405D8A432D066517A1904E16751E8
:106D90007B19D8B428D0000E8B6F000E8A6F000EBE
:106DA000896F000E886F000E01014D6F000E4C6F51
:106DB000000E4B6F000E4A6F00018705D8A405D066
:106DC000000E0101496F010E486F010E00018D6F29
:106DD000010E8E6F66C000F167C001F1010E010166
:106DE0009E6F000EA96F000E00019A6F01019E05B3
:106DF000D8A406D0A951D8A403D0010E0001B36FC6
:106E00000001B305D8B45AD05DD082EC1FF0010167
:106E10000051021924E101510319D8A420D0000E19
:106E2000A96F02C176F003C177F002C178F003C107
:106E300079F06000E0F1BCF06000E4F1BDF05FECDF
:106E40000BF0000E01019E6F000E236F000E226FEB
:106E5000000E0001B36F0A0EA26F010E9F6F0101B9
:106E6000235104E1C80E225DD8A028D0000E0001F5
:106E7000D76F000ED66F100ED86F020ED96F0B0EA3
:106E8000CCECD7F0010E0101A96F000E9E6F000E31
:106E9000236F000E226F000E0001B36F0A0EA26F67
:106EA000010E9F6F410E0001F46FF00EF36F330E71
:106EB000E82EFED7F32FFCD7F42FFAD70001B30545
:106EC000D8B4A3D7000ECC6F000ECD6F000ECE6FDE
:106ED000000ECF6F120ECFECE7F0E806D8A407D073
:106EE00074C066F075C067F0010E01013C6F000EC2
:106EF0000001CC6F000ECD6F000ECE6F000ECF6F75
:106F0000130ECFECE7F0E806D8A409D06000DCF05F
:106F100066F06000E0F067F0010E01013C6F000ECA
:106F20000001CC6F000ECD6F000ECE6F000ECF6F44
:106F30000F0ECFECE7F0E806D8A471D0030EB1191C
:106F4000D8A425D0600098F1C9F060009CF1CAF087
:106F50005A0ECB6FABEC08F0F36F060EF36105D061
:106F60000A0E6627000E672304D03C0E665F000EF3
:106F7000675B675104E13E0E665DD8A004D0000E49
:106F8000676F3D0E666F010E01013C6F48D0020E27
:106F9000B119D8A415D0600098F1C9F060009CF137
:106FA000CAF05A0ECB6FABEC08F0F36F090EF36129
:106FB00005D00A0E6627000E6723E5D75A0E2BD0A0
:106FC000B105D8A42CD0600098F1C9F060009CF104
:106FD000CAF0540ECB6FABEC08F00009D8A40BD06C
:106FE000600098F1C9F060009CF1CAF05A0ECB6FB6
:106FF000ABEC08F0DAD7600098F1C9F060009CF1C2
:10700000CAF05A0ECB6FABEC08F0F36F020EF361CF
:1070100001D0CFD7140E665F000E675BB4D7000EA9
:107020000001CC6F000ECD6F000ECE6F000ECF6F43
:10703000100ECFECE7F0E806D8A430D0020EB1195C
:10704000D8B42CD0B105D8A429D0600098F1C9F0EB
:1070500060009CF1CAF0540ECB6FABEC08F0000955
:10706000D8A415D0600098F1C9F060009CF1CAF076
:10707000480ECB6FABEC08F0F36F090EF36105D04F
:10708000640E6627000E672306D0840E01D0E80E3A
:10709000665F030E675B010E01013C6F00016651E4
:1070A000335C67513458D8B009D06000CCF066F03A
:1070B0006000D0F067F0010E01013C6F00016651E5
:1070C0006711D8A407D0000E676F010E666F010E1E
:1070D00001013C6F000E0001CA6F400EC96F55ECF4
:1070E0001BF0E806D8A40AD0000E986F010E01012B
:1070F000CD6F000E00017F6F000E7E6F000ECA6F15
:10710000400EC96F8CEC1DF0E806D8A412D07F5158
:1071100004E1510E7E5DD8A00CD00A0EA26F010EC4
:107120009F6F000E0101CD6F000E00017F6F000EFA
:107130007E6F000ECA6F400EC96F76EC1BF0E8063A
:10714000D8A43CEFAFF07F5108E1510E7E5DD8B07E
:107150003CEFAFF06E0E39EFC3F03CEFAFF0780EBE
:10716000A219D8A484D09951D8A409D0010E996F3E
:107170007AC043F27BC044F2010E0101766F1E0E0D
:107180000001A619D8B404D01E0E07EC15F0A66FA6
:107190004950D8B409D0600088F2BCF09551D3ECC6
:1071A00011F0946F010E966FA305D8A402D0010EC2
:1071B0009E6FA405D8B40CD01ED0790E07D07A0EDD
:1071C00005D0780E03D07C0E01D0810EA26F11D0B5
:1071D0009551010AD8B4F1D7030AD8B4F0D7010AFF
:1071E000D8B4EFD7070AD8B4EED7010AD8B4EDD790
:1071F000E8D7010E9F6F000ECA6F400EC96F55ECA5
:107200001BF0E806D8A408D0010E0101CD6F000ED6
:1072100000017F6F000E7E6F000ECA6F400EC96FB7
:107220008CEC1DF0E806D8A412D07F5104E1510E79
:107230007E5DD8A00CD00A0EA26F010E9F6F000ECB
:107240000101CD6F000E00017F6F000E7E6F000EFA
:10725000CA6F400EC96F76EC1BF0E806D8A43CEF6D
:10726000AFF07F5102E133EFC3F03CEFAFF0790EA6
:10727000A219D8A47AD09951D8A409D0010E996F37
:107280007AC043F27BC044F2010E0101766F1E0EFC
:107290000001A619D8B404D01E0E07EC15F0A66F95
:1072A0004950D8B408D001016A5130EC1AF00101FC
:1072B0006A6F010E696F0001A405D8A404D0780E8E
:1072C000A26F010E9F6F600080F2CCF0000ECD6FB8
:1072D000000ECE6F000ECF6F140ECFECE7F0A06F54
:1072E000A005D8A406D0A2C0A1F00A0EA26F010E7C
:1072F0009F6F000ECA6F400EC96F55EC1BF0E80679
:10730000D8A408D0010E0101CD6F000E00017F6FDF
:10731000000E7E6F000ECA6F400EC96F8CEC1DF020
:10732000E806D8A412D07F5104E1510E7E5DD8A0AA
:107330000CD00A0EA26F010E9F6F000E0101CD6FDF
:10734000000E00017F6F000E7E6F000ECA6F400EB0
:10735000C96F76EC1BF0E806D8A43CEFAFF07F5184
:1073600002E124EFBEF03CEFAFF07A0EA219D8A4F0
:10737000DAD09951D8A409D0010E996F7AC043F29E
:107380007BC044F2010E0101766F1E0E0001A619AA
:10739000D8B404D01E0E07EC15F0A66F4950D8B42F
:1073A00009D0600088F2BCF09551D3EC11F0946FD5
:1073B000010E966FA305D8A402D0010E9E6FA405FE
:1073C000D8B408D012D0010E03D0020E01D0030EA3
:1073D000B06F0BD09551010AD8B4F5D7030AD8B4D1
:1073E000F4D7010AD8B4F3D7EED7B051B119D8B455
:1073F00048D0000E8F6F010E01015A6F010E00017F
:107400008D6F010E0101566F0001B05186EC02F044
:10741000B16F000E8B6F000E8A6F000E896F000E29
:10742000886F000E01014D6F000E4C6F000E4B6F08
:10743000000E4A6F000E0001A96F000EA86F000E2B
:107440004C6E000EA76F000E0101806F00018705D2
:10745000D8A405D0000E0101496F010E486F00014C
:107460008605D8A405D0000E0101456F010E446FBA
:1074700000018505D8A405D0000E3D6E010E010166
:10748000426F600080F2CCF0000E0001CD6F000E64
:10749000CE6F000ECF6F140ECFECE7F0A06FA005FB
:1074A000D8A406D0A2C0A1F00A0EA26F010E9F6F51
:1074B000000ECA6F400EC96F55EC1BF0E806D8A449
:1074C00008D0010E0101CD6F000E00017F6F000E8C
:1074D0007E6F000ECA6F400EC96F8CEC1DF0E8067F
:1074E000D8A412D07F5104E1510E7E5DD8A00CD0FB
:1074F0000A0EA26F010E9F6F000E0101CD6F000EEC
:1075000000017F6F000E7E6F000ECA6F400EC96FC4
:1075100076EC1BF0E806D8A43CEFAFF07F5101E118
:1075200093D33CEFAFF07B0EA219D8A448D0995169
:10753000D8A409D0010E996F7AC043F27BC044F2FF
:10754000010E0101766F000E0001CA6F400EC96F77
:1075500055EC1BF0E806D8A408D0010E0101CD6F50
:10756000000E00017F6F000E7E6F000ECA6F400E8E
:10757000C96F8CEC1DF0E806D8A412D07F5104E14D
:10758000510E7E5DD8A00CD00A0EA26F010E9F6F27
:10759000000E0101CD6F000E00017F6F000E7E6FA7
:1075A000000ECA6F400EC96F76EC1BF0E806D8A437
:1075B0003CEFAFF07F5101E147D33CEFAFF07C0EE1
:1075C000A219D8A4A1D29951D8A409D0010E996FBB
:1075D0007AC043F27BC044F2010E0101766F1E0EA9
:1075E0000001A619D8B404D01E0E07EC15F0A66F42
:1075F0004950D8B409D0600088F2BCF09551D3EC62
:1076000011F0946F010E966FA305D8A402D0010E5D
:107610009E6FA405D8B435D23BD2780EA26F010E6E
:107620009F6F36D2000E4F6E010E4E6E000E5A6ED8
:10763000000E5B6E22D282EC1FF00001B351D8A481
:1076400091D0070ED66F6000D8F3D7F0020E06EC8B
:107650001AF0000ED76F000ED66F100ED86F030E03
:10766000D96F0A0ECCECD7F03F0EC26FFD0EC36F80
:10767000070EC46F010EC56F010EC66F1E0EC76FD9
:10768000060EC86F000EC96F000ECA6F000ECB6FDA
:10769000000ECC6F000ECD6F6000D8F3CEF0C0ECC2
:1076A00006F03F0EC26FFD0EC36F070EC46F010ED2
:1076B000C56F010EC66F250EC76F060EC86F000E90
:1076C000C96F000ECA6F000ECB6F000ECC6F000E9C
:1076D000CD6F6000D8F3CEF0C0EC06F03F0EC26F65
:1076E000FD0EC36F070EC46F010EC56F010EC66F8E
:1076F0002C0EC76F060EC86F000EC96F000ECA6F42
:10770000000ECB6F000ECC6F000ECD6F6000D8F373
:10771000CEF0C0EC06F03F0EC26FFD0EC36F070E39
:10772000C46F010EC56F010EC66F330EC76F060E14
:10773000C86F000EC96F000ECA6F000ECB6F000E2F
:10774000CC6F000ECD6F6000D8F3CEF0C0EC06F029
:10775000000EF56F010E0101C26F000EAE6F010E3B
:107760000001B36F1D0E0101C16500D1000EC16F94
:107770000001F52BF505D8A43BD03F0EC26FFD0EDE
:10778000C36F070EC46F010EC56F010EC66F330EB7
:10779000C76F060EC86F000EC96F000ECA6F000ECD
:1077A000CB6F000ECC6F000ECD6F6000D8F3CEF023
:1077B000C0EC06F03F0EC26FFD0EC36F070EC46F24
:1077C000010EC56F020EC66F1E0EC76F060EC86F84
:1077D000000EC96F000ECA6F000ECB6F000ECC6F8B
:1077E000000ECD6F6000D8F3CEF0C0EC06F0BED036
:1077F000020EF519D8A43BD03F0EC26FFD0EC36F29
:10780000070EC46F010EC56F010EC66F1E0EC76F47
:10781000060EC86F000EC96F000ECA6F000ECB6F48
:10782000000ECC6F000ECD6F6000D8F3CEF0C0EC30
:1078300006F03F0EC26FFD0EC36F070EC46F010E40
:10784000C56F020EC66F250EC76F060EC86F000EFD
:10785000C96F000ECA6F000ECB6F000ECC6F000E0A
:10786000CD6F6000D8F3CEF0C0EC06F07FD0030EF1
:10787000F519D8A43BD03F0EC26FFD0EC36F070EA3
:10788000C46F010EC56F010EC66F250EC76F060EC1
:10789000C86F000EC96F000ECA6F000ECB6F000ECE
:1078A000CC6F000ECD6F6000D8F3CEF0C0EC06F0C8
:1078B0003F0EC26FFD0EC36F070EC46F010EC56F82
:1078C000020EC66F2C0EC76F060EC86F000EC96F72
:1078D000000ECA6F000ECB6F000ECC6F000ECD6F86
:1078E0006000D8F3CEF0C0EC06F040D0040EF519DD
:1078F000D8A43CD03F0EC26FFD0EC36F070EC46FFD
:10790000010EC56F010EC66F2C0EC76F060EC86F35
:10791000000EC96F000ECA6F000ECB6F000ECC6F49
:10792000000ECD6F6000D8F3CEF0C0EC06F03F0E35
:10793000C26FFD0EC36F070EC46F010EC56F020E3E
:10794000C66F330EC76F060EC86F000EC96F000EEC
:10795000CA6F000ECB6F000ECC6F000ECD6F6000B3
:10796000D8F3CEF0C0EC06F0000EF56F4F04D8A4AB
:1079700049D0000E0101C26F000EC16F000E236FCF
:10798000000E226F000E0001B36F000E4E6E000E4F
:107990000101AE6F000E506F070E0001D66F600040
:1079A000D8F3D7F0040E06EC1AF0000ED76F000ED5
:1079B000D66F100ED86F020ED96F0C0ECCECD7F02C
:1079C0007A0E0001F46FC10EF36F810EE82EFED720
:1079D000F32FFCD7F42FFAD700D00A0E0001A26FC4
:1079E000010E9F6F9051D8B407D0030EC2ECF9F08E
:1079F000040EC2ECF9F006D0010EC2ECF9F0020E52
:107A0000C2ECF9F0DC0E0101225D050E2359D8A06D
:107A100034D0000EC26F000EC16F000E236F000E37
:107A2000226F000E0001B36F000E4E6E010E0101B9
:107A3000AE6F070E0001D66F6000D8F3D7F0040ECA
:107A400006EC1AF0000ED76F000ED66F100ED86F2E
:107A5000020ED96F0B0ECCECD7F07A0E0001F46F4A
:107A6000C10EF36F810EE82EFED7F32FFCD7F42F53
:107A7000FAD700D0010E00019F6F4E04D8A408D0A1
:107A8000DAD59551010AD8B4C8D5030AD8B4CAD5F5
:107A9000000E0001CA6F400EC96F55EC1BF0E806DE
:107AA000D8A408D0010E0101CD6F000E00017F6F38
:107AB000000E7E6F000ECA6F400EC96F8CEC1DF079
:107AC000E806D8A412D07F5104E1510E7E5DD8A003
:107AD0000CD00A0EA26F010E9F6F000E0101CD6F38
:107AE000000E00017F6F000E7E6F000ECA6F400E09
:107AF000C96F76EC1BF0E806D8A43CEFAFF07F51DD
:107B000001E1A2D03CEFAFF0810EA219D8A4A6D01B
:107B10009951D8A409D0010E996F7AC043F27BC065
:107B200044F2010E0101766F0001A305D8A403D031
:107B3000010E0101A66F0001A405D8A44CD00101DB
:107B4000A605D8A448D0AEECF3F00009D8B4FBD712
:107B5000070E0001C46F0D0E35EC1CF0070E00017E
:107B6000C46F0F0E35EC1CF0070E0001C46F0E0E33
:107B700035EC1CF0070E0001C46F100E35EC1CF044
:107B800057ECE3F0410E0001F46FF00EF36F330E8B
:107B9000E82EFED7F32FFCD7F42FFAD7020E000100
:107BA000C46F0D0E35EC1CF0020E0001C46F0F0EF9
:107BB00035EC1CF0030E0001C46F0E0E35EC1CF00A
:107BC000030E0001C46F100E35EC1CF00A0E00010C
:107BD000A26F010E9F6F000E0001CA6F400EC96FA9
:107BE00055EC1BF0E806D8A408D0010E0101CD6FBA
:107BF000000E00017F6F000E7E6F000ECA6F400EF8
:107C0000C96F8CEC1DF0E806D8A412D07F5104E1B6
:107C1000510E7E5DD8A00CD00A0EA26F010E9F6F90
:107C2000000E0101CD6F000E00017F6F000E7E6F10
:107C3000000ECA6F400EC96F76EC1BF0E806D8A4A0
:107C40003CEFAFF07F5108E1510E7E5DD8B03CEFC4
:107C5000AFF0780E39EFC3F03CEFAFF0820EA2190F
:107C6000D8A47ED09951D8A409D0010E996F7AC0BA
:107C700043F27BC044F2010E0101766F1E0E00013B
:107C8000A619D8B404D01E0E07EC15F0A66F495003
:107C9000D8B409D0600088F2BCF09551D3EC11F053
:107CA000946F010E966FA305D8A402D0010E9E6FAB
:107CB000A405D8B40FD018D0830E0AD0840EA26FBA
:107CC000000E8F6F000E406E000E9A6F0BD0820E6A
:107CD000A26F08D09551010AD8B4EED7030AD8B4E0
:107CE000EDD7F5D7010E9F6F000ECA6F400EC96F1A
:107CF00055EC1BF0E806D8A408D0010E0101CD6FA9
:107D0000000E00017F6F000E7E6F000ECA6F400EE6
:107D1000C96F8CEC1DF0E806D8A412D07F5104E1A5
:107D2000510E7E5DD8A00CD00A0EA26F010E9F6F7F
:107D3000000E0101CD6F000E00017F6F000E7E6FFF
:107D4000000ECA6F400EC96F76EC1BF0E806D8A48F
:107D50003CEFAFF07F5102E133EFC3F03CEFAFF007
:107D6000830EA219D8A42DD29951D8A409D0010EFE
:107D7000996F7AC043F27BC044F2010E0101766F25
:107D800000018C05D8A408D0DC0EA619D8B404D004
:107D9000DC0E07EC15F00AD08C51D8A408D01E0ECA
:107DA000A619D8B404D01E0E07EC15F0A66F4950E2
:107DB000D8B41ED08C05D8A412D06000C0F1BCF09D
:107DC0006000C4F1BDF089EC11F06000F0F270F0D9
:107DD0006000F4F271F0010E0101526F09D06000F1
:107DE00088F2BCF09551D3EC11F0946F010E966FB0
:107DF0000001A305D8A404D0000E986F010E9E6F59
:107E0000A405D8A485D08C51D8B46ED078D0010EFA
:107E10008C6F000E9A6F010E986F010E916F78D0E3
:107E2000B751010A0101516F51C1B7F00001B851BA
:107E3000B7190101596F010E0001916F010E9E6F7C
:107E4000000E986F65D09105D8A43ED07A51701974
:107E500004E17B517119D8B402D0010E01D0000E9B
:107E60009A6F7051351804E171513618D8B42ED07C
:107E70009A05D8A42BD0000E8B6F000E8A6F000ECF
:107E8000896F000E886F000E01014D6F000E4C6F60
:107E9000000E4B6F000E4A6F00018705D8A405D075
:107EA000000E0101496F010E486F000E00018F6F37
:107EB000010E01015A6F010E00018D6F010E0101CB
:107EC000566F000E4E6F02D0000E9A6F000E00012A
:107ED000986F0A0EA26F010E9F6F9051D8A418D010
:107EE000060EC2ECF9F014D09551010AD8B48FD720
:107EF000030AD8B495D7010AD8B4A5D709D09505F7
:107F0000D8A404D0000E8C6F000E986F010E966FEF
:107F1000600080F2CCF0000E0001CD6F000ECE6F3D
:107F2000000ECF6F140ECFECE7F0A06FA005D8A421
:107F300006D0A2C0A1F00A0EA26F010E9F6F8C05A1
:107F4000D8A4E1D0000ECC6F000ECD6F000ECE6F26
:107F5000000ECF6F120ECFECE7F0E806D8A407D0E2
:107F600074C070F075C071F0010E0101526F000E07
:107F70000001CC6F000ECD6F000ECE6F000ECF6FE4
:107F8000130ECFECE7F0E806D8A409D06000DCF0CF
:107F900070F06000E0F071F0010E0101526F000E10
:107FA0000001CC6F000ECD6F000ECE6F000ECF6FB4
:107FB0000F0ECFECE7F0E806D8A466D0030EB11997
:107FC000D8B404D0020EB119D8A425D06000C0F1F5
:107FD000C9F06000C4F1CAF05A0ECB6FABEC08F0E8
:107FE000F36F060EF36105D00A0E7027000E7123A1
:107FF00004D03C0E705F000E715B715104E13E0EC7
:10800000705DD8A004D0000E716F3D0E706F010E30
:108010000101526F39D0B105D8A436D06000C0F14B
:10802000C9F06000C4F1CAF0540ECB6FABEC08F09D
:108030000009D8A415D06000C0F1C9F06000C4F1F7
:10804000CAF05A0ECB6FABEC08F0F36F090EF36178
:1080500005D00A0E7027000E7123D9D75A0E10D002
:108060006000C0F1C9F06000C4F1CAF05A0ECB6FD5
:10807000ABEC08F0F36F020EF36101D0EAD7140EF7
:10808000705F000E715BC3D7000E0001CC6F000E55
:10809000CD6F000ECE6F000ECF6F100ECFECE7F05D
:1080A000E806D8A430D0020EB119D8B42CD0B1054E
:1080B000D8A429D06000C0F1C9F06000C4F1CAF0B2
:1080C000540ECB6FABEC08F00009D8A415D06000BB
:1080D000C0F1C9F06000C4F1CAF0480ECB6FABEC40
:1080E00008F0F36F090EF36105D0640E7027000EDF
:1080F000712306D0840E01D0E80E705F030E715B11
:10810000010E0101526F0001705101010A5D000171
:10811000715101010B59D8B006D00AC170F00BC1E2
:1081200071F0010E526F000170517111D8A407D087
:10813000000E716F010E706F010E0101526F000E83
:108140000001CA6F400EC96F55EC1BF0E806D8A4B9
:108150000ED0000E986F010E0101CD6F000E0001D0
:108160007F6F000E7E6F000E9A6F000E8C6F000EF8
:10817000CA6F400EC96F8CEC1DF0E806D8A412D06F
:108180007F5104E1510E7E5DD8A00CD00A0EA26F83
:10819000010E9F6F000E0101CD6F000E00017F6F79
:1081A000000E7E6F000ECA6F400EC96F76EC1BF09A
:1081B000E806D8A43CEFAFF07F5101E102D23CEFDA
:1081C000AFF0840EA219D8A405D29951D8A409D031
:1081D000010E996F7AC043F27BC044F2010E010197
:1081E000766F00018305D8B403D08205D8A408D0E7
:1081F000C80EA619D8B404D0C80E07EC15F007D0E5
:108200001E0EA619D8B404D01E0E07EC15F0A66FEA
:108210004950D8B439D08351D8A40DD08251D8A4B4
:108220000AD0600088F2BCF09551D3EC11F0946F45
:10823000010E966F29D08305D8A412D06000C4F037
:10824000BCF06000C8F0BDF089EC11F06000F0F205
:1082500031F06000F4F232F0010E0101406F14D0F1
:108260008205D8A411D06000BCF0BCF06000C0F062
:10827000BDF089EC11F06000F0F22FF06000F4F234
:1082800030F0010E01013F6F0001A305D8A404D016
:10829000000E986F010E9E6FA405D8A4ADD0835137
:1082A000D8A4A2D08251D8B458D09ED0010E836FEA
:1082B000000E826F04D0010E826F000E836F010EDC
:1082C000986F9AD08451D8A425D0AF51D8A403D0A8
:1082D000AE51D8B43ED0010E0101B86F000E0001BE
:1082E0008D6F000E8E6F000E8F6F000E406E000EB1
:1082F0000101586F000E0001B86F06C176F007C18A
:1083000077F006C178F007C179F0010E3C6E010EDE
:10831000846F1FD03C04D8B41CD0000E846F000EB4
:108320000101B86F000E1F6F000E1E6F010E0001DD
:108330008D6F010E8E6F000E8F6F000E406E000E5F
:108340000101586F000E0001B86F0A0EA26F010EF6
:108350009F6F010E0001966F4FD09551010AD8B45E
:10836000A5D7030AD8B4A7D7010AD8B4ABD744D04D
:10837000000E836F6000C4F006F16000C8F007F1E2
:1083800001010451065D05510759D8A0E2D7010E3D
:1083900031242F6E000E3220306E6000BCF004F1EC
:1083A0006000C0F005F1010E3F6FD3D7000E826F61
:1083B0006000BCF004F16000C0F005F1010104515F
:1083C000065D05510759D8A0C4D7FF0E2F24316E82
:1083D000FF0E3020326E6000C4F006F16000C8F07D
:1083E00007F1010E406FB5D79551010AD8B4C0D737
:1083F000030AD8B4DBD7ADD7AF51D8A403D0AE5160
:10840000D8B492D08405D8A47DD03C04D8A412D08E
:1084100001011F5104E10A0E1E5DD8A00BD0000E11
:108420001F6F000E1E6F020E3C6E0C0E00018F6F50
:108430000C0E2FD0020E3C18D8A416D001011F51EB
:1084400004E1640E1E5DD8A00FD0000E1F6F000E59
:108450001E6F030E3C6E010E586F010E0001B86FC7
:10846000080E8F6F080E15D0030E3C18D8A413D039
:1084700001011F5104E18C0E1E5DD8A00CD0000E2E
:108480001F6F000E1E6F040E3C6E000E00018F6FFA
:10849000000E406E37D0040E3C18D8A433D0010132
:1084A0001F5104E1280E1E5DD8A02CD0000E1F6FB6
:1084B000000E1E6F000E586F000E0001B86F010114
:1084C00004510001785D0101055100017959D8B0CE
:1084D00009D0010E3C6E764B772B76C078F077C0D2
:1084E00079F010D0000E846F000E0101B86F000EFD
:1084F0001F6F000E1E6F010E00018D6F010E8E6F3B
:10850000010E966F00017A510201431906E1000144
:108510007B5102014419D8B407D07AC043F27BC022
:1085200044F2010E0101766F000E0001CA6F400E89
:10853000C96F55EC1BF0E806D8A41CD0000E846F60
:10854000000E0101B86F000E1F6F000E1E6F000EAF
:1085500000018F6F000E406E000E826F000E836F61
:10856000000E986F010E0101CD6F000E00017F6FAC
:10857000000E7E6F000ECA6F400EC96F8CEC1DF0AE
:10858000E806D8A412D07F5104E1510E7E5DD8A038
:108590000CD00A0EA26F010E9F6F000E0101CD6F6D
:1085A000000E00017F6F000E7E6F000ECA6F400E3E
:1085B000C96F76EC1BF0E806D8A43CEFAFF07F5112
:1085C00007E1510E7E5DD8B03CEFAFF0820E51D086
:1085D0003CEFAFF06D0EA219D8A458D09951D8A491
:1085E00009D0010E996F7AC043F27BC044F2010EAC
:1085F0000101766F000E0001CA6F400EC96F55EC85
:108600001BF0E806D8A408D0010E0101CD6F000EC2
:1086100000017F6F000E7E6F000ECA6F400EC96FA3
:108620008CEC1DF0E806D8A412D07F5104E1510E65
:108630007E5DD8A00CD00A0EA26F010E9F6F000EB7
:108640000101CD6F000E00017F6F000E7E6F000EE6
:10865000CA6F400EC96F76EC1BF0E806D8A43CEF59
:10866000AFF07F5111E1510E7E5DD8B03CEFAFF01D
:10867000640EA26F010E9F6F000E0101CD6F000E00
:1086800000017F6F000E7E6F3CEFAFF0A205D8A413
:1086900088D00F0E926F000ECA6F800EC96F8CECDF
:1086A0001DF0516E0201685104E18C0E675DD8A087
:1086B00027D05150D8A424D0000E0101C06F000E65
:1086C0000201686F000E676F0A0E0001A26F010EB3
:1086D0009F6F000EBD6F070EBC6FFBEC1EF05A0AB9
:1086E000D8A408D0000E0001BD6F080EBC6FFBECD3
:1086F0001EF001D00D0E0001926F010E0101AF6F4F
:1087000000018005D8A406D0A2C0A1F0030EA26F7C
:10871000010E9F6F000ECA6F400EC96F55EC1BF023
:10872000E806D8A408D0010E0101CD6F000E0001AB
:108730007F6F000E7E6F000ECA6F400EC96F8CEC0B
:108740001DF0E806D8A410D07F5104E1320E7E5D02
:10875000D8A00AD0040EA26F0A0EA16F010E9F6F5F
:10876000000E7F6F630E7E6F000ECA6F400EC96FE2
:1087700076EC1BF0E806D8A473D17F5103E1320EEA
:108780007E5DD8B06DD1000E0101CD6F000E0001ED
:108790007F6F000E7E6F000E0201686F8C0E676F98
:1087A0005FD1030EA219D8A42ED001012C5140088C
:1087B0000001C26F01012D51D8A0E82A0108000173
:1087C000C36F000EC56F640EC46FB0EC19F0C251D8
:1087D000456E010171514518D8B402D0010E706F79
:1087E00000018051D8A43CD18105D8A439D1A2512F
:1087F000A119D8A403D00A0EA26F02D0A1C0A2F082
:10880000010E9F6F2DD1040EA219D8A447D07E511E
:108810004008C26F7F51D8A0E82A0108C36F000E3C
:10882000C56F640EC46FB0EC19F0C251936F0101B3
:108830006F5100019319D8B409D0410E7E5D010E2D
:108840007F59D8B003D0010E01016E6F000E0001F8
:10885000CA6F400EC96F8CEC1DF0E806D8A40FD08B
:10886000400E7E5D010E7F59D8B004D008D08FEC49
:10887000FEF0506E5050D8B4FAD7A1EC1FF0000EA5
:108880000001CA6F400EC96F76EC1BF0E806D8A451
:10889000E7D0A251A119D8B4AED7B0D7050EA2190E
:1088A000D8A49FD00B0ECB6FB80ECA6F79EC16F020
:1088B00001015B51D8B403D05C05D8A40CD00001F1
:1088C000A251A119D8A403D00A0EA26F02D0A1C050
:1088D000A2F0010E9F6F000E0001CA6F100EC96F4B
:1088E00055EC1BF0E806D8B409D0000ECA6F100E84
:1088F000C96F76EC1BF0E806D8A40FD06000A4F294
:10890000CCF0600050F6CDF0600010F6CEF0000E16
:10891000CF6F0A0ECFECE7F0A96F000ECA6F200EE2
:10892000C96F55EC1BF0E806D8B409D0000ECA6F29
:10893000200EC96F76EC1BF0E806D8A40FD06000BB
:10894000A0F2CCF060004CF6CDF060000CF6CEF05A
:10895000000ECF6F0B0ECFECE7F0A86F8005D8A408
:1089600006D0A2C0A1F0030EA26F010E9F6F000EF1
:10897000CA6F400EC96F55EC1BF0E806D8A408D0AA
:10898000010E0101CD6F000E00017F6F000E7E6FA2
:10899000000ECA6F400EC96F8CEC1DF0E806D8A41B
:1089A00010D07F5104E1320E7E5DD8A00AD0A2C063
:1089B000A1F0040EA26F010E9F6F000E7F6F630E79
:1089C0007E6F000ECA6F400EC96F76EC1BF0E80692
:1089D000D8A446D07F5144E1320E7E5DD8A0D3D6D4
:1089E0003FD0060EA219D8A43BD0E00E0101205DB5
:1089F0002E0E2159D8A032D02F0E205D310E2159D4
:108A0000D8B013D020512E080001C26F01012151AE
:108A1000D8A0E82A31080001C36F000EC56F640EAC
:108A2000C46FB0EC19F0C251436E01016851431894
:108A3000D8B402D0010E676F6851D8A411D043504A
:108A4000D8A40ED065EC05F003D08FECFEF0506E8C
:108A50005050D8B4FAD7A1EC1FF002D0000119D7BA
:108A60000001A25139ECC5F0A25100EC80F0E3EF17
:108A7000AAF0DC6F3B50D8A433D06E0E0001DC1995
:108A8000D8B420D06F0EDC19D8B41CD0700EDC190D
:108A9000D8B418D0780EDC19D8B414D0790EDC19FB
:108AA000D8B410D07A0EDC19D8B40CD07B0EDC19F7
:108AB000D8B408D07C0EDC19D8B404D0810EDC19EF
:108AC000D8A407D060002CF1CCF0020ECBECF0F073
